:020000040800F2
:1000000000000120D51A0508711B05087D92010822
:10001000D5900108711B0508711B05080000000040
:10002000000000000000000000000000711B050837
:10003000711B050800000000711B0508BD83010845
:10004000711B0508711B0508711B0508711B05084C
:10005000711B0508711B0508F1A10008F9A1000832
:1000600001A2000809A2000811A20008DD9F0008F3
:10007000F19F000805A0000819A000082DA00008A5
:1000800041A0000855A00008711B0508711B050858
:10009000711B0508711B0508711B050819A20008D2
:1000A00085C9000871C8000895C9000861C8000822
:1000B00099C80008A9C80008B9C80008999900089B
:1000C0008D990008CD990008C1990008711B050899
:1000D000711B0508098301081583010821830108A4
:1000E00021A20008711B0508711B0508A5C900089D
:1000F0005DC90008711B05084DC9000869A000080A
:10010000711B0508711B0508C9C80008711B05088B
:100110002D83010839830108D9C80008F5D40408E3
:100120007DA0000891A00008A5A00008B9A00008C3
:10013000CDA000080000000000000000000000004A
:1001400000000000000000000000000055E104086D
:10015000E1A00008F5A0000809A1000845830108F6
:10016000019A0008F5990008711B0508711B050824
:10017000711B0508711B050800000000000000004D
:10018000711B0508711B0508711B0508711B05080B
:10019000711B0508711B050800000000711B050894
:1001A000000000000000000000000000711B0508B6
:1001B000711B0508711B050800000000000000000D
:1001C000000000000000000000000000000000002F
:1001D000000000000000000000000000711B050886
:10800000084A0346D0F8E4005268D3F8F010121A78
:1080100000209142B8BFC3F8F020012283F81C2150
:10802000704700BF001000E01B4B1C4A03F5727C38
:10803000016803E063452BD053F82C2F9142F9D10E
:1080400070B593F804E0427996450AD0634505D0AF
:1080500053F82C2F9142F4D06345F9D14FF0FF3003
:1080600070BD9E4684680022DEF80C50A54208D000
:1080700001320EF10C0E032AE8D0DEF80C50A542B6
:10808000F6D1DEF81050C668B542F1D150B270BDDD
:108090004FF0FF30704700BF603605080000014018
:1080A0004368426D30B49A61EFF31182502383F339
:1080B00012884168D2B2856C0B68046D23EA05030F
:1080C00023430B6082F31188436981681A68096849
:1080D00022F00102D0E908541A60826A1D605C61D6
:1080E0005A60D0E90B429C60DA600023B0F86C2043
:1080F00030BCCA620377704730B5FAB18E464FEA9A
:10810000014C034600F1C005002419680C3353F8F4
:10811000042C43F8084C41EA0C0142EA0E02AB423F
:1081200043F80C1C43F8042CEFD1D0F8C03043EADC
:108130000E03C0E93144C0F8C03030BD4FEA014EF3
:108140008C46DEE783695969B3F810C00A6830B419
:108150009C6822F0010224680A60E26822EA0C02AC
:10816000E260027D04681F2A06D9203A082065686B
:108170009040284242D0FEE70820256890402842DF
:10818000F9D1202000FA02F2A260254A1278002AD2
:1081900032D01A7F012A36D0D3F800210132C3F839
:1081A0000021EFF31181502282F312885868C9B27E
:1081B0009D6C0268DC6C22EA05022243026081F3B6
:1081C00011885A699968D3E90D40096814605061B3
:1081D000D3E90F40546090605C6CB3F8B400D46095
:1081E0000124C8621068204310601A8A1C7783F843
:1081F000FD40CB681343CB6030BC7047202000FAB1
:1082000002F2E260C1E70022D3F8040183F8FD2006
:1082100001300A68C3F8040122F001020A60EBE7AA
:10822000C801002010B40C4C6368002B11DD002045
:1082300004F1080C0146DCF8AC3003F1C0025960CF
:108240000C339342FBD1013063680CF5867C83428A
:10825000F1DC5DF8044B7047C8010020704700BF97
:10826000024B03EB401090F855047047C801002002
:10827000704700BF0B4890F86C1589B101EB4101C4
:10828000002300F27450490010B41C4650F823201B
:10829000063302B114608B42F8D15DF8044B70478D
:1082A000704700BFC80100200B4890F86C1589B1D9
:1082B00001EB4101002300F27450490010B41C4648
:1082C00050F82320063302B114609942F8D15DF8CA
:1082D000044B7047704700BFC80100200120704761
:1082E000034B00EB400003EBC00090F8850570479E
:1082F000C8010020204890F86C35002B3AD00022AD
:1083000000F274534FF02C0C2DE9F0434FF0500E57
:108310001A4E1B4D144607E053F8181B01320C602F
:1083200090F86C15914223DD197C0029F4D05F6828
:108330004FF0FE08B90AA1F580115229294498BFCF
:1083400091F8F483EFF311818EF31288D7F824901B
:108350000CFB0868C9B209F10109C8F82890D7F8E0
:10836000148048F00108C7F8148081F31188D3E71E
:10837000BDE8F083704700BFC8010020B01801209D
:108380006036050807EE900AB8EE670A704700BF2E
:10839000BCEEC00A10EE103A98B27047B4224FF407
:1083A000A57C4FF4EB71002382801F22A0F802C04D
:1083B0004FF4E17C02814FF48772C1809621828163
:1083C00044220370A0F80AC0C18143820282704730
:1083D0000346012200205A77704700BF08B5D0E954
:1083E0000B2183690B4483610AB108469047002042
:1083F00008BD00BF436A02461B681B6A5B685B7866
:1084000013F0010008BF5077704700BFC26281615E
:10841000704700BF704700BF043070470C4B93F8A3
:108420009822D3F8941202440844D2B2C3F89402BA
:1084300083F8982293F89822120605D593F898228B
:1084400082F0800283F89822024B01221A70704752
:10845000B0180120000001202DE9F84F154FD7F882
:108460009C52ED0A20D00026DFF84CA007F52879B1
:10847000B046AC19D7F8A012102352466410D1F8B8
:1084800028B04846C7F8CC82E102D8470F280BDD58
:10849000094B03F1100253F8041B013107D1934239
:1084A000F9D12546B542E4DCE802BDE8F88F661C48
:1084B000F8E700BFB018012000000020184BD3F8E7
:1084C000D412D3F8D8228A1A322A15D8D3F8EC223B
:1084D0008A4200D37047D3F8DC22E2B1106832310F
:1084E000928810B44469C3F8EC1222425DF8044B40
:1084F00018BF120482617047D3F8DC223AB193F8B6
:10850000E8021168C007928848BF12048A610022FD
:10851000C3F8EC2270473231C3F8EC12704700BF49
:10852000B0180120064AD2F8DC323BB192F8E812CA
:108530001A68C9079B8848BF1B04936100207047D5
:10854000B0180120044B4FF4007C0020D3F8F8321F
:10855000A2F800C00B607047B018012000207047DF
:10856000012070470120704700207047134BD0F85E
:10857000D8105B68D0F8E02010B50446581A824243
:1085800000DC22B9D4F8E4200A44C4F8DC2094F8D2
:10859000D020C4F8D830012A05D0D4F8D430013323
:1085A000C4F8D43010BD04F1E801201D0FF026F905
:1085B000D4F8D4300133C4F8D43010BD001000E03A
:1085C000CB070AD490F82830012B08D0C368B3F148
:1085D000807F03D9012303777047704770471B4A98
:1085E000D2E9CA1310B5B1EB930F8CB04FEA9302E6
:1085F000446A4FF0020306D252085B0091429BB2DC
:1086000001D2FF2BF8D9C268A380B2F1807F1BD9B9
:108610000122002301A94FF0B70C027720460492F3
:108620008DF814208DF828208DF804C00B93CDE927
:10863000021302A9CDE90633CDE908330FF0DEF8C5
:108640002268136A002BFCD10CB010BDB0180120B9
:1086500030B590F828308BB00446012B05D0407F10
:1086600048B1002363770BB030BD456A2B681A7B95
:1086700022BB637F13B901200BB030BD1249022029
:10868000002301220290081F8DF80C208DF8202075
:108690000993CDE9001069462846CDE90433CDE9B8
:1086A00006330FF0ABF82A68136A002BFCD1074B96
:1086B0005B7C03F0010383F00100D3E71B6A002B0E
:1086C000D7D00020CFE700BF14000020000000201A
:1086D0002DE9F0411F4F8AB0044690F82820A7F1F9
:1086E0000408A7F11406437F012A06D00BB100232A
:1086F000637701200AB0BDE8F081656A2A68117BC2
:1087000009BB002BF5D00023694628460993CDE923
:108710000433CDE9063301238DF80C308DF8203079
:108720000223CDE9007802930FF068F82A68136AF3
:10873000002BFCD1737C03F001036377002BD8D0AE
:1087400094F82820D0E7126A002AD7D1002BD0D085
:10875000D9E700BF14000020244A002330B50446A6
:1087600095B0101D224D0693019002200B9310939B
:10877000139311930290207F009200280495CDE975
:108780000E334FF001038DF80C3007938DF8203035
:108790008DF834308DF8483002F10803A2F1080258
:1087A000059314BF052304230A920C93114B0993DC
:1087B000636A1A68136A002BFCD1A0B10E480A0E36
:1087C00000F11A0342760A0A9970080C69465A7039
:1087D0001870606A0FF012F8636A1A68136A002B47
:1087E000FCD115B030BD054BEDE700BF20000020E7
:1087F000F5830008D1830008000000201900002044
:1088000010B594B004465022074968464AF0E6FC89
:108810006946606A0EF0F2FF636A1A68136A002BF9
:10882000FCD114B010BD00BFA83A0508F8B5054644
:10883000406A0068046A002CFCD1287F002839D0E7
:10884000A8690527254E4FEA106C254C2E3606F8F0
:1088500001CC6763B0704FEA104C000A012B86F818
:1088600000C070704FF000000E6826641668A664A1
:108870002E63A06524D0022B1BD1536801222065F2
:108880001E444968E365174B84F84C0061652E630C
:1088900084F860206366144B697F03F11402686AF0
:1088A000002914BF194611460EF0A8FFEB6A73B1F8
:1088B000286BF8BD04200A4C0C4E6063A869C9E718
:1088C000084A84F84C306065E0652265E3E76B6A2E
:1088D0001A68136A002BFCD1EAE700BF00000020F1
:1088E00000000120DD830008040001202D0000208D
:1088F00000B583B08161019201A9049A009301231C
:10890000C2626A46FFF792FF03B05DF804FB00BF46
:1089100070B51D46436A94B006461B681C6A002C5D
:10892000FCD13A4B02204FF0010C0694029003F167
:108930003C008DF80CC0009003F1400001903448D9
:10894000049003F134000590307F00284BD00B9247
:108950000A0E36338DF8204003F8012C05220C95C1
:108960008DF834C08DF848C013940792CDE90944BE
:10897000CDE90E44CDE910440A0C9970254C090A42
:108980001A705970706AD4E9CA32B3EB920F4FEA89
:1089900092014FF0020206D2490852008B4292B275
:1089A00001D2FF2AF8D9737F8280D3B905A90EF0CE
:1089B00025FF706A03681A6A002AFCD10222D4E9F2
:1089C000CB34B4EB930F4FEA930106D2490852001F
:1089D0008C4292B201D2FF2AF8D98280284614B084
:1089E00070BD6946E3E70B92042235338DF8200011
:1089F0000C958DF834C08DF848C013900792CDE9DE
:108A00000900CDE90E00CDE91000B5E70000002017
:108A1000F5830008B01801208369F0B593F8DC20D5
:108A20008BB00546012A27D0023A012A2FD893F8A5
:108A30004C21EC46D3F89C1062F07F03154C0B7070
:108A40008669D6F8A0305F1C0FCCACE80F00D6F8D2
:108A50009C30CDE900370FCCACE80F0094E8030060
:108A60008CE80300694606F110000EF0C7FEAB6902
:108A700019690A6A002AFCD1D3F8A0305A8852BA80
:108A8000EA819A8852BA2A82DB885BBA6B8201201B
:108A90000BB0F0BDF83A0508F0B590F8DC308BB0BB
:108AA0000446D0F8A060012B4BD015D8D0F89C30EC
:108AB0004FF0FF3205211A605A609A60DA60D0F8F0
:108AC000E030C0F8F010B3F57A7F54D8032380F873
:108AD000DC3001200BB0F0BD023B012BF9D890F83F
:108AE0004D31EC46D0F89C2063F07F03384D137075
:108AF000D0F8A0305F1C0FCDACE80F00D4F89C304C
:108B0000CDE900370FCDACE80F0095E803008CE805
:108B10000300694604F110000EF070FE2269136A2A
:108B2000002BFCD1738801205BBAA4F8D030B38845
:108B30005BBAA4F8D230F3885BBAA4F8D4300BB097
:108B4000F0BD90F84C2190F84D319B1A5B10013329
:108B5000DBB236F8132006EB430653BAA0F8D03048
:108B600073885BBAA0F8D230B3885BBAA0F8D4306F
:108B700001200BB0F0BD03691A7B2AB35B691BB3FC
:108B800090F8983003B390F84C310122D0F89C0053
:108B900063F07F03C4F8A4400E49037094F84D318C
:108BA00094F84C0184F800211B1A84F8DC20D4F8D6
:108BB000A0200733C4F804110132D4F89C10C4E992
:108BC0003E23C4F8F41084E7022384F8DC3080E705
:108BD000F83A0508018000082DE9F041304F07EB15
:108BE000401898F854340BB9BDE8F08100EB8003CD
:108BF0000E460021044607EB4313450193F8362641
:108C000083F8361688F83A244AF022FDB8BB3D4472
:108C10002448A5F8386400EB44104AF01DFD3B7869
:108C2000D5F85024A3B1D5F83C140124D2F8AC30C7
:108C30008C4003F1C001420010F4004F90B202D109
:108C40005A6822435A600C339942F4D1BDE8F0814E
:108C5000D5F83C140124D2F8AC3001F1100203F134
:108C6000C0019440420010F4004F90B202D15A6803
:108C700022435A600C339942F4D1BDE8F0810A4B8B
:108C800093F8AC2302EB420203EBC203234493F8B4
:108C90005963002EBBD0012388F83A34B7E700BFF0
:108CA000C801002000060020B01801202DE9F84F6F
:108CB000374D2B7813B90120BDE8F88F354F05F5F6
:108CC000876A05F634360024D7F8D4B24FF6FE7919
:108CD0004FF6FF7815E0B0F5606F4AD0B081B0EB89
:108CE00008012D4B4FF05C005A4618BF012100FBD4
:108CF00004300EF099FB01340AF1200A1436082CD6
:108D000031D0D5F81C2FA2422DDDDAF81800DAF8A0
:108D10000420D0E93D014AF04BFC484597F8352343
:108D200014D0542A04D1B7F838230132A7F83823D5
:108D3000D5F83C2B404502F10102C5F83C2BCAD1C5
:108D4000D5F8382B0132C5F8382BC8E7542AD2D1D0
:108D5000B7F83A2301340AF1200A14360132082CFC
:108D6000A7F83A23CDD10123012085F8383CBDE88E
:108D7000F88F97F8AC2302EB420207EBC2022244C1
:108D800092F859230D2AA9D18022B277A7E700BF14
:108D9000C8010020B0180120040E00202DE9F8437E
:108DA0000FF060FB2F4E4FF0000C0746DFF8BC8041
:108DB0002D4C716800294ADD00234FF486701D4652
:108DC00000FB0362013392F80521994245EA02054E
:108DD000F6D145EA0C0C5FFA8CF9D8F80430C3F3ED
:108DE00008038BBBEFF3118373BB4FF0E02CD4F877
:108DF000D432DCF81810D4F8D4229342F7D1D4F846
:108E0000B0239142F3D8D4F8B4C34FF47A7202FB82
:108E10000CF0401AB0FBFCF002FB0300C31BB3F5DF
:108E2000FA6FCCBF4FF0000C05F0010CBCF1000F45
:108E3000BFD1B9F1000F04D00B4B93F83523542A5E
:108E400008D04846BDE8F8830FF0DEFAE6E7E146D1
:108E50000025C2E7B3F83C2348460132A3F83C237F
:108E6000BDE8F883C8010020B018012000ED00E043
:108E700010B5044649F03AFC0146204689B2BDE8E7
:108E80001040A9E638B50B4D00EB400005F27453D5
:108E9000C40003EBC0032C4493ED027AD3ED037AB4
:108EA000E7EE007AB0EE670A49F020FCD4F874359A
:108EB000186038BDC80100202DE9F0414AF0A8FB38
:108EC00080B31B4F7D68002D12DD3846002410F85A
:108ED000086BA046013416B1037F012B1DD04269F7
:108EE000AC4200F58670136843F001031360F1D1C2
:108EF0000FF0B8FAD7F8204F002C0CDD0D4B03EB28
:108F0000C4041968083333F8042CC8689C4242EA48
:108F10000002CA60F5D1BDE8F08180F8FC80FFF75F
:108F2000BFF8DCE742F098FD0028CAD1BDE8F08127
:108F3000C8010020EC1000200C4AF8B513685569F0
:108F40002B4003EA000555617DB1094F0126B5FAB2
:108F500085F4C4F11F0407EB840306FA04F4D3F884
:108F6000BC0303689847A543F1D1F8BD003C01401C
:108F7000B01801200269C3682DE9F04712EA03091D
:108F80002AD005460E464FF000474FF00008B9FAC8
:108F900089F327FA03F21B3BD24309EA02092A614B
:108FA000042B16D8DFE803F03B30251A0300B36A20
:108FB000002B3FD003F1FF3AC6F828801FFA8AFA47
:108FC000746A34B123682046514698476468002C7F
:108FD000F8D1B9F1000FDAD1BDE8F0877068002848
:108FE000F7D0696B036889B29847B9F1000FCED109
:108FF000F2E7B0680028ECD0A96B036889B2984703
:10900000B9F1000FC3D1E7E7F0680028E1D0E96BC0
:10901000036889B29847B9F1000FB8D1DCE730692D
:109020000028D6D0296C036889B29847B9F1000F9F
:10903000ADD1D1E7E96A1FFA81FAC1E7836910B5BA
:109040001A4C04EB8303D3F81C043EF077F9B4F810
:109050003C340C2B0ED8DFE803F0070D0D0D220D6C
:109060000D0D1B0D0D0D1400D4F8FC23D36823F453
:109070000073D3600122002384F8392484F83E343D
:1090800010BDD4F8FC23D36823F48053D360F1E7F8
:10909000D4F8FC23D36823F40063D360EAE7D4F860
:1090A000FC23D36823F48063D360E3E7B018012086
:1090B00080699C303EF042B9830AA3F58013522B9D
:1090C00052D8F0B504466A4885B0034493F8F403D7
:1090D0000D2847D8674D860105EB8013D3F84074FF
:1090E000A7423FD00139C3F8404489B2C3F84C14B9
:1090F000D5F82C13B1FBF2F2013AC3F84424002254
:10910000C3F85024C3F84824C3F8542493F87D24AA
:1091100002F0FF014AB358490223AF1901EB801155
:10912000204687F87D3404313EF072FE012387F833
:109130007D34524B9C421BD0B4F1804F18D0A3F524
:109140007C439C4275D003F580639C4271D04C4AAD
:1091500003F57C439C4218BF944249D003F57053F9
:109160009C4245D005B0F0BD704783F87C14D2E72F
:1091700000234FF48051AA19CDE9001392F87C1412
:109180000129CDE90233EDD00221D2F840040124B7
:1091900082F87D143B4987683940816082F87D44BC
:1091A00082F87C340023AA19CDE90033029392F8A7
:1091B0007C34012BD6D0D2F8403402212F4882F8DB
:1091C0007D1483425A6899684ED000F580608342CE
:1091D0004AD022F0700221F08001354401205A600B
:1091E0009960002385F87D0485F87C3405B0F0BDD6
:1091F00000214FF48053CDE90031AB1993F87C2462
:10920000012ACDE90211ADD0D3F84004022283F83F
:109210007D241C4A87683A4082601B4A83F87C148C
:109220000121944283F87D14BCD0154B9C4299D106
:10923000B8E700224FF48051AB19CDE9001293F842
:109240007C140129CDE902228CD00221D3F84004FC
:10925000012483F87D140B4987683940816083F8C5
:109260007D4483F87C249DE722F47002B1E700BFBF
:1092700060360508B0180120F01C012000000140F4
:10928000000C00408800FEFF000401402DE9F84377
:10929000DDF820800F4616460021202204461D4698
:1092A0004AF010F8B8F1000F0CD0D8F80030B8F838
:1092B0000A20E3811B0C2382D8F804306282E38207
:1092C0001B0C2383384647F005FDF30619D4431ED3
:1092D000B8B107EB000C01E0013B12D31CF801ED23
:1092E000BEF12E0FF8D1C01A03F10109421EB94494
:1092F000032AA8BF0322082BA8BF082390461A46BA
:1093000006E008280246B9464FF00008A8BF082228
:109310004FF02033394620462360636049F05EFFFA
:1093200004F108031748424649462081A0721846B6
:1093300049F054FF04F1FF3C0346E21D1CF8011FF5
:10934000A1F1610E2039BEF1190F98BF8CF8001001
:109350006245F3D1184604F10B0110F8013BA3F16B
:109360006102203B192A98BF00F8013C8842F4D1E1
:10937000182365832D0CE6722373099BA582E36194
:10938000BDE8F883202020002DE9F04FDFF88C9411
:1093900087B0D9F8D402C9F8D802002B00F0DA80DF
:1093A0001344154601F1200601F5FE77DFF870A49D
:1093B00003931FE0002D63D0D9F80423AA4200F0E4
:1093C000CD80D9F80023AA4200F00281D9E9C22158
:1093D000AA424CD8A94200F2CF81691A184641F03E
:1093E000C1FB0135039B06F5007607F500779D422A
:1093F00000F0B080D9F81043A6F12003AC42D9D8D0
:109400002C1BD9F82083E208D8F8301004F00704A8
:1094100002328A4203D3D8F838108A420DD9414625
:1094200010460593049241F06DFB8046DDE904236C
:10943000002800F0C181C9F8200398F80410002921
:1094400040F03F81D8F828B0BBF1000F00F0AD81AB
:109450001846D8F830304FF40071D21AD8F80C30D2
:1094600004EBC20203EB42224346D847B9E7A942C4
:10947000B3D918464FF40072002149F023FFB0E73A
:109480004FF400722946184649F01CFF802203461B
:10949000D94886F89E210C2286F8A221D9F800131B
:1094A000D9F8F8228142C3F8C611C3F8CA2100F3E3
:1094B0006881D24B013AD24C83FB0103C81784FB6D
:1094C00001C40B44C0EB6313C0EB2430CD4C84FBD0
:1094D00003C4C3EB831C86F8A1018010A1EB0C012F
:1094E0001C4420F03F000131014386F8A011D91738
:1094F000C1EBE4110B4486F89F31BF4B9A4200F355
:109500004C81BE4BBE4883FB0213D11780FB024047
:109510001344C1EB6313C1EB2031BA4880FB034015
:10952000C3EB831486F8A5118910121B184421F08F
:109530003F0101320A4386F8A421DA17C2EBE0109A
:10954000034486F8A331552386F8DE31AA2386F832
:10955000DF3146E7002007B0BDE8F08F4FF0FF3263
:109560000024A6F11C00049383F8EC21214683F823
:10957000ED2183F8EE2183F8EF2152221A705A7000
:1095800061229A7083F8E7214122DA7083F8E6219C
:10959000722283F8E42183F8E521D9F81823C3F86F
:1095A000E8214FF4F07249F08DFE049B5522C6F875
:1095B000D041C6F8D441C6F8D84183F8FE216FF0F7
:1095C000550283F8FC4183F8FD4183F8FF2108E749
:1095D0008D4C00214FF40072184649F073FE03468B
:1095E0004FF0000C022203CC46F8191CEB2146F880
:1095F0001D0C082006F8201C582106F81F1C90217D
:1096000006F81E1CF8211A7383F80BC006F8130C19
:109610009A7383F80FC006F8102C06F80B1C83F819
:109620002C20D9F80013D9F8F82283F819C0521A5F
:1096300083F81BC083F81DC01A6283F81EC083F82C
:109640001FC083F82DC083F82EC083F82FC0D9E93E
:10965000C212521A80215A623F221A764FF0FF320C
:109660009A763E221A77012283F8302083F831C09F
:1096700086F820102921654B86F82210942186F85F
:10968000260086F823100E21614A86F824100D2149
:1096900086F82510552186F8DE11AA2186F8DF11FB
:1096A00003CBC6F82B101988C6F827009B78A6F8BC
:1096B0002F1086F8313003CAC6F83200C6F83610CB
:1096C0008FE64FF400721846002149F0FBFDD8F8F0
:1096D00040200346002C76D1002A00F0A380D8F861
:1096E000303011224B49CDE90044FFF7CFFDD8F8C7
:1096F00040301A6C002A00F0A1801B6BCDE90044B9
:109700001122454930464FF4E07BFFF7BFFD06F1DB
:109710002003D8F84480B8F1000F3FF462AE03F1A3
:1097200020049B44049523464446984610E05CF888
:109730001C1B0025236BCDE900C5FFF7A7FDABEB94
:109740000803A46C08F12008002C18BF1F2B51D966
:109750002379A44604F11C0E1122A8F12000002B4D
:10976000E5D162792569236B42F021022168CDE9B8
:1097700000E5FFF78BFDE2E7A91A184641F0F2F980
:109780002FE6FF23013A86F89F3186F8A13186F84B
:10979000A031194B9A427FF7B4AEFF2386F8A3316C
:1097A00086F8A53186F8A431CDE6594618464FF41F
:1097B000007249F087FD14E6A6F1240343F804AFD4
:1097C0009F42FBD10DE6002AD8F844800CBF01224D
:1097D0000222C2EB0414B8F1000F3FF402AE42467D
:1097E000013C926C002C01DD002AF9D190464FF427
:1097F000007B90E7049DF4E5FF03FB0083200882D3
:10980000975545418180808088B6050894B6050843
:10981000A0B6050880B6050884B60508B018012072
:10982000DEADBEEF23460822D9F8FC124FF4F07BE0
:10983000CDE90044FFF72AFD33466AE72346CDE928
:1098400000445DE730B490F8443000F10801484A24
:10985000012BC2F800186ED083684649DC68464D7B
:1098600024F46004AB42DC60DC6844F46004DC6037
:109870009C6B24F440149C639C6B44F480149C63A4
:109880009C6B24F4F8449C639C6B44F488449C6374
:109890009C6824F470249C609C689C609C6824F400
:1098A00040149C609C689C605C6824F480645C60EC
:1098B0005C6824F480545C605C6901EA04015961CD
:1098C0005969596147D0DC682A4924F0E064DC60BA
:1098D000DC6844F0E064DC609C6B24F440149C631E
:1098E0009C6B44F480149C639C6B24F478249C63EC
:1098F0009C6B44F410249C639C6824F470249C604A
:109900009C689C609C6824F440149C609C689C60EB
:109910005C6824F480645C605C6824F480545C605F
:109920009C692140144C9961A3429969996118D0AE
:10993000002380F844301148114B848DC18D408D37
:10994000091BC2F80848C2F8040893FBF1F330BCC5
:10995000C2F80C3870470B4C616841F4000161603B
:10996000B1E708494B6843F400034B60E0E700BFF0
:10997000B018012000F0FFFF00200140007AF01F26
:109980008038010000230140704700BF01483DF0CE
:10999000E5BE00BFD4200120084810B4D0F8243818
:1099A000D0F8584899691A682CB1234600F624006B
:1099B0005DF8044B18475DF8044B7047B018012060
:1099C00001483DF0CBBE00BF34210120084810B44F
:1099D000D0F88438D0F8B84899691A682CB1234671
:1099E00000F684005DF8044B18475DF8044B70479F
:1099F000B018012001483DF0B1BE00BF9421012004
:109A0000084810B4D0F8E438D0F8184999691A68B1
:109A10002CB1234600F6E4005DF8044B18475DF8CE
:109A2000044B7047B01801200328D4BF4FF0000C3E
:109A30004FF0010C2DE9F047B0F1FF3F14BF644631
:109A40004CF0010482B0002C71D1444E00EB400C6C
:109A50004FEA400E06EB4C1CDCF82458002D62D077
:109A60009CF86578202F5ED1AD6915F400455AD178
:109A70009CF86478012F56D00A9F9BB24FF0220ABF
:109A80004FF04009CCF84878354FD6F890898CF8DB
:109A900065A88CF86698CCF86858ACF84E38CCF8C5
:109AA00050780127BCF84E388CF864789BB22D4F63
:109AB000FF2BCCF858784CD8BCF84E384FF00077D4
:109AC0009BB286442848CDF800804FEA410900EB5C
:109AD0004E1006EB4E1849461430A8F84C3819239E
:109AE00042F06EF940BBD8F8242849EA0701DFF8B4
:109AF00088C0536898F84C7803EA0C031B4CD8F8DC
:109B000058680B4343EA07431C43194B9E42546079
:109B100088F8640803D0174B9E4218BFF4251368D9
:109B200001241D431560204602B0BDE8F0870024E3
:109B3000204602B0BDE8F087B6F8943900222046EE
:109B4000013388F864289BB2A6F8943902B0BDE8C6
:109B5000F087FF234FF08077B3E700BFB0180120F4
:109B60000000FFFFE5250408C0200120002400803C
:109B70005944040859270408009800FC30B40469CB
:109B8000002341684025E46882690C3154624469CD
:109B90009560536093631160C2E90333C2E90533F2
:109BA000C2E90733C2E90A33C2E90C3384B1C2699E
:109BB000E068936350621160C2E90133C2E9033384
:109BC000C2E90533C2E90733C2E90A33C2E90C33FB
:109BD00030BC7047114A037A0168D35C10B4CC588A
:109BE000CA1824F00104CC501368DB07FCD4037DB1
:109BF0001F2B09D9203B20225DF8044B02FA03F306
:109C000043F01803CB60704720225DF8044B02FA42
:109C100003F343F018038B60704700BF3CB705089F
:109C2000F0B50668356A00295CD12F68AC68D6F8B3
:109C300018E0002F5FD0364B3B40B3F1005F61D09E
:109C400007F01F0104F11F0327F01F02194421F040
:109C50001F01BFF34F8F00290BDD114402F12003D8
:109C6000DFF8B0C08B42CCF868221A4603F120031B
:109C7000F8D1BFF34F8FBFF36F8F03684FF480624B
:109C8000CEF80470CEF814205B69CEF8204043B3C0
:109C90006868F669002837D01D4B0340B3F1005FB8
:109CA0001AD000F01F0220F01F011F32224422F0C0
:109CB0001F02BFF34F8F002A0ADD0A4401F120037F
:109CC000144D9A42C5F87012194603F12003F8D1D9
:109CD000BFF34F8FBFF36F8F4FF48063706073617A
:109CE0003462F0BDEC69002CFBD06F691435D6F8F6
:109CF00018E0002F9FD1084A3346CEF81470CEF8F2
:109D00000420C1E73346B9E7044B70617360E7E7AD
:109D10000000FFFF00ED00E04400002048000020AC
:109D2000F8B507680646D7E90454002C50D0A06166
:109D30002B7D1F2B39D82022286802FA03F343F029
:109D400018038360237D1F2B3AD92022203B02FA7F
:109D500003F3226843F01803D36063680022696844
:109D60000A601A601A6842F010021A60BA69297A09
:109D700045F032F9FA69217A206845F02DF92A7AFE
:109D80002A492F6833688D5C5A687B59206843F0F4
:109D900001037B51237AC95C435843F001034350CC
:109DA000536843F003035360F8BD203B202228682A
:109DB00002FA03F343F01803C360237D1F2BC4D8BA
:109DC000202202FA03F3226843F018039360C4E7E9
:109DD0002A7D6B681F2AA8611FD82021286801FAF4
:109DE00002F242F0180282600021BA691960196813
:109DF00041F010011960297A45F0EEF82A7A0B49F2
:109E000033682868895C5A68435843F0010343501B
:109E1000536843F002035360F8BD203A20212868BC
:109E200001FA02F242F01802C260DDE73CB7050811
:109E300010B1036882889A61704700BF18B18388A7
:109E400002681B049361704708B51D200EF0A8F846
:109E500008B183794BB11E200EF0A2F808B18379C6
:109E600003B108BD5523C38008BD5523C380F2E765
:109E7000D3B2012B23D802EB42024FF0000C70B595
:109E80004FEA820E0F4C634622460EF1080504E0AD
:109E90000133172B11D012F81CCF6045F8D192F87E
:109EA00001C08C45F4D15659002EF1D0C3EBC30349
:109EB0000EEB83030433E01870BD002070BD00205A
:109EC000704700BFA03B050810B40C4C002304F6FB
:109ED000981C01E0152B0CD003EB430201331CF856
:109EE00002108142F6D122445DF8044B92F99A099E
:109EF00070474FF0FF305DF8044B7047B0180120F9
:109F0000D3B2022B21D802EB4202002330B54FEA34
:109F1000820C0F4D0F4C2A460CF10C0E04E001335D
:109F2000172B10D052F82C4FA042F8D114798C4244
:109F3000F5D152F80E40002CF1D02C2202FB03C3C5
:109F40000833E81830BD002030BD0020704700BF46
:109F50006036050800000140002838D0002330B5E5
:109F60001B4D90F804C005F6981401E0152B2CD079
:109F700003EB43020133A15C6145F7D12A44046835
:109F800090F805E092F99A39DAB2022A1DD803EB6B
:109F90004303104810494FEA830C024600230CF19A
:109FA0000C0504E00133172B0FD052F82C1F8C4204
:109FB000F8D111797145F5D151590029F2D02C22EF
:109FC00002FB03C30833184430BD002030BD704786
:109FD000B018012060360508000001400348D0F8A1
:109FE00090300BB180301847704700BF000001204F
:109FF0000348D0F8B4300BB1A4301847704700BF05
:10A00000000001200348D0F8D8300BB1C830184701
:10A01000704700BF000001200348D0F8FC300BB1AE
:10A02000EC301847704700BF000001200348D0F80B
:10A03000203113B100F588701847704700000120E7
:10A040000348D0F8443113B100F59A7018477047AF
:10A05000000001200348D0F8683113B100F5AC705E
:10A0600018477047000001200348D0F88C3113B125
:10A0700000F5BE7018477047000001200348D0F873
:10A08000B03113B100F5D0701847704700000120BF
:10A090000348D0F8D43113B100F5E2701847704787
:10A0A000000001200348D0F8F83113B100F5F47036
:10A0B00018477047000001200348D0F81C3213B144
:10A0C00000F5037018477047000001200348D0F8DE
:10A0D000403213B100F50C701847704700000120A2
:10A0E0000348D0F8643213B100F515701847704773
:10A0F000000001200348D0F8883213B100F51E702B
:10A1000018477047000001200348D0F8AC3213B163
:10A1100000F5277018477047000001200138074BF1
:10A12000074A00EBC00003EB8000D0F880009042AB
:10A130000CBF9520962041F0E9BF00BF0000012030
:10A140000060024001382DE9E84100EBC000134DEA
:10A150001E46134B05EB800590460F46D5F8800050
:10A1600098420CBF9520962041F0D0FF95F99500BC
:10A170004FEA9811C5F89070C5F8986041F0CAFE92
:10A1800095F99530002B07DB03F01F0001225B09D6
:10A190000449824041F82320BDE8E8810000012005
:10A1A0000060024000E100E0800AA0F58010522823
:10A1B00008D8054B184490F8F4330D2B02D8034A05
:10A1C000D056704700207047603605082CB7050848
:10A1D00058B183884FF00042B3FA83F332FA03F3A5
:10A1E00003D002490A6813430B607047003C0140EA
:10A1F0000120FEF7A1BE00BF0220FEF79DBE00BFFA
:10A200000420FEF799BE00BF0820FEF795BE00BFF0
:10A210001020FEF791BE00BF4FF47870FEF78CBEA1
:10A220004FF47C40FEF788BE30B1036882881B691A
:10A230001A4214BF01200020704700BF2DE9F04FE3
:10A24000884683B004461746002800F0BC800268A8
:10A250005E4B13449B0A5E4AC8F3411B134493F8B8
:10A26000C40741F053FFC8F38103B4F804E008F0D9
:10A270000302256801939EFAAEF0B0FA80F002F175
:10A28000FF3A3EFA00F35ED00126032103E00130DD
:10A290003EFA00F357D006FA00F313EA0E03F6D0A5
:10A2A000D5F8009093FAA3F4B4FA84F493FAA3FCDB
:10A2B000BCFA8CFC6400BAF1010F4FEA4C0C01FAB5
:10A2C00004F402FA0CFC29EA040444EA0C042C60AD
:10A2D00049D9D5F80C9093FAA3F4B4FA84F493FA1C
:10A2E000A3FCBCFA8CFC6400022A4FEA4C0C01FA75
:10A2F00004F40BFA0CFC29EA040444EA0C04EC60B4
:10A30000C5D193FAA3FCBCFA8CFC1C0ABCF1070F64
:10A3100041DC2C6A93FAA3FCBCFA8CFC93FAA3F3FD
:10A320004FF00F09B3FA83F34FEA8C0C01309B0016
:10A3300009FA0CFC07FA03F324EA0C0423432B620A
:10A340003EFA00F3A7D1BAF1010F09D86B68C8F340
:10A35000001823EA0E030EFB08FE4EEA03036B60AF
:10A3600003B0BDE8F08FD5F8089093FAA3F4B4FADF
:10A3700084F493FAA3FC6400BCFA8CFC01FA04F4A4
:10A380004FEA4C0C29EA0409019C04FA0CFC49EA46
:10A390000C04AC609DE7D5F824C094FAA4F9B9FA8E
:10A3A00089F994FAA4F30F24B3FA83F34FEA8909E5
:10A3B0009B0004FA09F907FA03F32CEA090C4CEAAA
:10A3C00003036B6263E74FF0FF3344E70000FEBF17
:10A3D0006036050800B131E770472DE9F84FC04FEE
:10A3E0006023064603FB0073D3F81048002C00F0EE
:10A3F0006B81D3F818A8BAF1000F04D09AF8063090
:10A40000002B40F06181602303FB0673D3F81C58D6
:10A410001DB1AB79002B40F05781731CDBB2BAF150
:10A42000000F04D015228AF807308AF8062015B1EB
:10A430001622EB71AA714FF06009207E41F066FE92
:10A44000294609FB06F9504646F092F8042207EB2C
:10A450000908504698F82038002B14BF3E211E21D1
:10A46000FFF7B8FF98F8203828469E4D002B4FF094
:10A4700004024D4414BF3E211E21FFF7ABFF4C22C6
:10A480000021284648F01EFFD8F810389FED967A34
:10A49000B0EE084A5B68F7EE003AB8F822984FF041
:10A4A000000EC8F8243840F21458904B9FED905A93
:10A4B0009A68904BC2F38222134493F8CC27D7F8C2
:10A4C0002C33D34007EE903AF8EE677AC7EE275A5E
:10A4D00007EE909A9FED887AF8EEE77AC7EE274A62
:10A4E000DFED867AB0EE007AE5EE877AA5EE875A40
:10A4F00025EE844A37EE856A74EEE72AB9F5C87FFF
:10A500000EF1010CD5BF642332234FF496707820EE
:10A5100007EE90CAD8BF4FF4167A0344C8BF4FF471
:10A52000827AB8EEE77AD8BF414607EE903AC8BFC4
:10A530004FF4FA7127EE257A01EB0A03F8EEE76A89
:10A5400086EE873A73EE636AFCEEE67A17EE902A9F
:10A5500007EE90AAB8EEE73A07EE903AF8EEE77AFF
:10A5600023EE243AC3EE276A36EEC53A72EEE66A67
:10A57000C3EE077A77EEE37AFCEEE77A17EE901AED
:10A58000C6EE877A77EEE37AFCEEE77A17EE903A3A
:10A5900003F1020A0AEB010BF0EE466A07EE90BAED
:10A5A000F8EE677AE7EE276AF4EEE64AF1EE10FA83
:10A5B00000F38E805FFA82FABAF10F0F00F28A8000
:10A5C000323807EE900AF8EEE77A77EEC47AC7EEF3
:10A5D000876AFCEEE67A17EE900A5FFA80FABAF123
:10A5E0000F0F77D81FFA81FABAF1FF0F72D81FFA4E
:10A5F00083FABAF1FF0F6DD812054AEA0E7302F022
:10A600007F620004134300F47F003D4A034302EAE3
:10A6100001210B43602000FB067600272846C6F880
:10A6200028380123C6F82C78C6F83038C6F83478B4
:10A63000C6F83878C6F84078C6F8447845F082FC09
:10A6400096F86538202BD9B21AD196F86438012BC8
:10A6500016D0242386F86538D6F824381A6822F0F4
:10A6600001021A601A6822F480521A601A681A608D
:10A670001A6842F001021A6086F8651886F8647854
:10A68000002194F91A0041F045FC94F91A30A27E99
:10A69000002B07DB02F01F0101225B098A401949E8
:10A6A00041F82320002194F9190041F033FC94F97A
:10A6B0001930627E002B07DB02F01F0101225B09CB
:10A6C0008A40104941F82320BDE8F88FE64615E797
:10A6D00001315FE7BCF10F0FF8D100239AE700BF0B
:10A6E000B0180120D4200120286B6E4E00380240A3
:10A6F00000001643603605080024744900007042CB
:10A7000000FFFF0000E100E02DE9F047814DC0EBC4
:10A71000001605EBC606D6F8D839002B00F0B88035
:10A720000446070196F8480A41F0F0FC96F8483ACA
:10A73000012203F01F015B09013B8A40032B0AD869
:10A74000DFE813F0DC000400E200D60072494B6A37
:10A7500023EA02024A623B1B04F1010905EBC30331
:10A760005FFA89F993F8DC090DF01AFC064618B176
:10A77000122380F8079083713B1B05EBC30393F80A
:10A78000DD090DF00DFC824618B1132380F8079007
:10A7900083713B1B05EBC30393F8DE090DF000FC4E
:10A7A000804618B1142380F8079083713C1B5046F3
:10A7B0002E2105EBC40595F8E029FFF70BFE95F86F
:10A7C000E1290E214046FFF705FE95F8DF292E21ED
:10A7D0003046FFF7FFFDD5F8D83950491A688B424B
:10A7E00022F040021A6055D04D4A934269D002F5DA
:10A7F0008062934258D1484A116A41F40041116283
:10A80000116A21F4004111625A6842F480525A6080
:10A810001A68520634D443491E68D1F8D442D1F89C
:10A82000E002D1E9B025B0F5005F42EA0502D1F8B7
:10A83000CC5242EA0502D1F8D05242EA0502D1F8E0
:10A84000D85242EA040242EA0502D1F8DC5242EA56
:10A850000502354D42EA000205EA060542EA050214
:10A860001A60D1F8C8225D6842EA14422F4C04EA0B
:10A87000050442EA04025A6002D1B1F8E4221A61E6
:10A88000DA6922F40062DA611A6842F040021A6062
:10A89000BDE8F087204A516A41F480515162516A03
:10A8A00021F480515162AFE7214A934213D11A4AF1
:10A8B000516A41F400515162516A21F400515162D0
:10A8C000A2E7154A116A41F480411162116A21F42C
:10A8D0008041116298E7174A934295D10E4A516A16
:10A8E00041F480115162516A21F4801151628BE769
:10A8F00009490B6923EA02020A612CE706494B6900
:10A9000023EA02024A6126E703490B6A23EA0202AC
:10A910000A6220E7B01801200038024000300140F0
:10A9200000380040000001204000FFFFFBF0FFFF67
:10A93000003401400050014008B100227EE470471D
:10A94000F8B5CB7813B900252846F8BD00F11007FB
:10A950000C460646897838460CF0D4FD054600289A
:10A96000F1D0E0780DF01CFBB06123780133DBB24D
:10A9700010B1C371222383710D21FFF7DDFFB06990
:10A98000FFF756FA0D4AD2F8D432632BFBD90C48A4
:10A990000CF0A4FD03463846B38239F03FF9034674
:10A9A00030B9E0781D460DF0FBFA0DF057FBCBE710
:10A9B000306986F8D83045F023FFC5E7B01801208C
:10A9C00040420F0070B50E4CD4F81C6F002E15DD00
:10A9D00004F58764002503E0B54204F120040DD09E
:10A9E000237F0135002BF7D0E06800220028F3D048
:10A9F000217D2034FFF722FCB542F1D1012070BD4A
:10AA0000C8010020AB4B2DE9F04F91B093F8CA8BF1
:10AA1000A94B0025A94F0093A94BA3F6B40ADFF870
:10AA2000B892DFF8B8B24E46B30AA3F58013522BA2
:10AA300055D8534493F8F4330D2B50D8B8F1010F87
:10AA4000FC5640F01E81012C3FD14FF000094946D1
:10AA500020460EF0C5F90EF04BFA90F800C0BCF19C
:10AA6000000F18BFBCF1540F14BF4FF0010C4FF092
:10AA7000000C40F0028109F104091FFA89F9B9F1CB
:10AA8000100FE4D1002D00F0BA808B4A00210DE0B8
:10AA9000534493F8F4330D2B0FD8FB56A3420FD039
:10AAA000013102F58672A94280F2A58090680368A0
:10AAB0009B0AA3F58013522BEAD90023A342EFD1BE
:10AAC00043799BF805009842EAD17D4B5B4513D052
:10AAD0005BF81C6FB30AA3F58013522BA9D9B8F108
:10AAE000010FF2D001230024B8F1020FADD1002BE9
:10AAF000ABD0734B5B45EBD1009B013503F58673FF
:10AB0000042D00938BD1DFF8D8814FF0000B08F5AE
:10AB10009E77A8F5876ADAF81C3F5B4568DDD8F8B0
:10AB20000C60002E64D098F81030B088D6F80090F1
:10AB3000DAF8045063490193B0FA80F34944002DD8
:10AB40000293C3F11F034FEA9121009340F3CD809C
:10AB5000594B002405E0013403F58673AC4200F044
:10AB6000C1801A688A42F6D14FF48673524A03FBB9
:10AB70000424009A0BF1010B019B5100C8F804203A
:10AB800088F810300323C8F80C6003FA01F5C8F800
:10AB90001840B371012386F807B01646A26C03FA79
:10ABA00001F12A43A264226D0A4322659AF800202B
:10ABB000002A6BD003FA06F11A46636D0B4389B283
:10ABC0006365C9F81800D4F8AC00FDF795FA204683
:10ABD00008F12008FDF764FA0123BBF1080F07F123
:10ABE000180708F8043C08F8033C07F8073C92D122
:10ABF00011B0BDE8F08FBCF1000F7FF466AF58468E
:10AC0000FDF712FA9BF80540C3B2022B00F24C8309
:10AC1000431C2D4A5BB203EB430398002B4B03F517
:10AC2000727104E0994200F03F8353F82C2FB24236
:10AC3000F8D11A79A242F5D11A58002AF2D09446D6
:10AC40000023234A51680133614513D0102B02F1D0
:10AC50002402F7D14FF0FF3303EBC3031D4A02EB8D
:10AC6000830393F89C30002B7FF42FAF009BC3F835
:10AC700008B041E7DBB2013BEEE7002D7FF405AF02
:10AC800023E7B4F1080318BF01232DE7029900045C
:10AC9000C1F12F05009903FA01F1AB40656D89B24E
:10ACA0002B436365C9F81800D4F8AC00FDF724FA0B
:10ACB0008DE700BFB0180120D00100202CB7050897
:10ACC000143F05080000FEBF000001406036050883
:10ACD000800001200000012000040140343E0508EE
:10ACE00000060020032C00F399824FF4867303FBC7
:10ACF00005A31869002800F0C18299600131CAB229
:10AD000083F811210492542283F810216B1C0268ED
:10AD1000CAF8043044790392FDF786F9A04B8646C1
:10AD200093F8E13B0593C3B2022B00F2BD8200F120
:10AD3000010C9C499C4800234FFA8CFC039A0CEBB5
:10AD40004C0C4FEA8C0C05E00133172B00F0AC8261
:10AD500051F82C0F9042F7D10879A042F4D151F864
:10AD60000C000028F0D02C210EEB4E0E002401FB2D
:10AD700003F303EB8E0E8B4B734419694FF4867308
:10AD800003FB05A3C3E90701884B9C46DCF80410CC
:10AD9000884217D001340CF1240C102CF6D1844BCE
:10ADA00093F87820002A00F06282824B824883491F
:10ADB000834AC3F84804C3F84014C3F8502411B0C0
:10ADC000BDE8F08F611C7A48C9B2013901EBC101BD
:10ADD00000EB810191F89C0006900028E5D10498D1
:10ADE0004FF08C0C81F89D004FF4867000FB05F449
:10ADF0002046542481F89C400446811071480394F5
:10AE0000544400FB01F1C4F800C101FB0CF001EB5C
:10AE10004101C4F80C9001EB011C6B4901EB4000AF
:10AE2000A1F54C7101EB8C01C4F8FC00C4F8B4101E
:10AE30003321C4F8B8106549039C0C195849D1F85E
:10AE40002C930599062900F00E8207296048614974
:10AE5000DFF888E10CBF84468C465F4908BF714625
:10AE600010460593039BB9FBF1F1B9FBFCFC4A1EAC
:10AE70004FF486790CF1FF3192B209FB05A9A9F8CC
:10AE8000BC1003F15801A9F87420504B226600222F
:10AE90001944A4F858206266E26544F019F8D9F81C
:10AEA000103018680493026842F0800202605A79F8
:10AEB000059B0C2A08D8DFE802F06B070707640738
:10AEC00007075C07070754004FF4867202FB05A2D0
:10AED00051694FF0600C02684FF000094FF0020E0C
:10AEE000CDF820C04FF4807C22F00102CDF82890EC
:10AEF000CDF838C04FF0010CCDF83490CDF824C017
:10AF00004FF00A0CCDF83C900593CDE90BCE0260D2
:10AF100008AA43F09BFE4FF48672049B02FB05A235
:10AF200019685269059B012A5AD0042A58D0102A60
:10AF300000F0A981402A53D0B2F5807F00F0A681AD
:10AF4000B2F5806F00F0A281B2F5805F00F0A481BD
:10AF5000B2F5803F4FF03C090CBF08224FF400626D
:10AF60003FE04FF486724FF4805102FB05A251611D
:10AF7000AFE74FF486724FF4807102FB05A2516176
:10AF8000A7E74FF48672102102FB05A25161A0E7EA
:10AF90004FF48672012102FB05A2516199E700BFBF
:10AFA000B018012060360508000001408000012033
:10AFB00000000120C01200207957010875570108D0
:10AFC000815701086B4CA407501A0020D0010020C3
:10AFD0001055220044950800D0DD060040771B0084
:10AFE000082201F1180050F809C042EA0C0240F8AA
:10AFF0000920049A1079002840F01C814FF48671D2
:10B00000002201FB05A1D1F810C0C869DCF800C01E
:10B01000DCF8001041F00101CCF800105968013251
:10B02000884200F00381102A03F12403F6D14FF087
:10B03000FF339F4A03EBC30302EB8303D3F8800083
:10B040009C4B98420CBF9520962041F05FF84FF43E
:10B05000867303FB05A31A6953790C2B00F2E38076
:10B06000954901EB4303B3F8D0C84FF486731068D9
:10B07000924903FB05A3A3F818C0002306E0904201
:10B0800000F008810133042B00F00B8151F83320CC
:10B09000002AF4D1DAF8202F0132CAF8202F0AEB67
:10B0A000C302DB00C2F8240F1944069823469022FD
:10B0B000B1F804E0DFF818924CEA0E0CA1F804C0D5
:10B0C0007F49FFF73FF84FF486734FF4403C40212F
:10B0D00003FB05A50023E869026842F01002026044
:10B0E000026842F014020260C4F8A830C4E91F33B9
:10B0F000C4E9283304232A6AC4F898C04FF4804C6A
:10B10000C4F89C304FF48063A167C4F88430C4F85D
:10B110009420D5F8B820C4F89020C2B220F0FF00E7
:10B12000103AA9FB0231EA68039B18320909226729
:10B130004FF48052C4F8882003F17002614B1A4426
:10B14000D5F8B430C4F88CC0636743F045FFE869B4
:10B15000039B4FF40031D0F800E04FF4006C03F192
:10B16000B802584BC4F820E0D0F814E01A44002389
:10B17000C4F824E0D0F804E0C4F828E0D0F808E0EF
:10B18000C4F82CE0D0F80CE0C4F8C830C4F830E0C3
:10B19000C4F8F030C4E93033C4E93A332B6A03937E
:10B1A0000423C4F8E4304FF48063C4F8CC30039B2C
:10B1B000C4E93731D5F80031C4F8D830C3B220F033
:10B1C000FF00103BA9FB0331EB68C4F8D0C010337B
:10B1D0000909C4F8B830D5F8FC3003934FF4804324
:10B1E000C4F8D430039BC4F8BC3043F0F5FEEB69DF
:10B1F000B0881A68D6F8009062635A69A2635A68E8
:10B20000E2639A682264DA6862641A6842F01002A3
:10B210001A601A6842F014021A60AAE403232A4A48
:10B2200082F8E03BC1E54FF0000C1EE7D3B2069375
:10B23000013BFEE6079305910CF0B2FE05998146AD
:10B24000079B58B105930221049BDA79FEF7F6FFBC
:10B25000049B5422A9F806201968059B4A6C42F405
:10B2600000424A64CAE6DFF86CC01849F8E5049960
:10B27000542283F8791083F8782096E50223124A45
:10B2800082F8E03B91E54FF40062AAE608224FF015
:10B290000409A6E6DB0007E74FF400624FF004095B
:10B2A0009FE600239B88FFDE00235B68FFDE00BF74
:10B2B000000001200060024060360508EC1000200C
:10B2C00045810008D0010020B0180120A0BB0D006E
:10B2D000ABAAAAAA882A1100F8B590F8B2311C09C5
:10B2E000013C052C0FD81B4E054603F00F0306EB5F
:10B2F0004402B2F8EC0840FA03F2D20703D595F8FD
:10B30000BD71012F01D00120F8BD07FA03F33444C9
:10B31000013B184046F00AFA94F8F82813180E4A30
:10B3200002EBC30152F833208B8810691840EBD030
:10B33000002395F8B3210846022185F8BD31FEF7B8
:10B340007DFFD5F820213846136843F008031360C9
:10B35000F8BD00BF60360508942401202DE9F04FA8
:10B3600000228DB02F2107460DF01AFED0B19B4E62
:10B3700005464379D0F80080A6F83C34FEF7ECFD92
:10B3800080B1446874B1DFF88CB2002259464B6832
:10B39000013224319C4210D0102AF8D1904B93F8FE
:10B3A00078201AB100200DB0BDE8F08F2F21104693
:10B3B00083F8792083F87810F5E7D2B2DFF820A27D
:10B3C000013A02EBC2020AEB820292F89C90B9F1B8
:10B3D000000FE7D12F218368C6F8FC83A2F89C10E8
:10B3E000D6F82C237F4901938A4280F0D8804946C1
:10B3F000120AC6F800147C490020A1FB02317B4BE5
:10B40000C6F80C040A09C6F804040909A3FB0232B1
:10B41000C6F808145208A6F8E62E5200A6F8E42E44
:10B4200096F8392402F0FF01002A00F0C4800222BD
:10B4300040466F4986F839243CF0EAFC0122384640
:10B4400086F839240CF0ACFDC6F8E80E28B12F219F
:10B45000C1804E21EA79FEF7F1FE664A0021019B88
:10B46000C6F8F81EC6F8F03EC6F8081FC6F8101F4A
:10B47000C6F8181FC6F81C1F106BC6F8EC4E40F437
:10B4800000101063106B00F4001003900398106B11
:10B4900040F480001063126B02F480020492049A5C
:10B4A0004022C6F8F42E4FF48062C6F8FC2E4FF40A
:10B4B0008052C6F8002F4FF48042C6F8042F4FF494
:10B4C0000032C6F80C2F0322C6F8142F96F83C243D
:10B4D0000C2A73D8484901EB4202B2F80079B84609
:10B4E000083746485946002206EB870CCCF8FC0387
:10B4F000A0F52F60C6F8240F486801322431844239
:10B5000062D0102AF8D14FF0FF3202EBC2020AEBF0
:10B51000820A3B4ADAF8800090420CBF95209620C0
:10B5200040F0F4FD0022DBF8041001320BF1240B93
:10B530008C4246D0102AF6D106EB87074846434690
:10B5400060223049FEF7FEFDD7F8FC033BF010FE09
:10B5500000287FF427AF60210A90AB79059159004C
:10B560000B90DB00069001F00201099003F0080344
:10B57000B6F83C242448CDE9071305A940F0EAF8C1
:10B5800000287FF40FAFAB79B6F83C149B071E4838
:10B590001DD53CF0C9FCB0FA80F0400903E71B4917
:10B5A0001B481144A0FB0131890D013989B2481CA7
:10B5B000B2FBF0F21CE786F8381438E788460F46ED
:10B5C0008EE75FFA82F9B7E7D2B2013A9DE73CF025
:10B5D000EFFBB0FA80F04009E5E600BFB0180120AB
:10B5E00000000120006CDC02598B4F01ABAAAAAA13
:10B5F000B01C012000380240603605089C2701205D
:10B60000006002403D900008AC1C012000366E0135
:10B61000819F5E1680000120014B53F82000704787
:10B6200050280040014B43F820107047502800403C
:10B630001D4B1E48196C1E4A41F0805130B41964EC
:10B6400082B0196CFF2401F08051019101990168C9
:10B6500041F480710160CA20196C41F48061196461
:10B66000196C01F4806100915321009D5462506275
:10B6700051625B6FDB000DD40E4B00210E4A43F884
:10B68000041B9342FBD10D4B0D4AC3F8502802B066
:10B6900030BC7047094A0A4BD2F850289A42EBD185
:10B6A00002B030BC704700BF00380240007000405C
:10B6B00000280040542800406C2800400020004032
:10B6C000316665422DE9F0470646086888B00C46A9
:10B6D0004FEA902CBDF84080ACF5801C9DF844905A
:10B6E000BCF1520F64D8374FBC449CF8F4530D2D75
:10B6F0005ED81946FDF7E0FC334A2368617902EB16
:10B70000851A94F806E0B9F1000F54D1F4469B0A6B
:10B71000A3F58013522B23D83B4493F8F4030D2850
:10B720001ED84FEA4C034FF480774FEACC0CCDF88B
:10B73000088003F0020302EB80100A4601A903937C
:10B740000CF008030493602301934FF40073CDE9D8
:10B750000673002305933FF0FDFF617994F806E03E
:10B760001EF0020F504629D03CF0DEFB174BA8011B
:10B77000022203EB8515D5F8401485F87D24144A80
:10B780008D682A40062A06D0B2F5803F03D00A68A9
:10B7900042F001020A600344012283F87D242168FB
:10B7A000637901F1340271600021D0183060D1500A
:10B7B00008B0BDE8F0878EF0010CA8E73CF0F8FA7D
:10B7C000D4E700BF60360508F01C0120B018012046
:10B7D00007000100F0B50446D0F89400434B83B055
:10B7E000A16804F1640204F118070E68C1B220F0E8
:10B7F000FF0001921039A3FB0131090943F036FC27
:10B80000616D0023019A012984F8583018D0042969
:10B8100016D0102955D0402912D0B1F5807F53D0D1
:10B82000B1F5806F50D0B1F5805F55D0B1F5803F54
:10B830004FF03C030CBF6FF0080C6FF4006C01E09C
:10B840006FF0080C06F118053046E95801EA0C01C2
:10B85000E950616D43F0FAF9636D012B16D0042BAA
:10B8600014D0102B0FD0402B10D0B3F5807F2FD0E9
:10B87000B3F5806F2CD0B3F5805F31D0B3F5803F46
:10B8800006F1540502D04FF4006100E008212B6856
:10B890003A46D4F894000B4340212B602162C1B298
:10B8A000124B20F0FF001039A3FB0131090943F0CE
:10B8B00093FBD4F89420136843F01003136003B093
:10B8C000F0BD6FF4006CBDE76FF0080C0423B9E71E
:10B8D00006F11C050821DAE76FF4006C0423B1E7D8
:10B8E00006F11C054FF40061D1E700BFABAAAAAA7C
:10B8F0002DE9F04FDFF85CB29BF800402DED028B94
:10B9000087B034B90124204607B0BDEC028BBDE8F6
:10B91000F08F8B4BDFF840A2D3F8D43208EE103A08
:10B920000CF0A0FD9AF8243C0390002B00F001815C
:10B930000BF234670BF634330BF63C4400263D46DD
:10B9400001930597DAF81C34039AD31A03D4EA6DED
:10B950009A4200F3D08006EB86030BEB431393F877
:10B960008C3603F0FF020292002B00F08D80D5F898
:10B970009410AB6873481A68CBB221F0FF01103BFA
:10B98000A0FB030370481B09C35C19444B68A989D9
:10B990001FFA83FCD368CCF1160C23EA0103BCF137
:10B9A000070FD36070D9DBF83C3B00220121013343
:10B9B00096468946CBF83C3BD5F89C301F4604930D
:10B9C00057F8048B40461CE0D7F80080BEF1140FF6
:10B9D000A8EB000340461CDC13F1080848BF03F144
:10B9E00017084FEA28130EEB281E03F1FF38013128
:10B9F00002FA03F3043709FA08F28C4542EA03021B
:10BA000007D38C45E0D8CEF1150338684FF0150EFA
:10BA1000EBE7BEF1150F65D14C49C2F38423C2F3A5
:10BA2000441001EB830301EB8000D3F81C39D0F8FC
:10BA30001C091B0243EA001302F01F00C2F3C432C8
:10BA400001EB800001EB8202D0F81C19D2F81C290E
:10BA50000B4343EA023383EA132282EA121202F012
:10BA60000F020F2A3ED1C3F30F134FF6FF7293421A
:10BA700038D0B3F5606F45D0019A9381029918EEE2
:10BA8000102A20460BF0D0FC019B284601365C347E
:10BA90001433A0350193FFF79DFE9AF8243CB3427E
:10BAA0003FF750AF0122059F8BF8382C0022CAF8CF
:10BAB0001C24002B3FF426AF03EB830307EB431357
:10BAC0003A7CA03757F84C0C12F0020F57F8982C1C
:10BAD00011680A6A14BF42EA80020243BB420A624A
:10BAE000EED10FE7DBF8383B0133CBF8383BCEB172
:10BAF00000230293C2E70024204607B0BDEC028B6E
:10BB0000BDE8F08F0E4991F8AC2302EB420201EB45
:10BB1000C202324492F859230D2AADD18023019AF2
:10BB20009377ABE704995822094847F057FB0296F0
:10BB3000A4E70122CAF81C348BF8382CE3E600BFD6
:10BB4000B0180120ABAAAAAA3CB7050860360508C0
:10BB5000A80D0020C8010020C0120020D0F820113C
:10BB6000242200232DE9F041C0F8942104460A68FC
:10BB7000806804F5907522F001020A600B604B604A
:10BB80008B6094F805C0C4F89C314FEA8C22C4F84D
:10BB9000943184F8903102F48052C4F89831C4F89A
:10BBA0003831C4F828214FEA0C32C4F8403102F48D
:10BBB0000052C4F834312379C4F82C214FEA0C2206
:10BBC000C4F8240113F0010002F48062C4F83021AB
:10BBD00002D00422C4F8342113F0020305D0D4F8B3
:10BBE000342142F00802C4F834211CF0010F0DD0BA
:10BBF00048B1D4F8442142F00202C4F844214FF481
:10BC00008032C4F84C21002B40F0FF80A84B03F198
:10BC1000200053F8042F944200F0BD809842F8D1E0
:10BC20001CF0080F40F0CD80D4F89431002B00F0C8
:10BC3000168124232846C4F894310B6823F00103AD
:10BC40000B603CF095F9012815D0D4F84431002B55
:10BC500040F01881D4F8203128465A6822F49042E6
:10BC60005A609A6822F02A029A601A6842F0010229
:10BC70001A6044F03BF92379DA0761D5D4F8FC2047
:10BC8000002A00F0D9800023D4F8041104F13C0606
:10BC9000E263A3644FF480623046E264C4E91013A7
:10BCA000C4E91433C4E91833C4E91A334FF48033B8
:10BCB000E3654FF48073A36544F092F930463BF09E
:10BCC00057FAD4F89881C4F88C61B8F1200F6567F1
:10BCD00031D1E368626999B26AB3B1FA81F77F0939
:10BCE00049B394F89001012825D030460126C4F8C4
:10BCF0009C710B4684F890612226A4F87811C4F850
:10BD000098616C4ED4F82011A6676B4E2431C4F8AC
:10BD10007421E667694EC4F88C70C4F888603BF003
:10BD2000C5FA002800F0B280102384F89071C4F89E
:10BD30009C31C4F89481E26B23795268C4F81421D1
:10BD40009B0777D5D4F80021002A69D00023D4F8C6
:10BD5000081104F19C06C4F89C20C4F8A8304022C5
:10BD6000C4F8B8303046C4E92C33C4E93033C4E9F0
:10BD700032334FF48033C4F8BC304FF48063C4E9ED
:10BD80002812C4F8AC3044F02BF930463BF0F0F9FF
:10BD9000002867D0FEE7002C3FF442AF94F8BC3196
:10BDA000002B3FF43DAFD4F844311CF0080F43F0B2
:10BDB0000803C4F844314FF40043C4F854313FF44D
:10BDC00033AFD4F89431002B55D024232846C4F83F
:10BDD00094310B6823F001030B603CF0C9F8012893
:10BDE0003FF449AFD4F84431002B47D1D4F8203187
:10BDF00028465A6822F490425A609A6822F0220239
:10BE00009A609A6842F008022EE7D4F8443143F071
:10BE10000103C4F844314FF40033C4F84831F5E667
:10BE2000D4F8A0311A6842F080021A601A6842F011
:10BE300040021A60BDE8F081D4F8A021116841F4F5
:10BE400080711160916841F001019160116841F0C9
:10BE500020011160116841F01001116070E784F851
:10BE60009031E6E6D4F89C30C4F88861C4F8D45028
:10BE70005860BDE8F08184F89031A6E728463CF090
:10BE800031FAB3E728463CF02DFAE3E6D4F8203146
:10BE900084F890011A6842F480721A609A6842F03D
:10BEA00001029A609A6842F040029A6043E700BF3C
:10BEB000E81E0020FD2904082D2A0408312A040860
:10BEC000F8B5EFF31185502383F31288D0F80031D1
:10BED0001B6813F0010303D0EDB285F31188F8BDA0
:10BEE000D0F894210446D0F898110A4302F02102B8
:10BEF000212AF1D0D0E90901884253D043D82269E0
:10BF00001846531A9BB2D4F894710022A062202FD5
:10BF100084F8A421E0D1A2695118DDD0B3FA83F6E8
:10BF20007609002BD8D094F89021012AD4D0012290
:10BF3000D4F88801A4F8723184F890212122C4F841
:10BF40009C61C4F86C11A4F87031C4F89421E8B174
:10BF5000DFF858C0D4F82021C0F83CC0DFF850C04A
:10BF600028320665C0F840C0DFF848C0C0F84CC0B1
:10BF70003BF09CF950B1102384F89061C4F89C31D7
:10BF8000C4F89471A8E7431A9BB2BCE7D4F82031F7
:10BF900000224021196284F890219A6842F08002C0
:10BFA0009A6099E7012384F8A43195E7D52904081C
:10BFB000F9290408312A040870B5D0F82041054653
:10BFC000E369990614D5606AEB6AC0B2002B74D09D
:10BFD000296B9847D5F82041236823F480732360A8
:10BFE000A36823F00103A360A36943F00803A361DE
:10BFF000E369DA0701D501232362E3699B0701D5D1
:10C0000002232362E3695E0701D504232362E36907
:10C01000180701D508232362E369590614D5402384
:10C02000236295F8BD61002E31D0D5F80031CBB137
:10C030002846FFF745FF95F8A4311BB195F8BD617F
:10C04000002E4BD0D5F82041D5F8003163B1E3691B
:10C05000DB0606D56B6B13B19847D5F8204110234A
:10C06000236270BDD5F82041E3691A06EFD5D5E902
:10C07000092393422DD0AA69D25C0133D2B2A262C5
:10C080002A69B3FBF2F102FB1133AB62DFE795F8EB
:10C09000B2010BF085FF236823F00803236001231E
:10C0A00085F8BD310028C0D032462021FEF7C6F801
:10C0B000D5F80031002BBBD1D4E7EB696A69D054C5
:10C0C000EB69EA680133B3FBF2F102FB1133EB6178
:10C0D00080E7236823F080032360B8E795F8B20176
:10C0E0000BF05EFFD5F820410122236823F00803FE
:10C0F000236085F8BD210028A6D032462021FEF716
:10C100009DF89FE72DE9F04FAF4C83B004EB80041E
:10C11000D4F82C4C002C6BD0D4F8AC511F46DFF86F
:10C12000C4B290466B680646A84AC4F8A0316B6B4F
:10C13000DFF8B49263612B6BA160A3616B8FE36046
:10C140002B8FC4F8A82123610BF69C1323602A7857
:10C1500009EB420393F94C0F53000193C3B2012B37
:10C1600040F28680D4F8003183B1994900209C4682
:10C170004B68013024319C4500F0F6801028F7D13F
:10C18000944B93F87810002900F05381D4F8FC0008
:10C19000002840F0C2806B68C4F8203195F8280070
:10C1A000002840F0D28094F8B2010BF0F9FE022191
:10C1B0003A07034694F8B09184F8BD111CD558B3E2
:10C1C00017F0510F4FF00B0206F1010614BF0A21C0
:10C1D0001A2117F0410FC671827114BF402320232A
:10C1E00094F8B3211943FEF729F8D4F8FC3043B38F
:10C1F000204603B0BDE8F08F18F0020F0CD058B104
:10C200000B223B06827106F10102C27100F1188116
:10C2100094F8B321FEF712F848460BF0C1FE00284F
:10C22000E3D018F0010FE0D00C2201360221C671D4
:10C23000827194F8B121FEF701F8D4F8FC30002B9C
:10C24000D6D195F82C1095F92A0089093FF062FEA5
:10C2500095F92A3095F82A20002BC9DB02F01F023D
:10C2600001215B095C4801FA02F240F82320BFE794
:10C2700008234FF00C0A0BF5A86C1AFB003A0023B8
:10C28000E64619460131172962D01EF81C3F042BDF
:10C29000F8D19EF801309342F4D15EF80A30002BB9
:10C2A000F0D08E460199C4F800318944CEEBCE011E
:10C2B00099F94DEF890000EB4009BEF1FF3F01EB1A
:10C2C00089015944D1F84C15C4F808113FF44DAF19
:10C2D0000021013117293FF447AF1CF81CEFBEF1D4
:10C2E000050FF6D19CF801E09645F2D15CF80AE022
:10C2F000BEF1000FEDD0C1EBC101C4F8FCE000EBD2
:10C300004000890001EB80008344DBF84C15C4F841
:10C310000411002B7FF429AF70462D4A0023516889
:10C3200001332432814261D0102BF8D1294B93F88C
:10C330007820002A7FF42FAF2A78013283F8792001
:10C340000C2283F878206B6826E73FF0DFFE2AE7AF
:10C35000019B9944D4F8003199F94D1F0131B7D1AF
:10C36000002B7FF402AF11E75FFA80F9194B01321D
:10C3700009F1FF31D2B201EBC10103EB810393F864
:10C380009C1000297FF402AF83F89D201348D3F856
:10C39000802082420CBF952096200B2283F89C209F
:10C3A0003FF0B4FE2346484695F82B200C49FDF794
:10C3B000C9FE6B68D4F8FC002833C4F81831002893
:10C3C0003FF4E9AEA9E700BFC0120020D9B20008CF
:10C3D000800001200000012000E100E00060024038
:10C3E000B190000860360508B0180120DBB2184A89
:10C3F000013B03EBC30302EB83032A7893F89C1001
:10C400000132D2B200297FF4C6AED3F8800083F89F
:10C410009D20104A90420CBF952096200C2283F854
:10C420009C203FF073FE6B6803F12402C4F81C21CA
:10C43000B2E6013283F879200B2283F87820A5E652
:10C440000123204684F8BD31FEF746FFE4E600BF35
:10C450000000012000600240BFF34F8F0549064BEA
:10C46000CA6802F4E0621343CB60BFF34F8F00BF92
:10C47000FDE700BF00ED00E00400FA0530B583B031
:10C48000FFF7D6F80320FFF7C7F801284BD0324C4E
:10C490000025324A0523C4F89850C4F89C50C4F8CB
:10C4A000A020C4F89430BFF34F8FBFF36F8F4FF6C7
:10C4B000FF01E2682A4B0A4013432A4AE360536FA4
:10C4C0003BF0DCF9284B2949A3FB0023D4F8FC20DE
:10C4D0009B0C42F08072C4F8FC20C1F8B433D1F850
:10C4E0002C332349234AA1FB031323499B09C2F898
:10C4F000B01F5560013B1168B3F1807F41F001012D
:10C50000116008D24FF0E022F0215361072384F834
:10C510002310956113614FF0E022136943F0040387
:10C52000136103B030BD02210320FFF77BF80D4BF0
:10C5300012485A6C124942F480425A645B6C03F40C
:10C5400080430193019A02680B68026083F30888B4
:10C550004B689847FEE700BF00ED00E01B000006B7
:10C560000005FA050038024083DE1B43B0180120A5
:10C57000D34D6210001000E055CEACC5003801402C
:10C580000000F01F800AA0F5801052281CD80F4B25
:10C59000184490F8F4330D2B16D8013910B40C4C14
:10C5A00004EB831CD4F82C438BB2DCF840040CF26F
:10C5B0004441CCF84C34B4FBF2F2013A5DF8044B40
:10C5C000CCF844243BF024BC704700BF603605081B
:10C5D000B018012070B504460068830AA3F58013E3
:10C5E000522B05D82E4E334493F8F4530D2D00D919
:10C5F00070BDFCF761FD2B4BA801022203EB8515F2
:10C60000D5F8401485F87D24274A8D682A40062AEB
:10C6100006D0B2F5803F03D00A6842F001020A60FA
:10C62000034401202168214A83F87D040023204827
:10C6300001E050F8332091420AD001330E2BF8D19B
:10C64000012100203FF066FC1A4B01221A6070BDE8
:10C6500006EBC303012193F9D14993F8D169204630
:10C660003FF058FC002CC3DB06F01F0301216409D6
:10C67000104D01FA03F31B2E45F8243008D02E2E5E
:10C68000B6D12C203FF046FC4FF480536B6070BD58
:10C6900019203FF03FFC4FF000732B6070BD00BFCE
:10C6A00060360508B01801200700010000000140B5
:10C6B0002C40050800E100E003689B0AA3F5801305
:10C6C000522B56D870B53B4C234493F8F4C3BCF1BD
:10C6D0000D0F4DD84079850800294ED00CEB8C0306
:10C6E0004FF0020E840834480CEB43030EFA04F4B6
:10C6F0002B4400EB8C15D5F8405400EB830EEE680C
:10C70000CEF804103443CEF81420EC604FEA8C14B9
:10C71000EFF3118E502383F312882C2303FB0CF3C9
:10C72000C258C11832B3131D4A622C22234D02FB9A
:10C730000CF215441432024452F8041B19B119606A
:10C7400052F8043C04339542F6D100225FFA8EFE83
:10C750001A608EF311882C2303FB0C0C2044DCF8A8
:10C760002430D0F8402403B3D36843F00103D360EE
:10C7700070BD704724330344D7E70CEB8C030E489D
:10C780002C460CEB43032B4400EB8C15D5F840648E
:10C790000225A540F46824EA0504F46000EB830454
:10C7A000616062614FEA8C14B2E7D36823F0010341
:10C7B000D36070BD60360508B0180120D418012080
:10C7C00003689B0AA3F58013522B00D97047144AC3
:10C7D000134493F8F4330D2BF8D810B4114C79B9F5
:10C7E0004179022204EB83105DF8044B21FA02F335
:10C7F000D0F840149A40CB6823EA0203CB6070471C
:10C800004179022204EB83105DF8044B21FA02F314
:10C81000D0F8401402FA03F3CA681343CB607047A0
:10C8200060360508B018012003689B0AA3F5801341
:10C83000522B10D8084A134493F8F4230D2A0AD82F
:10C84000407902230549D84001EB82128340D2F897
:10C850004024DB431361704760360508B01801209F
:10C8600001490248FCF786BBB018012000000140D6
:10C8700010B5064C06482146FCF77CFB04F5C67152
:10C880000448BDE81040FCF775BB00BFB01801209C
:10C89000000001400044014002494FF08040FCF795
:10C8A00069BB00BFDC18012001490248FCF762BBEC
:10C8B000081901200004004001490248FCF75ABB56
:10C8C000341901200008004001490248FCF752BB1E
:10C8D00060190120000C00402DE9F843194E35691C
:10C8E000F3681D4010D04FF00047DFF85C80B5FAC8
:10C8F00085F227FA02F31F2A6FEA030305EA03050C
:10C90000336103D0002DF2D1BDE8F883D8F80431AB
:10C91000A3B103F1FF3900231FFA89F9C8F80431E4
:10C92000D8F80041002CEDD02368204649469847AE
:10C930006468002CF8D1002DD9D1E5E7F16A1FFA1F
:10C9400081F9EDE700100040B018012001490248CC
:10C95000FCF710BBE41901200004014010B5064C9F
:10C96000064804F59A71FCF705FB04F504710448C8
:10C97000BDE81040FCF7FEBAB018012000040140E9
:10C98000001C004001490248FCF7F4BA101A0120CB
:10C990000040014001490248FCF7ECBA681A012046
:10C9A0000048014001490248FCF7E4BA941A01200A
:10C9B000001800402DE9F0414FF425728EB000219F
:10C9C000664846F07FFC664B664E4FF080415A6CDD
:10C9D00006F68805374642F00102DFF89081A6F19D
:10C9E0008C045A645A6C02F001020092009A1A6C8C
:10C9F00042F001021A641A6C02F001020192019ADB
:10CA00001A6C42F002021A641A6C02F002020292DC
:10CA1000029A1A6C42F004021A641A6C02F00402C0
:10CA20000392039A1A6C42F008021A641A6C02F01C
:10CA300008020492049A1A6C42F010021A641A6CEA
:10CA400002F010020592059A1A6C42F020021A6454
:10CA50001A6C02F020020692069A5A6C42F0020208
:10CA60005A645A6C02F002020792079A5A6C42F416
:10CA700080325A645A6C02F480320892089A5A6CD6
:10CA800042F400325A645A6C02F400320992099A54
:10CA90005A6C42F480225A645A6C02F480220A9240
:10CAA0000A9A1A6C42F040021A641A6C02F04002B0
:10CAB0000B920B9A1A6C42F080021A641A6C02F004
:10CAC00080020C920C9A1A6C42F480721A641B6CED
:10CAD00003F480730D930D9B4246002301E054F84C
:10CAE000332091420BD001330E2BF8D11C3700209C
:10CAF0003FF00CFBAF420CD057F81C1CECE71A4A75
:10CB00001C3702EBC30393F8D0093FF0FFFAAF42A2
:10CB1000F2D14FF08041154F154C3A46002301E009
:10CB200054F8332091420BD001330E2BF8D11C3630
:10CB300000203FF0EBFAAE420CD056F81C1CECE79C
:10CB4000094A1C3602EBC30393F8D0093FF0DEFA22
:10CB5000AE42F2D10EB0BDE8F08100BFB0180120A6
:10CB600000380240B8400508603605080000014062
:10CB70002C400508800AA0F5801052280ED8084BDA
:10CB8000184490F8F4230D2A08D8064B03EB8213BF
:10CB9000D3F84024136843F001031360704700BFCB
:10CBA00060360508B018012038B5264C94F8643F6B
:10CBB000012B12D1042894BF002301236BB904EB8D
:10CBC00040000D4694F87C1FC4F8903FB4F87E2FC7
:10CBD000B0F8863FB4F8820F01B138BD07EE902A55
:10CBE000D4F8742F9FED180AB8EEE77ADFED177AC4
:10CBF00027EE277A07EE902A6422F8EE676A02FB96
:10CC000003F307EE903A02FB003366EE806AB8EE5B
:10CC1000E76A07EE903AF8EEE77A27EE067A87EEB3
:10CC2000270A20EE260A45F061FDD4F86C2FB4F8EF
:10CC3000803F1060D4F8D41219442944C4F8941FDA
:10CC400038BD00BFB0180120CA269B3E0AD7233C3E
:10CC5000F0B5A24CA5B0E368022B00F03A82A048E0
:10CC6000A04AA149121A46F0B9FAA048A04AA1491F
:10CC7000121A46F0B3FAA368012B00F2C28003EB4C
:10CC800043039D4A9D4D02EB430032F81320418837
:10CC90008388C5E9BA21C5F8F032994C994E9A4B70
:10CCA000B2FBF1F2994901FB02F20021C6F82C23F4
:10CCB000D4F8882042F47002C4F888201A6842F040
:10CCC00001021A609960924A1868024091481A60FD
:10CCD000C0F30807904A5A601A6822F480221A604A
:10CCE000D96007B1FEE78D49A0604FF6FF000A68E2
:10CCF0008B4B42F400720A60E26802401343E36027
:10CD00003FF000FDBFF34F8FBFF36F8FC4F8507239
:10CD1000BFF34F8FBFF36F8F636943F400336361D9
:10CD2000BFF34F8FBFF36F8FC4F88470BFF34F8F83
:10CD3000D4F8803043F6E07CC3F3C90EC3F34E331E
:10CD4000580100EA0C01734641EA8372013B5F1C03
:10CD5000C4F86022F8D1203810F1200FF1D1BFF3D0
:10CD60004F8F636943F480336361BFF34F8FBFF329
:10CD70006F8F6A49644B0A6842F480720A60196CCA
:10CD8000684A41F080511964196C01F08051029198
:10CD90000299116841F4404111601268D5F8E80227
:10CDA00002F44042D5F8EC42D5F8F0120192019A13
:10CDB0009A6802F00C02042A00F08D809A6802F052
:10CDC0000C02082A00F083804F4A136843F4803332
:10CDD0001360D6F8907904E0D6F89039DB1B642B09
:10CDE00074D813689B03F7D5474A936803F00C0384
:10CDF000082B6BD0136823F080731360D6F89079FA
:10CE000008E03E4DD5E9BA2147E7D6F89039DB1B5B
:10CE1000022B5BD813689B01F7D40B06640843EA26
:10CE20008013611E43EA01433F491943364B516069
:10CE3000116841F080711160D6F8901904E0D6F8BD
:10CE40009029521A022A41D81A689201F7D5196C12
:10CE5000344A41F0805119641B6C03F080530393F2
:10CE6000039B136843F480331360D6F8901906E0EF
:10CE7000D6F890395B1AB3F57A7F00F2CB8053680D
:10CE8000DF03F5D51368274943F400331360D6F860
:10CE9000902906E0D6F890399B1AB3F57A7F00F214
:10CEA000B9804B689C03F5D54FF400124FF0006336
:10CEB00004A804924FF4C07221930723CDE90823FC
:10CEC00003230A933AF00EFD80B3FEE7FEE75B68AA
:10CED0005A027FF579AF0C4B1B6885E7502800405C
:10CEE00000000000E83D0000C044060800000020EB
:10CEF000C801002049A606082449050800000120B1
:10CF000000ED00E0B01801200038024040420F0060
:10CF1000FFFFF6FE0000000810300024003C024035
:10CF20000003FA0500700040080040206C4A1368B6
:10CF300003F00F03062B0AD8136823F00F0343F006
:10CF400007031360136803F00F03072B63D1654BCE
:10CF50009A6842F4E0529A609A6842F460429A6099
:10CF60009A6822F0F0029A601A68900153D59A6884
:10CF700041F2883122F0030242F002029A60D6F8B0
:10CF8000900904E0D6F89029121A8A4243D89A6888
:10CF900002F00C02082AF5D1514A136819070AD584
:10CFA000136823F00F0343F007031360136803F0C3
:10CFB0000F03072B2FD14B4C4B4FA36823F4E053A7
:10CFC00043F4A053A360A36823F4604343F40043F5
:10CFD000A3603AF053FCA368C3F303133B4493F8F4
:10CFE000D831D840C6F82C033FF08CFB002304A8AE
:10CFF000CDE91333CDE91533CDE91733CDE9193335
:10D00000CDE91B33CDE91D33384B04933AF06AFC6C
:10D0100010B1FEE7FEE7FEE702234FF0007204A81E
:10D02000CDE90633D823CDE9042301230B933AF04D
:10D0300059FC00B1FEE7D4F88C3023F08073C4F8BB
:10D040008C30D4F88C3043F08073C4F88C30A368F3
:10D0500003F00C03042B36D0082B18D0244BC6F851
:10D060002C33204AD5E9BA31B3FBF1F39168D6F8F5
:10D070002C23C1F303110F4497F8D811CA401D495E
:10D0800001FB03F3C6F82C23934220D0FEE763682C
:10D09000626813F4800F636802F03F0218BF1649FC
:10D0A000C3F3881308BF1249B1FBF2F202FB03F38A
:10D0B0000C4A5268C2F3014201325200B3FBF2F350
:10D0C000C6F82C33CDE70C4BC6F82C33C9E725B096
:10D0D000F0BD00210320FEF7A5FAFFF7BDF900BF60
:10D0E000003C02400038024058470508C0FF0300DA
:10D0F0000024F40040420F0000127A000548D0F8E6
:10D10000A03223B1DB6A13B100F52870184702483A
:10D11000704700BFB01801204049050810B5174CF2
:10D12000D4F8983F1B883BB9002384F8A43F84F8C7
:10D130009832C4F8943210BDD4F89C2F002AF3DD45
:10D14000012A08D0D4F8A03F59880123A4F8A61FCB
:10D1500084F8A83FE8E7D4F8A01F8A8849880132FC
:10D16000521A9A42F1D10022D4F8A03204F5287064
:10D170001B69C4F8CC229847D6E700BFB01801203D
:10D180000748D0F89C3213B190F8A83F0BB10020AB
:10D190007047D0F8A03200F528705B68184700BFD0
:10D1A000B0180120174B10B4174C93F89822224462
:10D1B000C0E9002493F8980293F8A42F824217D86C
:10D1C00093F89802824206D300235DF8044B184678
:10D1D000C1E90033704793F89832002A5DF8044B98
:10D1E000C3F180030CBF012002204A600B6070472E
:10D1F00093F8984200230120121B5DF8044BC1E90B
:10D2000000237047B01801200C1F00200F4B93F82B
:10D21000982293F8A40F93F89822904293F89822BA
:10D220000FD8904204D3D3F89432002018447047AA
:10D2300093F89822D3F89432C2F180021044184433
:10D240007047801AD3F8943218447047B018012000
:10D2500010B51B4C84B01B4B94F8982203931344D5
:10D2600094F8A41F029394F89832994294F8983253
:10D2700014D899420AD294F898320191C3F18003EC
:10D280000093C9B901223F2B0ED868B994F89802CF
:10D29000401AB0FA80F0400904B010BD0022CB1A49
:10D2A000019201220093EEE76946002302A843F0B1
:10D2B00031FC94F8A41FE9E70B440222E3E700BF26
:10D2C000B01801200C1F00202DE9F043164685B050
:10D2D00000293CD0451E284CDFF8A4804FF00009FF
:10D2E0006F180DE094F8983208468B4294F8983203
:10D2F0001DD9C3F1800318443F281BD8AF4226D064
:10D3000094F8A40F15F8013F411C4044C9B280F8BD
:10D310004C3C0B0684F8A41FE4D5002094F8983206
:10D3200084F8A49F01468B4294F89832E1D8C01A41
:10D330003F28E3D994F898328B42DFD00F4B1B780B
:10D34000002BDBD00020FFF783FFAF42D8D1694626
:10D3500002A8FFF727FFDDE9003213443F2B00D975
:10D3600010B905B0BDE8F0830246334602A843F089
:10D37000D1FB05B0BDE8F083B0180120000001200A
:10D38000C012002030B585B0694602A8FFF70AFF39
:10D3900058B9094C04F52875D4F8A03228465B68C2
:10D3A00098470028F8D005B030BD0246012302A8F6
:10D3B00043F0B0FBEDE700BFB018012070B5114C91
:10D3C00016460A4682B0D4F89C3281190546994225
:10D3D00094F8A41F88BF1E1A94F89832994203D07B
:10D3E0000192FFF7CFFF019A002033462946C4F887
:10D3F000CC02D4F8A002846A0348A44602B0BDE877
:10D4000070406047B0180120501B01208C46134625
:10D41000014662461846D1E738B5244C002204F68E
:10D42000AC701346C4F89C220246117806320229D9
:10D430002BD00133062BF8D10022D4F8A032C4F847
:10D44000A02FF3B1DA6AE2B119489047D4F8A03FAF
:10D45000C4F8980FA3B159889A884368521A02FBFE
:10D460000333C4F89C32FAF7F7FF94F89832054674
:10D4700094F8A42F9A4201D0FFF784FFC4F8945285
:10D4800038BD0C4BC4F8983F38BD03EB4303D4F8C8
:10D49000A02200EB4303C4F8A03F12B1D26A002AD5
:10D4A000D2D1044A1046C4F8982FD4E7B01801200E
:10D4B000501B01204049050810B50A4CD4F8A03291
:10D4C0005B6A13B104F528709847D4F89432D4F805
:10D4D000982F013B5288134452421340C4F89432AF
:10D4E00010BD00BFB01801202DE9F043384E93B0B5
:10D4F000FFF714FEFFF790FF96F8983296F8A42FE6
:10D500009A4201D0FFF73EFF0025D6F89C72C6F87C
:10D51000945297B16C46DFF8BC802A4641462046BB
:10D52000203501F07BFD204643F0D4FB012201466B
:10D530002046FFF7C9FEAF42EFD896F8983296F82A
:10D54000A42F9A4201D0FFF71DFFD6F8983F9B7B8E
:10D55000012B36D096F8983296F8A42F9A4201D033
:10D56000FFF710FF0020C6F894026FB380466C46A8
:10D57000DFF86090054601E0AF421CD92A464946D3
:10D5800009A801F04BFD21220021204645F09AFE1A
:10D59000202221462846FFF711FF2022064609A92E
:10D5A0002046203545F0BBFF08B9202EE4D0AF421D
:10D5B00008F10108E2D8B8FA88F0400913B0BDE8D4
:10D5C000F083FFF779FFC5E7012013B0BDE8F083D2
:10D5D000B0180120ACB605080A4B93F8F40218B94C
:10D5E000094B93F8D00F7047084AD1680329F7D147
:10D5F00005494FF0010C81F8D0CF0021D16083F8AC
:10D60000F412704700000120B0180120502800409B
:10D610000321044608B50846FEF704F872B610491F
:10D62000D1F8D80FD1F8DC3F50EA03020AD100222A
:10D6300011460420FDF7F6FF11460520FDF7F2FF25
:10D64000FEF70AFFD1F8D42221B24EF66024121858
:10D6500004FB01F143F100038A1843EBE171E8E7B1
:10D66000B01801200021032008B5FDF7DBFF72B6DA
:10D67000FEF7F2FE184CD4F8E02F94F8E60F08B548
:10D680004AB11168938809690B40F8B9003B18BF8B
:10D690000123002BF4D114200BF03AFA00BFD4F888
:10D6A000E03F63B1196894F8E62F9B8809690B4045
:10D6B00042B9003B18BF01230BB1FFF7D3FFFAF7C4
:10D6C000FDFEEBE7B3FA83F35B09F5E7B3FA83F307
:10D6D0005B09002BD4D1DEE7B0180120F8B51C207F
:10D6E0000AF05EFC04461121FDF726F97CB3A388FD
:10D6F000C82022681B0493610BF00AFA2368A288F1
:10D700001B209A610AF04CFC08B12923C38029230D
:10D71000E380264CD4F8743213B10023C4F8743279
:10D720000023234E0125234FC4F8706287F8E83F99
:10D7300084F85C523FF002F906F11C03C4F874321D
:10D740001D4B93F8A131AB420CD02846F8BDC82040
:10D750000BF0DEF91B200AF023FC0028D9D0292386
:10D76000C380D6E7D4F89002543690F8BC33C4F89E
:10D770008C62AB4214D00168D1F8043823F0020364
:10D78000C1F80438D7F89029D7F890399B1A032BA1
:10D79000FAD98B68002243F001038B6080F8BC2328
:10D7A0000023064A184682F82330F8BDB02801202D
:10D7B000F8020120B0180120A829012000ED00E0A6
:10D7C0002DE9F04F00218BB041F69462BD4845F041
:10D7D00079FD0420FDF720FF01460520FDF71CFF21
:10D7E00051EA000340F05E81B74B03934C220021C5
:10D7F000B448012445F066FD00214C22B14845F0B3
:10D8000061FD039BAF4AD3F89C33B04D1471156092
:10D810005362C2E907333EF097FFFFF7FDFD002199
:10D8200008460AF049FCFAF717FEB0F1000B40F386
:10D830000981A44B0024A64D03F14C0AA54B2746B1
:10D84000A04605F5D279A44ECDE9013404E008F5EF
:10D850000068C34540F3AC80019AD2F8D432C2F8D4
:10D86000D832FAF72BFE202249464046FFF7A6FDA4
:10D8700012229A49484645F052FE0028E7D1474512
:10D8800021D0029B5A1C03EB4301954B029203EB00
:10D89000810394491846049301F0C0FB5246049B4F
:10D8A00042F84C3BDAF81C30CAF80C70A8EB0707BA
:10D8B000CAE908330123CAF808308B4BCAE9047758
:10D8C000CAF828309246039B47461222D3F89C336D
:10D8D000CAF81C30A918335D013291F8A41199429D
:10D8E0000BD00024202AF5D120374946BB453846C5
:10D8F00054DBFFF763FD0022ECE70134152CF1D176
:10D90000D0197A492022FFF759FD00230A2209A9DC
:10D910007648CDF8249001F00BFD074609980023C6
:10D920000A22013009A9099001F002FD07900023A5
:10D9300009980A2209A90130099001F0F9FC069022
:10D94000002309980A2209A90130099001F0F0FC8E
:10D95000059009A9099800230A220130099001F0D5
:10D96000E7FC0490002309980A2219460130099027
:10D9700001F0DEFC97B1DDE9063243EA4211049B77
:10D980005A01059B42EAC32242EA6003A7F2BC7235
:10D9900041EA422243EA0243CAF81C30029B642B4C
:10D9A00000F0F380474608F50068C3453FF754AFE1
:10D9B000029A642A00F0E280B84500F0DF800C2370
:10D9C000474DA8EB070602F1010803FB0255454944
:10D9D0004246454C284601F021FB029ADAF81C30F9
:10D9E000CAF80050951CCAF80C70CDF80880CAF827
:10D9F0002840CAE908330123CAE90466CAF8083096
:10DA00004C22304B00213A4F02FB05F501262B44F6
:10DA1000184645F057FC4C22002145F053FC294A9A
:10DA20005751039A8462029CD2F89C230234866088
:10DA30004262C0E904BBC0E907224FEA4B03B3F1DD
:10DA4000805F1EDA4C221F4B00212A4F02FB04F498
:10DA5000012502262344184645F034FC4C220021BF
:10DA600045F030FC174A03991751CBF10062D1F809
:10DA70009C13AA40467185604162C0E90711C0E964
:10DA80000422104B9D6835B91A461B791BB11368E7
:10DA9000002B40F08380002108460BB0BDE8F04F1A
:10DAA0000AF00ABB4FF47A72002343F0D7FD124B01
:10DAB00040F26D11022440F2B2720D46B0FBF3F356
:10DAC00024E000BFE030012000000120D44306081C
:10DAD000A8290120B0180120F0B60508CCB6050829
:10DAE0006C2B0120E0B605080DD400084C2B01205A
:10DAF00008B7050818B705088051010001325B1A04
:10DB000012F003040CBF4FF4B77129469942F5DDBA
:10DB10007449002C3CD003910399D1F86C139942BD
:10DB20006FDC714D01245B1A55F8041F01349942D2
:10DB3000F9DD0133A2F2BC72039D43EA44133C2495
:10DB400043EA4223694AB0FBF2F102FB11024FF4AF
:10DB50006160B2FBF0F100FB11221C20C5F87003DC
:10DB6000B2FBF4F004FB1022521042EA401242EAE7
:10DB7000C12242EA0343C5F89C3337E6029B0124E5
:10DB80005D1C002B3FF459AF00E06525584C37E78A
:10DB90000C4603911D21C4F87013BDE729462E469B
:10DBA0001564D563C2E91155D46C02F14C0354B32A
:10DBB0009C68481E1E648442DE63C3E9116612D06D
:10DBC000481C844216D08C427FF465AF084600287A
:10DBD0003FF461AF116CCC6B0134CC631964936476
:10DBE00001461A46E0E700293FF455AF884253F852
:10DBF0000C2CECD1117900293FF44DAF53641A6419
:10DC0000EEE7012495E73B490222264611E0CB6B63
:10DC10000A635B01C1E9046657D003F6FF77531E20
:10DC200003EB17335A1C0135C1E90D3351F84C0F82
:10DC3000C8B10B79002BEAD108690A63002848D1E2
:10DC4000531E10464F694863002F40D007F6FF77F8
:10DC500003EB1733201A8B635A1C0135C41851F893
:10DC60004C0F0028E5D124483E22013BC0F8184360
:10DC70003F24C0F800234022990F0190C0F824539C
:10DC8000C0F81433C0E9C1421C4AC0F8FC229A0013
:10DC90002BB340F2FF10121841F10001520A42EA80
:10DCA000C15202F140010198124C0A44C0F80C1311
:10DCB00002EBC303C0F810235902C0F8F832DA0DA2
:10DCC000C0E9C744C0E9BC12E5E61346AAE713461B
:10DCD000C0E700F6FF70531E03EB1030B2E70122DD
:10DCE000DFE700BF000001206C030120805101002C
:10DCF0000DD40008E0300120B018012024B7050839
:10DD0000032143F20122002343F2013C017243F25A
:10DD1000011102804FF6FF72A0F802C0438181809A
:10DD20008381C38102828374704700BFFF22174B37
:10DD30004FF0FF3CC27002710272427242738273F2
:10DD40008274C2740022F0B503F10C0766461725F1
:10DD500016244FF0150E02EB8202BB4200EB0201CB
:10DD600000F802E04C708D70CE7081F804C00BD0CA
:10DD700093F90620063393F801E09C78DD7893F957
:10DD8000046093F905C0E6E7F0BD00BFC44905088B
:10DD90004FF0000C01210222032380F805C081719D
:10DDA000C2710372704700BF0023022203704370E8
:10DDB0008370C37002717047302203230270437076
:10DDC000704700BF4FF4007141F2014200234FF44D
:10DDD0004D7C01804FF4E16142800122A0F806C031
:10DDE000038143818181C281704700BF4FF0010CE4
:10DDF0002C210222002380F800C041708270C37081
:10DE0000704700BF4FF4F07140F22E4C0023072200
:10DE100001804FF47A71A0F81EC04FF4FA6C41846F
:10DE20004FF4F5614371A0F820C040F2012C8371DA
:10DE3000438243F63813818443F23671A0F814C04C
:10DE400040F2034C018142F22011438142F22673D9
:10DE5000A0F816C040F2056C81810E21C381012318
:10DE60008270A0F818C080F826108276437400B53E
:10DE700040F2262EA0F81CE05DF804FB8388C3F373
:10DE80000B039342A8BF134670B51D460C461A46B5
:10DE90000646806845F0A2F96219084B9442B569BC
:10DEA00008D0074814F8011B00FB03F3A24283EAE1
:10DEB0000103F7D101202B6070BD00BFC59D1C81FF
:10DEC00093010001FF23037043708370C370704798
:10DED0001F2201234FF01E0C1D214270002280F8EA
:10DEE00000C0817003714371C2708371C371704748
:10DEF0000023037043708370C37070470023037066
:10DF000043708370C3707047002306214FF47A7208
:10DF100001700373C0E90123704700BF0023FF2293
:10DF2000411C10B500F8132001F8132001330B2B0E
:10DF3000F8D10B4B4FF0FF31002203F10F048C4658
:10DF400005E093F904C093F9051013F8032F00EBD3
:10DF5000420E9C4200F812C08EF80110F1D110BDA3
:10DF6000D84905084FF01A0C02210123002280F83D
:10DF700000C04FF0360C017180F803C04FF0370C31
:10DF8000C17180F806C04FF0380C817280F809C06A
:10DF90004FF0390C417380F80CC04FF0200C017425
:10DFA000262180F80FC04FF0270C81741021437098
:10DFB000827043710372C372827342740275C374B8
:10DFC000837580F815C0C2750176437682767047F6
:10DFD00000230370704700BF0A4491421AD001F138
:10DFE000FF3C41F2210100B502F1FF3E1CF8012F78
:10DFF000082380EA022010F4004F4FEA400281EA31
:10E0000040000CBF90B280B2013BF4D1E645EDD1A7
:10E010005DF804FB704700BF704700BF2DE9F04773
:10E02000089F002B0E4605463C4614BF4FF03009B2
:10E030004FF0200914F8011B41B3002A2CDD2346C0
:10E0400000E0B2B113F8010B9046013A0028F8D174
:10E05000A8F102086AB1C24649462846B04753466D
:10E060000AF1FF3A002BF7DC28EAE872397801322E
:10E0700049B1D71B2846B047E01914F8011B002905
:10E08000F8D1BDE8F0871046BDE8F087002A02F11C
:10E09000FF38E0DC0846F4E70022EAE703685A1C90
:10E0A00002601970704700BF024B186803681B6854
:10E0B000184700BF744F01200378092B01D0202B93
:10E0C00005D110F8013F202BFBD0092BF9D02D2BC7
:10E0D00063D02B2BB7EE000A08BF01300278A2F103
:10E0E0003003D9B2092961D8F2EE046ADFED4D7A26
:10E0F00007EE103A10F8012FB8EEC77AA2F13003FC
:10E10000D9B2A7EEA67A0929F0EE477AF0D92E2ADD
:10E1100050D0037803F0DF03452B3BD110B4427895
:10E120002D2A73D02B2A62D0A2F130030130092BA3
:10E1300063D80024002303EB830302EB430310F8AE
:10E14000012FA2F13001303B0929F4D9B3F59A7FB0
:10E150001A46B7EE007A28BF4FF49A72072B09D9F6
:10E160001346DFED316A083B27EE267A072BFAD8F3
:10E1700002F007022AB1F2EE046A013A27EE267A8B
:10E18000FBD1002C3BD0C7EE877A5DF8044B20EE24
:10E19000270A704720EE270A704742780130BFEE09
:10E1A000000AA2F13003D9B209299DD92E2ADFED48
:10E1B0001D7AAED143780130A3F13002D1B20929E2
:10E1C000A8D8B2EE047AF0EE475A06EE902A10F87C
:10E1D000013FB8EEE66AA3F13002D1B2C6EE076A9B
:10E1E000092927EE257A77EEA67AEED992E782788A
:10E1F0000230A2F13003092B9BD9B7EE007A67EE0B
:10E20000877A5DF8044B20EE270A70478278023047
:10E21000A2F13003092B01D801248BE7B7EE007A75
:10E22000B1E700BF0000000020BCBE4CF8B5164DA1
:10E230006B78BE2B25D1AC1C144F022229464FF619
:10E24000FF70FFF7C9FE22884AB1A618BE4218D255
:10E25000052A16D921463446FFF7BEFEF3E72146CC
:10E260000222FFF7B9FE0222A1180634FFF7B4FE1E
:10E27000074B641B9C8041F60F53C31A5842584108
:10E28000F8BD0020FCE700BF004000080080000847
:10E29000744F0120F0B5067906F0E003402B03D15E
:10E2A00045794FF0FF3406E0602B4FF00105F8D1BF
:10E2B000447905FA04F40023012006F00706AB4276
:10E2C00000D1F0BD052E0FD8DFE806F00308101DC1
:10E2D000242448B1C85CD75C78400FE020B1C85610
:10E2E000D756C71B784278410133E8E70028FBD0B6
:10E2F00031F8130032F81370784080B220420CBF1E
:10E3000001200020F0E70028EED031F9130032F9A7
:10E310001370E6E70028E7D051F8230052F8237085
:10E32000DAE7037903F01803102B1DD004D82BB1C2
:10E33000082B06D000207047182BFBD1B0F80B003B
:10E340007047114BB0F80B0093F90030591C09D1FC
:10E350000E4B1B7A03EB830203EBC20300EB83003B
:10E3600080B27047DBB2F5E7074BB0F80B0093F9CA
:10E3700001305A1C06D1054B5B7AC3EB031300EB4B
:10E380004300EDE7DBB2F8E7A0030120744F012062
:10E39000114A00234FF0280C0360838030B54FF4FE
:10E3A00048744FF0290E02F10C0503EB4303AA4217
:10E3B00000EB430100F813C081F801E0D3788C80B2
:10E3C0008B7008D092F90630063292F801C092F8AC
:10E3D00002E09488E9E730BDEC490508092917D027
:10E3E000B1FA81F35B0999B1013903604B0001F087
:10E3F000030103F00802C1EB01119300C1EB01110D
:10E40000A3EB92038900C3EB031381809B0043803D
:10E41000704700BF144B1522144910B50446186804
:10E420001B79206204F1250084F8243045F08BF834
:10E430000F4B4FF0010E1A7E84F83AE012B984F8BF
:10E440003B2010BD03F11C0CBCE80F002060616094
:10E45000A260E360BCE80F0084F83BE020616161EA
:10E46000A261E36110BD00BF48B7050850B70508B9
:10E47000744F01202DE9F84338220021064644F06C
:10E4800021FF01230922174C4525B373412186F84A
:10E49000213041F61E63DFF86090671EF384124B53
:10E4A00009F108083272B362104B114A336103F16B
:10E4B000C87303F2B63373610E4BC6E906234846B0
:10E4C00045F007F8631E294628B1DA1B4045A0EB4A
:10E4D000090338BFF25415B114F8015FEFE7BDE846
:10E4E000F88300BF61B705081E7D01016400DC05EB
:10E4F0000019750343080E0014FC0508202108B517
:10E5000044F0E7FF034618B11A780130202AF9D009
:10E51000184608BDB5EEC00ADFED357A0023F1EEEE
:10E5200010FA70B5C8BF30EE270A86B0D8BF30EEFB
:10E53000670ADFED307A054603A902936E4620EEA6
:10E54000270ACDE90033FDEEC07A17EE904A84EA3F
:10E55000E470A0EBE4703BF06BFB002C03A8ACBFB5
:10E5600020232D238DF8003042F0B4FB012829D060
:10E57000022833D003281DD003A9304644F09AFF67
:10E58000304642F0A7FB044631462846033CE4B23D
:10E59000224644F023FE002328462B5542F09AFBE6
:10E5A0002E22431C31192A54E81844F09FFF2846B4
:10E5B00006B070BD302303A930468DF8013044F019
:10E5C00079FFDDE7302303A930468DF801308DF85F
:10E5D00002308DF8033044F06DFFD1E7302303A9FA
:10E5E00030468DF801308DF8023044F063FFC7E704
:10E5F0006F12033A00007A4408F050BF13B568B1B7
:10E600004C1E14F8011F21B902B0BDE8104008F0FB
:10E6100059BF019008F042FF0198F2E702B010BD27
:10E620002DE9F3410023124D044600EB8106114F02
:10E6300005F83C3FB44203D10F4802B0BDE8F08179
:10E64000394628464FF0000844F034FF214668461A
:10E6500044F04CFF2021684644F03BFF28B969464E
:10E660002846043444F026FFE4E780F80080F1E710
:10E67000744F0120CD0A0608B04F0120014B186EDF
:10E6800031F008B8744F0120084B024608498B420C
:10E690000AD2184602E01C30884205D20388C3F330
:10E6A0000B039A42F7D1704700207047B0820608EA
:10E6B0008C8B060870B50546B0F80900FFF7E4FF3B
:10E6C000064B0446284693F86460FFF72AFE16B10D
:10E6D000E368184470BDA368FBE700BF744F0120D6
:10E6E00038B505460C46FFF7E5FF2B7903F0E0024D
:10E6F00003F00703602A2AD1052B0CD8DFE803F0CA
:10E70000030B0F0B1B1B6A79012393400278DBB2CA
:10E7100014B11343037038BD22EA0303FAE76A79A0
:10E720000123934002889BB214B113430380F2E7A4
:10E7300022EA0303FAE701236A7903FA02F2036883
:10E7400014B113430360E6E723EA0203FAE7052B5B
:10E75000E1D8DFE803F00303050507070470DAE7F3
:10E760000480D8E70460D6E770B585880B46044678
:10E770000021C5F30B0518462A4644F0A3FD616944
:10E78000084A0346914202D3074A914205D319B180
:10E790001846BDE87040084770BD2A46BDE8704085
:10E7A00044F01CBD8C8B0608998D060838B5064CC4
:10E7B000064DAC4206D2A16820461C34FFF7D4FFB8
:10E7C000AC42F8D338BD00BFB08206088C8B060877
:10E7D0000823484010F0800F4FEA400182EA4000D1
:10E7E0000CBFC8B2C0B2013BF4D1704730B5056868
:10E7F0008D421AD901F1FF3E6C1E00231EF801CF95
:10E80000082183EA0C0313F0800F4FEA430C82EADD
:10E8100043030CBF5FFA8CF3DBB20139F3D17445CB
:10E82000ECD16A1C02602B7030BD00236A1C0260B0
:10E830002B7030BD9FED067AF7EE007A60EE870A06
:10E8400020EE800A70EE277A80EE270A704700BF1C
:10E85000DB0FC940B0EEC07AF0EEE06A86FE876A50
:10E86000B5EE406AF1EE10FA3DD0C6FEC75AC5EECD
:10E87000867ADFED1E2ADFED1E3ADFED1E4A9FEDA0
:10E880001E5A9FED1E3AB7EE006A9FED1D4ADFED5E
:10E890001D5AE7EEE23AA7EE834AE7EEA34AA7EE57
:10E8A000846AA7EEA45AE7EE855AC5EE867AF4EE9E
:10E8B000C76AF1EE10FA03D59FED137A77EE677A07
:10E8C000F5EEC00AF1EE10FA03D59FED107A77EE5F
:10E8D000677AB5EEC00AF1EE10FA48BFF1EE677A3A
:10E8E000B0EE670A7047DFED077AE0E739094E3D81
:10E8F000E3B59E3E88FA163E45FE7F3F99FB243FD6
:10E9000069A2163EA7DFA834DB0FC93FDB0F4940E1
:10E9100091ED056AD0ED017AD1ED036A91ED047AAB
:10E9200067EEA66AD0ED005A27EE877AD1ED014A4C
:10E9300067EE867A91ED025A91ED004AA4EEA57A2F
:10E9400090ED026AE5EE257AD1ED064AE4EE256AFD
:10E9500091ED075AD1ED085AA5EE067AE5EE867AD2
:10E96000E4EE866A80ED017AC0ED027AC0ED006ABD
:10E97000704700BFDFED277AB4EEE70AF1EE10FA38
:10E980000CDDDFED256A9FED257AF0EE407A30EE62
:10E99000660AF4EEC77AF1EE10FAF6DCDFED207AC3
:10E9A000B4EEE70AF1EE10FA0CD5DFED1B6A9FED2D
:10E9B0001D7AF0EE407A30EE260AF4EEC77AF1EED8
:10E9C00010FAF6D4DFED187AB4EEE70AF1EE10FA99
:10E9D00014DDDFED107A37EEC00A60EE006A9FEDBD
:10E9E000136A9FED137ADFED137AA6EE867A20EE96
:10E9F000266AE6EE877AA6EE270A7047DFED0E7AE2
:10EA0000B4EEE70AF1EE10FAE7D5DFED057A37EE5E
:10EA1000C00AE2E7DB0F4940DB0FC940E4CB1641F7
:10EA2000DB0F49C0E4CB16C1DB0FC93F92E741B908
:10EA30009730083C15A82ABEDB0FC9BFFDEEC07A8F
:10EA400017EE903A2033402B00D893E79FED010A50
:10EA5000704700BF00000000D0ED005A9FED2B4A28
:10EA600008B535EE840AFFF7E9FFB0EE405AB0EE84
:10EA7000650AFFF7E3FFD0ED014AF0EE405A34EEAD
:10EA8000840AFFF7DBFFF0EE403AB0EE640AFFF7CE
:10EA9000D5FF90ED023AF0EE404A33EE040AFFF75C
:10EAA000CDFFB0EE404AB0EE430AFFF7C7FF25EEB8
:10EAB000236A65EE046AC1ED024A25EE847A25EEEA
:10EAC000005A81ED086A23EE844A23EEE53AB0EE5F
:10EAD000666A65EE805A81ED004AB0EE454A81EDE6
:10EAE000053A60EE637AA4EEE56AA4EE874AE4EEA6
:10EAF000E65AC1ED017AA4EE857A81ED046A81EDD2
:10EB0000034AC1ED065A81ED077A08BDDB0FC93F04
:10EB1000B7EE001A0022DFED050A10B544F090FDB3
:10EB20000023836143610362C36110BDF304353F79
:10EB30002DE9F04F1F461346894689B013F8011B93
:10EB4000002900F02B8215468046002609E0404649
:10EB500001361D46C8472B4613F8011B002900F05B
:10EB60008C802529F3D16978302900F0DD800235C9
:10EB70000023A1F1300C5FFA8CF2092A4FF0000259
:10EB80005ED96C297DD07829E5D8572967D9A1F1BC
:10EB900058002028DFD801A454F820F01DEE00080A
:10EBA00057EB000857EB000857EB000857EB00083D
:10EBB00057EB000857EB000857EB000857EB00082D
:10EBC00057EB000857EB00085BED000869ED000803
:10EBD00057EB000857EB000857EB000857EB00080D
:10EBE00057EB000857EB000857EB000857EB0008FD
:10EBF00057EB000853ED000857EB000857EB0008EF
:10EC000057EB000857EB00083FED000857EB0008F2
:10EC1000C3ED000857EB000857EB00081DEE000895
:10EC2000BEF1050F18D9BAF1050FAAD80A2CA8D140
:10EC300002EB820215F8011B04EB4202A1F1300C39
:10EC40005FFA8CF0A1F1610EA1F1410AA1F1370444
:10EC50000928E5D86446EBE7A1F15704E6E761B17E
:10EC600025297FF478AF25214046C8472B46013639
:10EC700013F8011B00297FF474AF304609B0BDE8DA
:10EC8000F08F15F801CBBCF1780F3FF664AFBCF103
:10EC9000570F4DD9ACF1580120293FF65CAF01A0C8
:10ECA00050F821F07FEE000857EB000857EB000802
:10ECB00057EB000857EB000857EB000857EB00082C
:10ECC00057EB000857EB000857EB000857EB00081C
:10ECD0005BED000831EF000857EB000857EB000828
:10ECE00057EB000857EB000857EB000857EB0008FC
:10ECF00057EB000857EB000857EB000853ED0008EE
:10ED000057EB000857EB000857EB000857EB0008DB
:10ED10003FED000857EB0008DFEE000857EB000856
:10ED200057EB00087FEE0008A9780123033520E7A0
:10ED3000BCF1000FA1D0BCF1250F94D00BE757F820
:10ED4000040B0023494600904046FFF767F906444C
:10ED500001E757F8043B1E60FDE657F8041B4046E8
:10ED60000136C9B2C847F6E6D7F800C0BCF1000FBB
:10ED7000C0F2AC8005ACA246BCF1090FE6464FF0EC
:10ED8000010108DD01EB81014900BCFBF1F009281C
:10ED9000F8D800293DD08948BEFBF1FBBBF10A0F32
:10EDA000A0FB01C001FB1BEE34BF4FF0300C4FF055
:10EDB000570CC0080929DC4401460AF801CBEAD8FF
:10EDC00027E038680121092809D901EB81014900B0
:10EDD000B0FBF1F4092CF8D8002900F0E68005AC6E
:10EDE0000393A246754BB0FBF1FBBBF10A0FA3FBEB
:10EDF000013C01FB1B00B4BF4FF0300E4FF0570E2B
:10EE00004FEADC0C0929DE4461460AF801EBE9D837
:10EE1000039B043700218AF8001029E057F804AB5F
:10EE20000120BAF10F0F40F2C6800001BAFBF0FCDE
:10EE3000BCF10F0FF9D8002800F0BA8005ACA3464A
:10EE400001E0BAFBF0FCBCF1090F4FF0300E05DD1C
:10EE500058290CBF4FF0370E4FF0570EE64400FB19
:10EE60001CAA00090BF801EBEBD100218BF8001074
:10EE7000494640460094FFF7D1F806446BE657F840
:10EE800004BB0121BBF10F0F40F28D800901BBFBD8
:10EE9000F1F00F28FAD8002900F0828005ACA246D4
:10EEA00001E0BBFBF1F009284FF0300E06DDBCF1AC
:10EEB000580F0CBF4FF0370E4FF0570E864401FB32
:10EEC00010BB09090AF801EBEBD1A3E72D21CCF126
:10EED000000C0DF1150A05AC8DF814104CE757F82D
:10EEE000040B0121092808D901EB81014900B0FB7D
:10EEF000F1F4092CF8D8002952D005AC0393A246AE
:10EF00002E4BB0FBF1FBBBF10A0FA3FB013C01FB55
:10EF10001B00B4BF4FF0300E4FF0570E4FEADC0C21
:10EF20000929DE4461460AF801EBE9D8039B71E741
:10EF300057F8040B002829DB05ACA24609284FF03E
:10EF400001010AD901EB81014900B0FBF1FCBCF1E0
:10EF5000090FF7D800293FF45DAF0393174BB0FBBF
:10EF6000F1FBBBF10A0FA3FB013C01FB1B0034BF0B
:10EF70004FF0300E4FF0570E4FEADC0C0929DE44FB
:10EF800061460AF801EBE9D8039B43E72D21404293
:10EF90000DF1150A05AC8DF81410CFE70E466CE69E
:10EFA00005ACA24636E7584678E705ACA24630E7FE
:10EFB00005ACA34659E7D44640E700BFCDCCCCCC46
:10EFC00073B5114C06460D460192A06EA0B10F49D3
:10EFD000FFF714FB3146A06EFFF710FB0C49A06E43
:10EFE000FFF70CFB0B49019B2A46A06EFFF7A0FD23
:10EFF0000949A06EFFF702FB94F86C3013B10123AE
:10F0000084F86D3002B070BD744F012029FC0508F2
:10F01000BEFF0508F9E5000836FC05080EB400B58A
:10F0200084B0084905AB019001A853F8042B039361
:10F03000FFF77EFD019B00221A7004B05DF804EB1F
:10F0400003B070479DE0000800232DE9F0411C4605
:10F0500082B0074603802146013438462AF054FD29
:10F06000082CF8D1002307F1FC06DFF8608087F850
:10F07000EA301D46C7F8EC30C7F8F030C7F8F43076
:10F08000C7F8F8301F462A46414601A83446FFF724
:10F09000C5FF032201A911F8013B5BB1013A04F855
:10F0A000013BF8D1013504362770082DEBD102B0B1
:10F0B000BDE8F081013520462021144444F002F9D6
:10F0C000082D06F104062770DDD1F0E76CB70508BE
:10F0D000F7B5114E074600230C46304615460F493A
:10F0E0006E3600F86E3F04EB45050D4B002F08BF50
:10F0F00019460C4F44F0DEF9AC4202D10A4803B085
:10F10000F0BD394634F8022B6846FFF787FF6946A1
:10F11000304644F0CFF9EFE7744F01203AFC050880
:10F1200043FC05084CFC0508E24F0120F7B500231D
:10F130000B4E044600EB41050A4F06F89F3FAC42D8
:10F1400002D1094803B0F0BD394634F8022B6846B5
:10F15000FFF764FF6946304644F0ACF9EFE700BFC3
:10F16000744F0120A7FC050813500120F8B54E1E6E
:10F17000054601F11F04054F16F8012F28463946B0
:10F180000235FFF74BFFA642F6D1F8BD51FC05084A
:10F1900003685A1C02601970090A03685A1C02604D
:10F1A0001970704702681146531C0360D31C11F894
:10F1B00002CB01605178036093781B0443EA01237A
:10F1C000111D43EA0C030160D07843EA00607047E8
:10F1D000A0F13003092B07D920F02000413819286D
:10F1E0008CBF00200120704701207047303809286B
:10F1F0008CBF002001207047413819288CBF0020A7
:10F2000001207047613819288CBF00200120704709
:10F2100020280BD0092809D00A2807D00D2805D0AE
:10F220000B3801288CBF0020012070470120704757
:10F23000A0F14103192B98BF20307047A0F1610362
:10F24000192B98BF2038704710B56FF00044024664
:10F25000044404E0B3EB0E0015D1A24214D012F81E
:10F26000013BA3F14100192811F8010BA0F1410C59
:10F2700098BF203300F1200EBCF1190FEAD91B1AF8
:10F2800004D10028E9D110BD002010BD184610BDE2
:10F2900002B3844610B5841804E0B3EB0E0014D119
:10F2A000A44513D01CF8013B11F8010BA3F1410256
:10F2B00000F1200E192AA0F1410298BF2033192A2B
:10F2C000EBD91B1A04D10028EAD110BD002010BDD3
:10F2D000184610BD1046704770B5044608460D46E6
:10F2E00041F0F8FC064602E014F8013F43B1204625
:10F2F00032462946FFF7CCFF0028F5D1204670BDE5
:10F300001C46204670BD38B507490546FFF7E4FFA7
:10F31000041E0649284618BF0124FFF7DDFF08B187
:10F3200044F00204204638BD56FC05086012060869
:10F330002DE9F041064686469EF800C070460EF163
:10F34000010EBCF1200FF7D0BCF1090FF4D0BCF1D5
:10F350000A0FACF10B05EFD0ACF10D04B4FA84F454
:10F360006409002CE8D1012DE6D9BCF12B0F3DD06A
:10F37000BCF12D0F39D0102A86463DD04FF0FF3515
:10F380009046B5FBF2F502FB05F7FF43FFB20EF125
:10F39000010E002010E0ACF1300C5FFA8CFC9445BB
:10F3A00012DA8542764602D334D1674532D21C4008
:10F3B0004FF0FF301EF801CBBCF1390FEBD94CF008
:10F3C000200CBCF1600F0BD801B10E602CB3B0F172
:10F3D000004F2BD9DB0729D54FF00040BDE8F08165
:10F3E000ACF1570C5FFA8CFCD9E70124102A00F12C
:10F3F000010E90F801C0C1D1BCF1300F19D04FF00F
:10F40000FF354FF01008B5FBF2F502FB05F7FF439F
:10F41000FFB2BCE708FB00C0CCE70028DEDA13F03F
:10F42000010F18BF6FF00040BDE8F0814042BDE819
:10F43000F0819EF801C00EF10106ACF14105604675
:10F44000192D01D80CF1200078280BD04FF0FF3592
:10F450004FF01008B646B5FBF2F502FB05F7FF4387
:10F46000FFB294E710229EF802C06FF070450EF1D3
:10F47000020E0F2790468AE701230A22002157E750
:10F4800070B50D461446FFF739F80646A0B1FFF7F0
:10F49000F3FF40F634039842A8BF1846B0F5617FE9
:10F4A000B8BF4FF46170A0F561731920B3FBF0F39E
:10F4B0002B702378013323703046FFF71FF8064680
:10F4C000A0B1FFF7D9FF40F634039842A8BF184611
:10F4D000B0F5617FB8BF4FF46170A0F5617319207A
:10F4E000B3FBF0F36B70237801332370304670BDAB
:10F4F0002DE9F04117461E4605464FF47A72002367
:10F5000038463146454C42F0A9F84549454A014440
:10F51000454882FB01C34FEAE17C0B44CCEB63130B
:10F5200082FB03C24FEAE37C1A44CCEB621284FBF9
:10F5300002C44FEAE27CCCEBA40C80FB0C404FEA07
:10F54000EC74C4EBE010C3EB0314A1EB8401A971CC
:10F55000C2EB0211A3EB81036B710CEB4C03A2EB2A
:10F56000C30240F2B55303FB10CC80002A71BCF5F6
:10F57000896F44DA40F2DA239C4547DCBCF5B77F5B
:10F580002A4BB4BF0022012202EB42014FEA42089B
:10F5900003EBC10391B2B3F8523008EB020E244CD6
:10F5A00004EBCE044FF00B0E163401E034F8023DAC
:10F5B00063451FDDBEF1010EF8D11C4B42444FF0F4
:10F5C000010E03EBC202938F00F5FA600CF1010CFF
:10F5D0004FF47A7285F802E00844ACEB030C314634
:10F5E00000232880384685F803C042F037F82A8186
:10F5F000BDE8F0810EF1010E5FFA8EFEE4E7032113
:10F6000040F296534FF006080A46C6E7022140F240
:10F6100029434FF004080A46BFE700BFABAAAA2A55
:10F6200080BC92C78988888873B06D16C449050864
:10F63000004A050808B50D4BD3E9002352EA030C34
:10F640000AD10146002340F2011218460B804A807D
:10F650008B808B710B8108BD054909688A1843F1BD
:10F660000003FFF745FF012008BD00BF88280120E7
:10F67000841B012090420B462DE9F041B0FBF2F6CD
:10F680000446154608D2124A05FB16441846135D77
:10F6900000F8013BBDE8F0819642B6FBF2F706D2D6
:10F6A0000B4A05FB1767D15D03F8011BECE7BA4273
:10F6B000B7FBF2F807D905FB1878054A12F80810CD
:10F6C00003F8011BEDE74046FFF7D4FF0346F2E7DE
:10F6D00074B7050830B5684C83B0B4F8D433B3F5CB
:10F6E0007A7F03D94FF47A73A4F8D433B4F8D633BD
:10F6F000B3F57A7F03D94FF47A73A4F8D633B4F80C
:10F70000D803B0F57A7F04D94FF47A731846A4F879
:10F71000D833B4F8DA13B1F57A7F03D90023194648
:10F72000A4F8DA33B4F8DC23B2F57A7F04D94FF4C5
:10F730007A731A46A4F8DC33B4F8DE33B3F57A7F73
:10F7400002D90023A4F8DE33884202D80021A4F8AD
:10F75000D813934202D30023A4F8DC33B4F8EA238D
:10F76000B4F8EC339A4202D90023A4F8EA33434BAD
:10F770001B8803B3424DAA78062A43D8414901EBBE
:10F78000820191ED270A2979002940D194F8F413D8
:10F7900007EE903AAB7907EE101AF8EEE77AF8EE3A
:10F7A000C76A86EEA77A0BB130EE000AB4EEC70A3C
:10F7B000F1EE10FA30DC637A032B14D8C3EB031399
:10F7C000314A02EB4302237A032BC4F8FC2312D8FC
:10F7D00003EB83012D4A03EBC10302EB8303C4F85F
:10F7E000003403B030BD0023274A6372237AC4F883
:10F7F000FC23032BECD90022244B2272C4F80034E2
:10F8000003B030BD29799FED220A0029BED0042A19
:10F8100021D8002ACFD021E067EE807ABCEEE77ACB
:10F820008DED017A9DF8042007EE102AB8EEC77A14
:10F83000F4EEC77AF1EE10FA01DD0132D2B2CAB1AC
:10F84000102AA8BF1022D2B28A42134638BF0B46F4
:10F8500084F8F433AFE7053A032AACD9F7EE007A1F
:10F8600087EE800A42F042FF2B88984228BF184654
:10F870002880A0E70122E6E7744F01208C1F0020BA
:10F8800068240120C44905083C500120B4500120DF
:10F890006F1203382DE9F04FDFF8F49283B099F836
:10F8A000043400AFA3F11702022A00F24D82AD4BDF
:10F8B0007B603AF01BFE002800F0688200240220E2
:10F8C00089F87C440CF09AFA99F88034022B00F005
:10F8D000D482002800F04D83A34B4FF47A7599F839
:10F8E0004DC5002403F524764FF0640E5A88B2F516
:10F8F0007A7FB3F8462088BF5D80B2F57A7F9A8818
:10F9000088BFA3F84650B2F57A7FDA8888BF9D8019
:10F91000B2F57A7F01D90022DC80998803F1660074
:10F920009142B3F85A10B3F85C2098BF9C80914282
:10F9300093F86B20194602F1FF3288BFA3F85A40B2
:10F94000632A93F86C2002F1010288BF83F86BE010
:10F95000D2B2092A4FF0000288BF83F86C4091F8B8
:10F960000AB0013210F801AB0631D34538BF00F8B8
:10F97000014C032AF3D1BCF1010F03F1A40318BF1A
:10F9800003F81F4CB342B1D1784EB378042B00F08A
:10F99000AB8223B93388B3F5F07F00F2FB81FFF728
:10F9A00099FE734899F86015FEF718FD103099F824
:10F9B0007F15FEF713FD99F88D150E30FEF70EFD3D
:10F9C000B9F89835B9F89A15B9F89C250B43134343
:10F9D0001BB213B10123A9F89E35D9F83C35654A0D
:10F9E0001A40002A00F0D482DA0700F12D825D046B
:10F9F00040F1D4816049D9F840250B400A40C9F84C
:10FA00003C35C9F8402513F4004200F00182002281
:10FA100089F8B32589F8C325D90440F1038299F800
:10FA2000E335022B02D1012389F8E335534D2B46F0
:10FA300005F1780402E006339C420CD01A78072ABC
:10FA4000F9D19978DA78914202D35A79002AF2D022
:10FA500007201DF0CDFA00234FF4806089F87C3434
:10FA60000CF0CCF9002800F07782DFF810B1DA460C
:10FA70009AF8051079B19AF8000050B12B4602E0CF
:10FA80000633A34207D01A788A42F9D15A79002A5C
:10FA9000F6D01DF0ADFA0AF1060A5445E8D1B57862
:10FAA000082D00F0DF8199F84D3599F8D123A3F1A5
:10FAB0000103032AB3FA83F34FEA531389F860363C
:10FAC00099F84E35A3F10103B3FA83F34FEA5313C8
:10FAD00089F86436D9F84035C3F3C03189F8621625
:10FAE00002D9002289F8D1232549D9F83C250B40B9
:10FAF0000A4099F81610C9F84035C9F83C25002984
:10FB000000F0E181B9F87836002B40F0D281D9F8C5
:10FB10007C3613F07F4F02D00023C9F87C36D9F829
:10FB20008436184A1A401AB140F20223C9F88436C2
:10FB300099F88036013B042B02D9012389F88036DD
:10FB4000053D032D40F258810F4B93F890A5BAF173
:10FB5000000F34D000233B606FF007020B4DA2EB87
:10FB600006081CE0C4490508B4500120682401209F
:10FB7000E454012009600002F6DFFFFD5C5501201E
:10FB8000FEDDDDFDFDFDFFFF8C1F00207024012048
:10FB9000744F012008EB05018A4540F2038115F8F6
:10FBA000010B0028F6D009F0E3F80028F2D08179A3
:10FBB0008B07EFD53A680123002A40F0F880B3792B
:10FBC0000BB10023B371B9F88E3613F00C0F03D1CB
:10FBD000C3F30313022B03D94FF42063A9F88E3625
:10FBE000B9F8903613F00C0F03D1C3F30313022BB3
:10FBF00003D940F60123A9F8903699F8FD2699F823
:10FC000009379A4200F2ED8099F8FC3699F80827F6
:10FC10009A4204D2002389F8FC36A9F8003799F8F3
:10FC2000FE2699F8F2379A4202D9002389F8FE3667
:10FC3000BA4D05F1780A15F8012C2B467968002099
:10FC400002EB42020A4492F870E292F871C292F812
:10FC500072621A7801307245A8BF724603F8012B10
:10FC600059799A786145A8BF6146B242A8BF324629
:10FC7000032859719A70ECD11E35AA45DBD1D9F809
:10FC8000D425002A00F027810020012103E00BF198
:10FC9000060B5C4511D09BF80030282BF7D19BF860
:10FCA0000130043301FA03F31342F0D00BF1060BD9
:10FCB00022EA030201205C45EDD108B1C9F8D42540
:10FCC000974D05F108042B4613F8012B072A7AD823
:10FCD0009C42F9D1E84688B02022FF216E4630468A
:10FCE00043F0F0FA8E4A12F8013B56F82310013126
:10FCF00070D1944246F82330F5D1B9F84625C5466F
:10FD0000B9F844359A4202D3864BC9F84435864B3C
:10FD1000FF22864C03F16C0089F8242893F9042013
:10FD2000142A04D0196834EA010100F0DA800C3397
:10FD30008342F3D17E4B5A79022A01D100225A71B3
:10FD40000C37BD46BDE8F08F7A4A11467A60DA007A
:10FD500001EBC30393F8B81021B1D3F8BC30002BEA
:10FD600000F0D7807B68134493F8B920002A3FF451
:10FD7000A0AD93F89831002B7FF49BAD182389F840
:10FD800004343AF0B3FB00287FF498AD66480AF0DB
:10FD9000ECF893E54FF4F073338000E61C075CD574
:10FDA000654928E63A680023002A3FF408AF727CD0
:10FDB000002A7FF408AF7279012A3FF400AF002BCC
:10FDC0007FF4FDAEFFE6E84688B02022FF216846BA
:10FDD00043F078FA002305F8013B0133082BFAD1F0
:10FDE0008BE7002299F8FC3689F8FD26002B3FF4BA
:10FDF00016AFA9F8002709E7002333714F4B93F89A
:10FE000090A5BAF1000F00F0C18001233B60A3E68A
:10FE100099F8B31500293FF4FFADD90489F8C3253B
:10FE20003FF5FDAD1A067FF5FAAD99F804141829CF
:10FE300006D80122424B8A401340002B7FF4EFADDD
:10FE4000404D05F1780406E63F49D9F840250B40BE
:10FE50000A40C9F83C35C9F8402598047FF5D3AD70
:10FE60003A49C8E5B379002B3FF41DAE737C012BF2
:10FE70007FF419AE0223737415E600283FF42CAD0D
:10FE8000334BFF2690F9045099F8CD1403F16C0020
:10FE900093F90820AA4203D1013901241E72C9B284
:10FEA0000C338342F4D1002C3FF416AD89F8CD1405
:10FEB00012E599F8740608F05BFF00287FF427AE7E
:10FEC000A9F8780623E623490A430B43C9F83C25E1
:10FED000C9F8403516E628201DF08AF8D9F8D4254F
:10FEE000D2E689F8242825E7D9F83C25D9F8403509
:10FEF000718C22F4805223F48053B1F57A7FC9F8D3
:10FF00003C25C9F84035BFF44AAD4FF47A73738489
:10FF100045E5172389F8043424E700BF3F5001204A
:10FF20007B240120AE014A01805301200100020020
:10FF3000442B0120C4490508FE9FFFFD8C1F0020B3
:10FF4000004100015C550120F79FFFFDF6BFFFFD5A
:10FF50004454012020041500D9F83C3523F00063F7
:10FF6000C9F83C35D9F8403523F00063C9F840356D
:10FF70007BE5D9F83C25D9F8403522F0800223F002
:10FF80008003C9F83C25C9F84035A5E453460EE77F
:10FF9000D9F8402543F0080342F00802C9F83C357F
:10FFA000C9F8402520E500BF2DE9F04FAE4E83B0E3
:10FFB000AE4B4FF0010AD6F83428DFF8F08202F297
:10FFC000DC524345C6F834284CD29B46A84BA94D79
:10FFD0009F1CA74B5988002900F021817A18AA425A
:10FFE00034BF00200120052998BF40F001000028FF
:10FFF00040F01581BBF800003C46C0F30B000BE05D
:020000040801F1
:10000000118814460A44002900F00981AA4280F0B0
:100010000681052940F2038161888142F0D161792E
:100020008B07EDD123885846DBF8081094F804902C
:100030000193FEF799FBBBF80010B9EB113F00F0FC
:10004000F6804FF0000ABBF804100BF11C0B5BF8B4
:10005000140CC1F30B013AF031FA5BF8042CC345E0
:100060001060B6D3D6F83C35834DC6F84035FFF75F
:1000700011FC337AA5F17801804C03EB830203EB8A
:10008000C203727AC2EB021205EB830301EB420258
:10009000C6F80034C6F8FC2319F08AFF4FF0FF338E
:1000A000D6F80004636021F047FB1CF0F3FF05F570
:1000B000956305F5A46103E00633994200F0C18021
:1000C0001A78002AF8D19D78D878854202D35879D9
:1000D0000028F1D096F8E0356421227203EB830307
:1000E00003EB83039B00632BD8BF6423C6F82C3833
:1000F000B6F8E43501FB03F3632B40F3A7801A46FF
:10010000C6F8303800235E4C5E49C6F83438C1F872
:100110001447C6F83838C6F83C38C6F84038C6F830
:100120004438C6F84828A6F84C3886F84E3822F0ED
:1001300037FDB6F86238DFED546A05EE903AB6F84E
:100140005E389FED527AF8EEE55A07EE903A9FED51
:10015000500AF8EEE77AB6F85C1865EEA65AB6F8DB
:10016000503896F8520867EE877A35EE800AC4ED6B
:10017000AF7AFDEEC07A17EE902A07EE901AF8EEED
:10018000E77A2032402A67EE877AC4EDB07A61D8E8
:10019000FEF7F0FBFDEEE57A3E4981ED000A17EE31
:1001A000902A2032402A5BD8B0EE650AFEF7E2FBC7
:1001B000F1EE407A96F86028C1ED017A07EE902AB8
:1001C0009FED357A9FED320AF8EEE77AA7EE870ABF
:1001D000FDEEC07A17EE902A2032402A3DD8FEF775
:1001E000C9FB07EE903ADFED2D6A2D4BF8EEE77A6A
:1001F000C6F87408A3EC010A86EEA77A83ED007AAC
:100200002FF0F6FA16F04AFF264B012250461B68E3
:1002100086F84D28C6F8343803B0BDE8F08FDBF817
:10022000081058464FF0000AFEF79EFA0BE7019BB4
:10023000A11D58469A1FFDF721FE00287FF403AF49
:10024000FFE6F27D003A18BF012243E70A46C6F8EE
:10025000301857E79FED140A9CE79FED130AC0E79B
:10026000DFED117AA6E700BF744F0120B0820608C7
:100270000040000800800008B4500120A0030120C5
:100280000C5501208C1F002088C3E43A17B7D138E1
:10029000DB0FC93FD857012035FA8E3CC0C9FB4857
:1002A000E0570120841B0120000000008C8B060811
:1002B00038B501221C4B032805461C4C83F81C272B
:1002C00020D96A1C00231A490220D2B24FF0140E22
:1002D0005200402A28BF4022C854023301EB030CCD
:1002E0009A420CF801ECF7D8FF2D4FF0FF034FF0C6
:1002F0000E0008BF0222224482F87838BDE8384058
:100300000BF0E8BE00EB800004F5A073257205EB4E
:10031000C00003EB8000C4F8000421F00DFA1FF0C8
:10032000EDFB1FF0BFFCCCE78C1F0020744F0120B9
:10033000EC570120054B0121D3F8BC2883F8B918EC
:1003400042F40012C3F8BC28704700BF744F01206C
:100350000368C3F30D032DE9F041054686B00C4652
:10036000002B41D1394A0120394E0221B242CDE958
:100370000233CDE9040120D3364B9A421CD303F556
:1003800080439A4224D3344B9A4223D903F58033D5
:100390009A4221D903F500339A421FD903F500335D
:1003A0009A421DD903F500339A421BD90A21052030
:1003B00008F00AFC3AF050FF034601A902A8039393
:1003C00039F0FEFF80B14FF0FF3006B0BDE8F0819C
:1003D0000B46F2E70323F0E70423EEE70523ECE7FF
:1003E0000623EAE70723E8E71C4E96F8D438012BEA
:1003F00002D16FF00100E8E701232F68D4F80080F4
:1004000086F8D43839F07CFFB0B9154C236923F451
:1004100040732361236943F400732361236943F02C
:1004200001032361C7F80080BFF34F8F39F068FFE5
:10043000236923F001032361002386F8D4380028C0
:10044000D7D12B6804332B60BFE700BF0040000802
:100450000040000800800008FFFF0008744F0120E2
:10046000003C02402DE9F041594F8AB03B78B12B56
:100470006ED1FDF7DBFE80F00104E4B2554B04F0D1
:100480000104554DB3F87F32544EADF80030B542FB
:1004900060D3002C00F09A801022002106A842F0C0
:1004A00011FF4F4B0497DB1B05934E4B1A69002A33
:1004B00005DA4D4A5A6002F188325A601B690123FD
:1004C00000250222694604A88DF82430089540F0E2
:1004D000ABF9022269464FF6FF703F4FFDF77CFDF6
:1004E0000446B74245D30025022201A904A8ADF86D
:1004F000045040F099F9022201A92046FDF76CFD55
:1005000040BA022202A9C043ADF8080004A840F096
:100510008BF9079868B106ABC0F10402294618446C
:1005200042F0D0FE089818B906A904A8FFF710FFFA
:1005300008909DF82430089823B12A4A136943F0A3
:1005400000431361B0FA80F040090AB0BDE8F081C1
:10055000012493E7A9881C3555F8140CC1F30B014D
:1005600039F0ACFF55F8043C1B68834218BF0124E6
:100570008DE7B7F8048002A904A88DF80D50C8F3E0
:100580000B081C3708F10603ADF8083037F81C3C9F
:10059000C3F30B021B0BADF80A2006228DF80C30BA
:1005A00040F042F9062202A92046FDF715FD044657
:1005B00057F8141C424604A840F036F9204657F874
:1005C000141C4246FDF708FD04468AE70120BCE7FB
:1005D00000400008C4490508B08206088C8B060854
:1005E00000800008003C02402301674570B5174DAC
:1005F000FFF750F90122164ED5F83438144685F825
:10060000DC2803F2DC53C5F83438FFF72BFF28B1A0
:100610003378B12B02D1FDF709FE18B9032C0ED0A7
:100620000134F2E70B4A00230121126885F8DC3817
:1006300085F84D1885F8DD38C5F8342870BD0A21D5
:10064000052008F0C1FA3AF007FE00BF744F012000
:1006500000400008841B012001230B4A10B50B4CFD
:1006600082F81C37A375FFF7C1FFFFF79DFC41F22D
:100670000242FF230E20A4F8782884F87A38BDE8D7
:1006800010400BF027BD00BF8C1F0020744F0120CD
:1006900090F88730F7EE002ADFED695A002103EE6B
:1006A000903A90F88B3006EE103A90F88930F8EED8
:1006B000E33A04EE103A90F88A30B8EEC66A04EED7
:1006C000903A90F88D3063EEA57A03EE903A26EEDC
:1006D000256AB8EEC44AF8EEE44AF8EEE33A26EEAC
:1006E000276A24EE254A64EEA54A63EEA53A24EE75
:1006F000064A64EEA74A63EEA73AF0B5514D0626C6
:1007000000F1660EA5F10C0CB7EE005A06FB01F2E3
:1007100090F88670AC180244F0EE456A15E00129A5
:1007200004F1060402F10602EED190F8883007EEDB
:10073000903A90F8903006EE903AF8EEE77AF8EEBC
:10074000E66A27EEA55A66EEA56A237866EE867AF3
:1007500007EE103AB8EEC77A27EE277AFDEEC77A91
:1007600017EE903A66EE847AFA2BA8BFFA2323EAB2
:10077000E3731372637807EE103AB8EEC77A27EE88
:10078000277AFDEEC77A17EE903AFA2BA8BFFA2324
:1007900023EAE37353725CF8213007EE903A002BA2
:1007A000F8EEE77A49DDA37807EE103A90F88C303E
:1007B000B8EE477A03EE103AB8EEC33A37EE677AEE
:1007C00023EE253A87EE272AB0EE627AA2EE037A6C
:1007D00064EEA77A66EEA36A67EE857A27EE877ADB
:1007E000FDEEE77ABDEEC77A17EE103AFA2BA8BFF6
:1007F000FA2323EAE373937217EE903AFA2BA8BF19
:10080000FA2323EAE3730EF801300131A38807EEDF
:10081000903AF8EEE77A67EEA67AFDEEE77A17EE01
:10082000903AB3F57A7FA8BF4FF47A738F4223EAE8
:10083000E3739381BFF673AFF0BDB7EE007AC7E7FD
:100840000AD7233C544C050890F88E306BB3B0F8AF
:100850005A308BB190F88F20642102EB8203C3EBF6
:100860000313B3FBF1F3A0F85A30962312FB03F302
:10087000B3FBF1F3A0F85C3043884BB190F88F30B4
:10088000642203EB8303C3EB0313B3FBF2F3438054
:10089000B0F846304BB1962290F88F3013FB02F33C
:1008A0006422B3FBF2F3A0F84630704790F8213091
:1008B0004BB3438B83B190F82230FA22642113FBAF
:1008C00002F203EB8303B2FBF1F2B3F57A7F4283CA
:1008D000A8BF4FF47A738383838843B1FA2290F8D8
:1008E000223013FB02F36422B3FBF2F38380C3884C
:1008F0004BB190F8223003EB8303B3F57A7FA8BFA6
:100900004FF47A73C380704770B50B4C002504F523
:10091000247694F8863013B12046FFF7B9FE2046BE
:100920000135FFF791FF3046FFF7C0FF042D04F1BA
:10093000A404EED170BD00BFB4500120034BD3F826
:10094000E00808B106F0BEBD704700BF744F01203B
:1009500008B50B4605490246D1F8E00828B104491C
:10096000FEF7E6F8BDE80840E8E708BD744F01204F
:10097000F9E50008024B0146D3F8E008FDF73EBE5A
:10098000744F01200048F5E7620706080CB4C3065F
:1009900007B500D561B905A904980191FFF7D8FF03
:1009A000FFF7F0FF012003B05DF804EB02B07047E1
:1009B0000020F8E708B5FFF7DDFFBDE80840E1E7F4
:1009C00010B504460348FFF7D5FF2046BDE81040A8
:1009D000F0E700BF59FC0508034B0146D3F8E008D7
:1009E00008B106F05BBD7047744F01200CB407B529
:1009F00010F020000BD079B92320FFF7EDFF05A9F7
:100A000004980191FFF7A4FFFFF7BCFF012003B09A
:100A10005DF804EB02B070470020F8E70FB407B5AB
:100A200004A951F8040B0191FFF792FF03B05DF8A0
:100A300004EB04B07047154B1B6870B52BB3002551
:100A4000134E1448FFF7B6FFFFF778FFFCF766FB7D
:100A5000FCF796FB044640B113200BF03BFBFFF77D
:100A600091FF0D48BDE87040A4E73046FFF7D6FF80
:100A7000782D06D80135FFF761FF642008F048F8AB
:100A8000E6E72546FFF77EFFF5E770BD4C1B01202A
:100A9000FF2906085EFC050878FC05080FB407B5B9
:100AA00004A951F8040B0191FFF752FFFFF76AFF09
:100AB00003B05DF804EB04B070472DE9F041037911
:100AC00003F0E002402A50D004D85AB1202A29D09D
:100AD000BDE8F081602A4BD0802AF9D18279417932
:100AE000254812E003F00703052B16D8DFE803F0D2
:100AF000101510150309D0F805102048BDE8F04185
:100B0000CCE7D0F8052051421D48BDE8F041C5E7CB
:100B1000B0F80720B0F80510F6E7B0F90720B0F9F3
:100B20000510F1E746790024164D174805EBC60578
:100B3000FFF720FF012395F8A872A74202D8BDE86D
:100B4000F0411FE7D5F8A4624FEA840856F8242044
:100B50004AB113B90D48FFF70DFF56F808100C48BD
:100B6000FFF75CFF00230134E7E741790948C5E757
:100B70000948BDE8F04191E7CDFC05087EFC050879
:100B800094FC0508C4490508ABFC050807000608E5
:100B9000F4100608BCFC0508E4FC05082DE9F04348
:100BA00087B0224EFCF7AAFA0269838900250188E2
:100BB000044602928268DFF88880019242881C4FC6
:100BC000DFF88090009242681A48FFF767FF15B976
:100BD0004046FFF7EFFE3B689D4212DA3378052B63
:100BE00021D809EB8303D3F86424B388294601355F
:100BF00011480093063636F8043CFFF74FFF062DE8
:100C0000E5D13AF001F881884388CB1A616803FB8B
:100C100001110591FCF7FAFA05990246074807B059
:100C2000BDE8F0433AE70022DFE700BF5C2801207F
:100C30004C280120FCFC050866FD050875FD05082B
:100C40005AFD0508C44905080249034801F5216118
:100C50000EC923E70070F01F92FD050810B575213D
:100C6000044622F057FB01460948FFF717FF1A21F7
:100C7000204622F04FFB01460648FFF70FFF1B21DD
:100C8000204622F047FB01460348BDE8104005E737
:100C9000A6FD0508B9FD0508CCFD050838B50C4DC5
:100CA00095F8D30310F0FD0405D10A48FFF7F6FECE
:100CB0002046FFF7D3FF95F8D333013B012B06D82D
:100CC0000548FFF7EBFE0120BDE83840C6E738BD18
:100CD000744F0120DFFD0508EAFD0508BF4BC04940
:100CE0001A68C04BC0482DE9F04FC04C93B0C04DBE
:100CF000C04FDFF82883B2FBF3F2FFF78FFEB4F8A2
:100D0000E4284FF47A730A20B2FBF3F103FB1122BB
:100D1000B4F9E63892B2B2FBF0F2B748FFF7BEFE84
:100D2000B64AB749B748FFF779FEFFF72BFEA17D1A
:100D3000B54A05EB8101B54BB548D31AD1F87C14FF
:100D4000A288FFF7ABFEB348FFF714FE94F8E8184B
:100D5000B148FFF763FEB148FFF70CFE94F8E918BD
:100D6000AF48FFF75BFEFFF70DFEAE48FFF702FE50
:100D700000210A4694F8EF334E1C0B4113F0010F8B
:100D800008D012B14046FFF7F5FD31463846FFF76F
:100D900045FE0122072E3146ECD1A34E96F86A1586
:100DA00006F5EC7306F13C02012918BF134693F8CF
:100DB000DC30032B02D09D48FFF730FE9C4B96F8A9
:100DC0006A15A3F5CE72012918BF134693F8DC30DB
:100DD000012B02D19748FFF721FE954B96F86A1533
:100DE000A3F5CE72012918BF13461B695B7B012B4B
:100DF00002D99148FFF712FEDFF89882FFF7C2FD93
:100E00000027D4F8EC3808F12009DFF88CB20393FE
:100E100058F8041B29B3012303FA07FA039B1AEAC3
:100E2000030F1CD01AF01F0F19D0844B59F827203C
:100E3000D85D52F8202037B18148CDE90412FFF780
:100E400099FDDDE904125846FFF7E8FDBAF1020FFB
:100E500005D196F83D1711B17A48FFF7DFFD01374C
:100E6000D6E7FFF78FFD94F8F418D4F8F02805EBD7
:100E700081017548137AD1F8B814527AFFF70EFE43
:100E8000724B734819684FF47A73B1FBF3F1FFF7B3
:100E9000C5FD07A8FEF7CEFB38B107A90AA83FF0A9
:100EA000EFFD0AA96B48FFF7B9FDFFF76BFDD4F81A
:100EB0008029002A00F08F8007EE902ADFED666A15
:100EC000B8EEE77AC6EE877AFDEEE77A17EE903A4B
:100ED000624F37F8800C58B107EE900ADFED5E6A7A
:100EE000F8EEE77A86EEA77AFDEEC77A17EE900A5B
:100EF000D4F8001959B107EE901ADFED576AF8EEF1
:100F0000E77A86EEA77AFDEEC77A17EE901AB6F862
:100F10007867642ECDE9000131465148A8BF6421AD
:100F2000FFF7BCFD17F87E3C17F87D2C05EB83031B
:100F300037F87C1C4B48D3F8CC34FFF7AFFD4A4B55
:100F40004A48198889B2FFF7A9FDFCF7D7F801696B
:100F500021B182684648120DFFF7A0FD4548FFF712
:100F600009FDD4F840351B0640F1C68017F8503C07
:100F7000032B8CBF40484148FFF7FCFC94F88034B9
:100F8000022B40F08B803E48FFF7F4FC17F8503CF2
:100F9000042B00F2A8803B48FFF7ECFC17F8403C1C
:100FA000002B00F0A78005EBC303D3F824153648C7
:100FB000FFF734FDFFF7E6FC3448FFF7DBFC0126C2
:100FC000D4F8BC48324F002C40F09A80FFF7DAFC8E
:100FD00013B0BDE8F08F13467AE700BFDC1B012099
:100FE000FDFD050840420F0002FE0508744F012078
:100FF000C4490508BDFE050815FE050800000120CE
:101000000008000036FE05080080000800400008C7
:101010005AFE050889FE05089BFE0508A3FE050883
:10102000A5FE0508ADFE05088C1F0020C6FE0508BC
:1010300064210020CEFE0508D3FE0508AC03012084
:1010400007000608E1FE0508E5FE0508841B0120EF
:10105000F7FE050811FF0508002474496C600120A3
:1010600024FF05086AFF05084422012091FF0508B6
:10107000A0FF0508BBFF0508C1FF0508CDFF050857
:10108000DDFF05083A2A0608250006084100060883
:1010900031000608484E0508DBFE050802200AF06C
:1010A000CDFE064608B91E486EE72EF087FB96F97E
:1010B000041005EB80000131D0F8E0241948FFF757
:1010C000ADFC94F88334012B04D11748FFF752FC90
:1010D000164859E7B379164805EB8303D3F8E014B3
:1010E000FFF79CFCF4E794F882340BB9114853E7FE
:1010F000114851E711495AE71148FFF73BFC59E7FE
:1011000094FAA4F33846B3FA83F306FA03F205EB34
:101110008303D3F8581524EA0204FFF77FFC52E753
:10112000E3FF0508EDFF05080100060806000608B4
:10113000C30906080A0006081A000608F5FD050896
:10114000350006082DE9F04FDFF86C8199B098F86A
:101150000B30002B00F093804E4800254E4EDFF8F8
:101160005CB1FFF727FC2F46DFF85491DFF854A15C
:101170000BA9E8B217F016FF9DF83430002B53D0BE
:10118000139C54B107EE904A9FED440AF8EE677A3B
:1011900080EE270A41F0AAFA04460B9A29465846DF
:1011A000FFF73CFC109A002A6BD002FB04F04FF4CE
:1011B0007A73B0FBF3F30993DDF848C0BCF1000F7C
:1011C00061D00CFB04F142F21073B1FBF3F1082D76
:1011D00098F80B3018BF7F18002B56D017984FF493
:1011E0007A7E0A2307901598069016980590119814
:1011F000B0FBFEFECDF810E00998B1FBF3FE03FB57
:101200001E11CDE902E10999B1FBF3F103FB1100D5
:10121000BCFBF3F3CDE9001021465046FFF73EFC3E
:101220000023B362C6E90D33013540361E2D9FD130
:1012300098F80B3003B31A4C4FF47A73194854E9F9
:101240000F12B1FBF3F3D20854F8341CFFF726FC5D
:101250000A221548B7FBF2F102FB1172FFF71EFCE0
:10126000124B1B78432B04D1114854E90C21FFF792
:1012700015FC002344F8343C19B0BDE8F08F0D484C
:101280006BE7099298E76146A1E721464846FFF7D8
:1012900005FCC5E7570006086C5801208096184BDE
:1012A0006C600120FE0006081E010608E51B0120F7
:1012B00042010608B5000608744F0120BF00060869
:1012C00090100608CE00060813B52948FFF752FB18
:1012D000284B93F8C535002B48D02748FFF76AFB09
:1012E00018F0F2FB80B1254B254893ED280A8DEDCF
:1012F000010AFFF73FFB234B9DED010A33F8803CC9
:101300003BBB2148FFF756FB204C2148B4F814188A
:10131000FFF784FB94F8103813B31E48FFF74AFB1D
:10132000B4F818181C48FFF779FB94F81238CBB1C1
:101330001848FFF73FFBB4F816181848FFF76EFB84
:1013400094F8113883B1134802B0BDE81040FFF79C
:1013500031BB41F0CBF981B21148FFF79FFBD3E7D6
:101360001048DBE70F48E4E70E48EDE70E48EBE7EF
:101370006C010608744F012082010608082700202E
:10138000890106086C600120A30106088C1F00205B
:10139000B2010608D2010608E2010608FC010608AF
:1013A000AD010608DB0106087D4306080EB403B54F
:1013B00003AA52F8041B0192FDF702FE064BD3F874
:1013C000E0281AB90549986EFDF718F902B05DF8E2
:1013D00004EB03B0704700BF744F0120620706089A
:1013E0002DE9F04798460B7981460F4603F0E0045B
:1013F0001646402C31D10024674DDFF8A081DFF87C
:10140000C09122E03B7903F00703013B042B04D891
:10141000DFE803F006080B0E2000315D28460AE0E5
:101420003157FBE736F81410F8E736F91410F5E7F2
:1014300056F824104046FFF7F1FA7B79013BA342AE
:1014400002DD4846FFF796FA01347B79A342D9DCE6
:10145000BDE8F08756F82410E0E703F00703052BFA
:1014600058D8DFE803F0030C141619313578602CD6
:101470005ED045D8002C66D0202C7CD0E8E796F9C9
:101480000050602C54D03BD8002CF5D148E0358872
:10149000EDE7B6F90050F4E7D6F800A0202C554649
:1014A00069D02BD8002CD3D151463C48FFF7B6FA6F
:1014B000D7F805108A4518D8B8F1000FC8D03848B9
:1014C000BDE8F047FFF7AABA202C356853D015D8ED
:1014D000002CBDD129463048FFF7A0FAD7F80510F7
:1014E000A94202DB4B42AB42E6DDFFF74BFA2B464B
:1014F0003A6848462B49BDE8F04757E7602C17D0BB
:10150000802CA5D13178284B2848002914BF3146BA
:101510001946D5E7202C2DD007D8002C98D1254688
:10152000B7F90540B7F9076011E0602CE8D1002554
:101530007B7945FA03F3DB07BDE8F0474CBF1C4855
:101540001C48FFF76BBAB7F80540B7F807602946A3
:101550001148FFF763FAAC42C7DCAE42C5DBB8F115
:10156000000F3FF475AF324621461348BDE8F047FF
:10157000FFF754BA00257A79104B03EBC20393F8B6
:10158000A8229542B1DAD3F8A43253F82500BDE879
:10159000F047FFF7EFB900BFA8FC050891FC05086C
:1015A0001C02060822020608CE2A0608F4100608C5
:1015B000F9FC05087D430608B50A0608C449050874
:1015C000A3FE050813B50446084601920091FDF7F5
:1015D00071F802462046DDE9001302B0BDE8104074
:1015E000FEE60EB403B503AA52F8041B0192FDF700
:1015F000E7FC054B0549986EFDF700F802B05DF871
:1016000004EB03B0704700BF744F01206207060867
:1016100002460149E5E700BF3C020608F8B50C4662
:1016200006460846FDF728FF20210546204641F0E2
:1016300050FF044618B93046BDE8F840E8E7114FBE
:10164000114E3B7832789A4201D0FBF79BFE0F4B4C
:1016500020461D603FF03EFB012201462046FBF77D
:1016600033FE3B7832789A4201D0FBF78BFE20465E
:101670003FF030FB2A4601460548BDE8F840FFF739
:101680000DBA00BF481B012054280120441B012033
:10169000530206082DE9F0410D4688B0064608467B
:1016A000FDF7EAFE20210446284641F012FF20B94A
:1016B000304608B0BDE8F041AAE7FDF7DDFE22465E
:1016C000054601460F48FFF7E9F985B1202D2A4666
:1016D0006946204628BF2022E846FBF76FFE002718
:1016E0000646B74208DBAD1B3444002EEDD1FFF7B0
:1016F00049F908B0BDE8F08118F8010B0137FFF790
:101700006BF9EEE76902060810B504460748FFF7D3
:1017100051F9FBF7E9FE20B10548BDE81040FFF79D
:1017200049B920460349BDE810405AE7810206083E
:101730008B02060893020608154B53F8283C2DE946
:10174000F041044688B0F3B11A6804A91846D56A76
:101750006A46A847064688B104AC6D460027DFF804
:101760003C80013735F8022B34F8021B4046FFF766
:1017700095F9BE42F5DC08B0BDE8F0810549204688
:10178000FFF72FFFF7E7044908B0BDE8F04128E76D
:101790006C600120B4020608CC0206089A02060812
:1017A00013B50446084601913FF094FA024670B121
:1017B0000D2804D10199094841F0B1FE38B1074B19
:1017C0002046074A074902B0BDE8104009E703492F
:1017D000054802B0BDE81040FFF760B950B70508F2
:1017E000D3020608DE0206080803060813B50446FD
:1017F000084601913FF06EFA0199024668B104284B
:1018000003D1094841F08BFE38B1074B2046074A07
:10181000074902B0BDE81040E3E60349054802B0BD
:10182000BDE81040FFF73AB948B7050816030608A7
:10183000DE020608260306082DE9F04300279BB0C8
:10184000064608460C463FF045FA05461C22394636
:1018500002A8019741F036FD25B3402D07D0402363
:101860002A46384930461BB0BDE8F043B9E60DF1D1
:10187000040804F1400902222146684641F063FE53
:101880000023102209A968468DF80270FDF750FD6B
:10189000099B0DF10202934222D1023408F8010B98
:1018A000A145E8D100213D220AA8099141F00AFD95
:1018B000002D3AD0244C257ED5B1202204F11C0104
:1018C00001A841F0D5FC98B104F11C0109A8FDF76D
:1018D0004DFC09AB1D4A30461D49FFF782FE04E06E
:1018E0001A7830461B49FFF77CFE1BB0BDE8F08339
:1018F00094F86430CBB9C5B901AD174C0FCD0FC406
:1019000095E80F0084E80F00144B012209A8A4F108
:10191000100103F8242CFDF729FC1148FFF750F8BB
:1019200009A91048FFF7BAF8DFE70C4B13F8243C7D
:101930001BB9054B1B7E002BF2D0074909A8FDF708
:1019400015FCEDE739030608744F012077030608FC
:10195000DE0206085B030608904F01206C60012040
:1019600081030608900306082DE9F74F3D4F834693
:1019700008460D463FF0AEF9D7F83C950446B8B995
:10198000394D0126394F3A48FEF7F4FF55F8041B4C
:1019900049B106FA04F313EA090F02D03846FFF7FB
:1019A0003DF80134F2E703B0BDE8F04FFEF7EABFBF
:1019B000024630492846FDF76BFC78B92A4C2E4D7B
:1019C0002E48FEF7D7FF54F8041B0029EBD00B7804
:1019D000002BF8D02846FFF721F8F4E72B782D2BC1
:1019E00011D10135013C4FF0010A1F4B002653F87D
:1019F000048BB8F1000F09D12A462149584603B09B
:101A0000BDE8F04FEDE54FF0000AEEE72246414613
:101A100028460193FDF73CFC019B00BB0123B3402A
:101A20009A0505D5174803B0BDE8F04FFEF7C2BFD1
:101A3000BAF1000F0DD029EA03031348C7F83C356B
:101A4000FEF798FF41460C4803B0BDE8F04FFFF7A2
:101A500025B849EA03030D48C7F83C35F0E70136DD
:101A6000C5E700BF744F0120844F0508A70306088F
:101A70009D030608BA00060831000608AB030608F5
:101A8000B6030608C7030608D3030608DC030608E6
:101A90002DE9F74F814608460E46174698463FF017
:101AA00019F90446E8B9404D4048FEF7B7FF204613
:101AB00009F0AEFF3B68184206D0204609F0BAFF95
:101AC00001462846FEF7AAFF0134182CEFD13B68E7
:101AD00013B93748FEF74EFF03B0BDE8F04FFEF7ED
:101AE00051BF024633493046FDF7D2FB0546A8B93F
:101AF0002C46314D3148FEF73DFF204609F088FF66
:101B000010EA080F06D0204609F094FF0146284647
:101B1000FEF784FF0134192CEFD1DDE733782D2B4C
:101B20002AD10136013C012548F080734FF0000AAC
:101B30000193504609F07EFF224683460146304617
:101B4000FDF7A6FB18BB504609F062FF019B03425C
:101B50001DD09DB1BAF1180F02D03B6840EA0308CE
:101B60001748C7F80080FEF705FF5946124803B032
:101B7000BDE8F04FFEF792BF0025D5E7BAF1180F88
:101B800002D03D6825EA00050E483D60EBE70AF10A
:101B9000010ABAF1190FCCD132460B49484603B0BD
:101BA000BDE8F04F1DE500BF30000608E40306085D
:101BB000EE030608BA00060831000608AB03060863
:101BC000D3030608DC030608B603060840F2022326
:101BD000004A5DE7F85501206FF07F43004A57E760
:101BE000F055012010B5044620F0A4FF20B920468E
:101BF0000449BDE81040F4E40348BDE81040FEF796
:101C00004DBF00BFF50306080404060870B505467D
:101C100008461646FDF730FC0D4B044693F8902518
:101C2000904205D201460B48FEF738FF204670BDB2
:101C30002EB1FF2803D10848FEF730FFF6E7013A3E
:101C4000064928464FF0FF34FFF7CBFCEEE700BF14
:101C50008C1F00200F040608200406083304060821
:101C60002DE9F04F074691B082480E46824DFEF7AF
:101C700015FF002381494024062205F81C3C30460C
:101C8000012391F8901545F820DC05F81B4C06F06F
:101C9000E7FC0A2006F03CFF15F81C3C0C2BDAB2DE
:101CA00040F2E4809DF80C50FE2D30D0FF2D0BBF8C
:101CB00015240F2401260026944240F0D780611E8F
:101CC0006846C9B234F0A6F804F140030DEB0304F2
:101CD00014F8413C834240F0C48006F1FF389DF87F
:101CE0000D305FFA88F8B8F1010F12D903F01F0721
:101CF0005C0961376248FEF73DFE022E6AD0013C66
:101D0000042C65D8DFE804F00B5E606462000226F4
:101D1000D2E79DF80E701D469DF80F40EAE759483E
:101D20006C464FF0000ADFF8B891FEF743FEDFF88B
:101D3000B4B15548FEF71EFE0AF1010A14F8011B62
:101D40004846FEF76BFEBAF10C0F49D1FEF71AFEBA
:101D5000022E4FD064223B464C48B5FBF2F102FB09
:101D60001152C9B2D2B2FEF799FEB8F1010F71D883
:101D7000474A484B9DF810104748002914BF1146A8
:101D80001946464DFEF78AFE9DF81110444B454812
:101D9000002914BF19462946FEF780FE022E59D1AC
:101DA0009DF812404048FEF7E5FD4CB3FF2C37D0BC
:101DB0000A223E48B4FBF2F102FB1142D2B2FEF716
:101DC0006DFE20E03A48ABE73A48A9E73A48A7E772
:101DD0003A48A5E700230DF11F008DF83F309FE73B
:101DE000374B03FB0AF2B2F1553FA5D85846FEF730
:101DF000C1FDA1E73A4629463248FEF74FFEB7E754
:101E00002846FEF7D7FD9DF813402F48FEF7B2FD98
:101E100044B1FF2C21D021462C48FEF73FFE04E0C0
:101E20002B48EEE71D48FEF7C5FD0DF11305002414
:101E30001A4E274FDFF8688015F8013F7BB1FF2B62
:101E40000CBF3A464246214601342248FEF726FEA0
:101E5000042CF1D111B0BDE8F08F1D48E3E7324604
:101E6000F1E71D493846FFF7BCFBF3E71B48FEF7D7
:101E7000A1FDEFE7790406086C6001208C1F0020AB
:101E80008A04060895040608BB040608CD04060863
:101E900059040608620406080405060869040608D1
:101EA000331206081B050608220506083605060833
:101EB0009C040608A4040608AC040608F5FD050801
:101EC000ABAAAAAAE90406083E050608A8FC05086C
:101ED0006D0406084E05060859050608690506083A
:101EE00051FC0508CE2A06082DE9F84F07460C4696
:101EF000DFF8A480DFF88490DFF8A0A020463EF051
:101F0000E9FE064660B91D4B1D4893F804241D4B9D
:101F100003EB8203D3F83816BDE8F84FFEF7BEBDD9
:101F2000024641462046FDF7B3F960B1DFF85CB0E8
:101F300000255BF8041BB1B9224638461249BDE8BA
:101F4000F84FFFF74EBB114C114D1248FEF712FD32
:101F500054F8041B19B12846FEF760FDF8E7BDE808
:101F6000F84FFEF70FBD324620460135FDF790F9D8
:101F70000028DED1544689F80454BFE7744F01208D
:101F800072050608C4490508B6030608005005088E
:101F900031000608AB030608BA0006085913060804
:101FA00038B50D460446052219492846FDF770F953
:101FB00068B9184B93F86C2022B9012183F86D2081
:101FC00083F86C101448BDE83840FEF7F3BC0322D8
:101FD00012492846FDF75CF9A0B90E4D95F86C3012
:101FE00063B195F86D304BB10D492046FFF7F9FA12
:101FF000002385F86C3085F86D3038BD0948FEF750
:10200000D9FCF5E720460849BDE83840FFF7E9BAB2
:1020100077110608744F01207C050608DC120608BB
:1020200092050608C9050608DD050608F8B5174C2F
:10203000054694F86C307BB194F86D3063B1144967
:10204000FFF7CFFA28461349FFF7CBFA002084F8B0
:102050006C0084F86D00F8BD0F4E16F8247C97B123
:10206000207E0028F7D10D4DA6F118040FCD0FC426
:1020700095E80F0084E80F00012386F8233007F06D
:1020800009F83846E7E70120E5E700BF744F012073
:1020900092050608EC0506086C600120904F0120AF
:1020A00008B5034610462AB1DB0600D511B1FEF78C
:1020B00087FC002008BDF8B50D4E054696F8643043
:1020C00093B9F8BD25B12388C3F30B039D4204D017
:1020D000A288D4E9020141F081F81C34BC42F1D35A
:1020E000002386F86430ECE7024C034FF6E700BFAC
:1020F000744F0120B08206088C8B06082DE9F04F42
:10210000164685B01A468246019130460021334C6E
:10211000FFF7C6FF4FF0000906F0100305460293D3
:10212000FEF70CFC2379019A03F01803934203D0C5
:10213000002A48D1182B46D14FF00D0B274B0BFB33
:102140000933B3F80900FCF79FFA80462046FCF7F4
:10215000E8F80746D8E90221024401442046FCF78A
:1021600099F880F001012A460390C9B23046FFF782
:1021700097FF0546DDE9022302B123BB174A0BFB9B
:1021800009FB52F80BB0B2060FD573B95946144883
:102190000393FEF743FCD8F808202146039B5046E2
:1021A0003A44FFF71DF9FEF7EDFB59460D48FEF7DF
:1021B00035FCD8F80C20002321463A445046FFF75E
:1021C0000FF9FEF7DFFB09F1010940F262230D343C
:1021D0009945A5D105B0BDE8F08F00BFE0630508C3
:1021E0000A0606080B0606080149FFF7FAB900BF00
:1021F0001506060838B50C46054615492046FDF774
:1022000023F830B9FEF780FB1248BDE83840FEF7EE
:10221000D1BB11492046FDF717F8A0B90F4A82F843
:10222000C60182F8CE0182F86A0282F8720282F850
:102230000E0382F8160382F8B20382F8BA0382F81A
:10224000F1030748E1E72846BDE83840CCE700BF86
:10225000240606082A06060845060608744F0120CB
:102260004D0606082DE9F043064687B008460C46A1
:102270003EF030FD082844D1671E03AD07342946DF
:102280003A46A84612F8010FFCF7D8FF01F8010BF7
:10229000A242F7D10023DFF880908DF8143017F8B0
:1022A000010FFCF7CBFF05F8010BC1B248460191C5
:1022B00041F00FF920B10199284641F00AF928B1FF
:1022C0003046FFF791FF07B0BDE8F083A742E6D1A3
:1022D0001049404620F0BEFB0E4808230E4910F876
:1022E000012B013B11F8014B02F118026A4402F87C
:1022F0000C4CF4D103A909488DF81430FEF7CEFB3D
:10230000E1E70028E8D0304607B0BDE8F043FFF72A
:102310007FB900BF1855012014FC0508690606089E
:1023200007B5009313460A460249FFF75AF903B06E
:102330005DF804FB7006060820B10078B0FA80F062
:1023400040097047012070472DE9F34106460846D1
:10235000FFF7F2FF0D46074670B1002401A92046A1
:10236000013437F065FC01463046FFF7EDFF122CD3
:10237000F4D102B0BDE8F0810846FDF77DF8C4B2A3
:10238000112C72D8681C3D4DFCF7B8F88046E8B9AE
:102390003B4B03EB440393F824108A1E51425141F6
:1023A000374B03EB440393F82420AA5C002955D053
:1023B00093F82530192040F2EE2100FB031321464B
:1023C000304802B0BDE8F041FEF768BB017828460E
:1023D00041F07FF878B1032C2B49A0EB050394BFA3
:1023E0000022012202EB42020A4452FA83F393F8DC
:1023F000A876032F04D1304602B0BDE8F041F3E6E1
:102400004046FCF77BF808B3022FF4D1FDF734F80F
:1024100040F6CA0280B21A4B904203EB4403A8BFB5
:10242000104640F2EE229042B8BF10461922A0F2A8
:10243000EE20B0FBF2F083F82500BB1E5942594153
:102440000F4B03EB440383F82470A9E7022FF4D168
:10245000304602B0BDE8F041FFF7DAB821460B483C
:1024600002B0BDE8F041FEF719BB11233A46084916
:10247000304602B0BDE8F04152E700BF24CC050869
:102480006C60012089060608C449050899060608FB
:10249000A60606082DE9F04F024691B008460B4605
:1024A000FFF74AFF044628B1104611B0BDE8F04FCF
:1024B000FFF7AEB84FF0FF3227462646DFF8E0823E
:1024C000DFF8E092DFF8E0A2CDE90820A24A126E20
:1024D00092F83810CDE90E02CDE90C10CDE90A00D2
:1024E00007AA9E49184640F0AFFE054604944DB930
:1024F000089A0C9FBA4262D19948FEF7CFFA11B000
:10250000BDE8F08F062F12D8DFE807F0041E23285D
:10251000454C510051462846FCF7DEFE78B14FF499
:102520008060012409F08AFC90F90430089307AA1E
:102530008A490020013740F087FE0546D7E7284644
:10254000FCF79AFF0890F2E72846FCF795FF099000
:10255000EDE72846FCF7D7FE0A90E8E728463EF06C
:10256000B9FB4146024605902846FCF791FE18B398
:10257000059A49462846FCF78BFE06460028D6D029
:102580002846FCF779FF04280646D0D9014675484D
:10259000FEF784FAB3E72846FCF76EFF00230C90A1
:1025A0000F93C4E72846FCF767FF0D90BFE7284666
:1025B000FCF7A9FE0E90BAE701230493B7E7DFF812
:1025C000EC8151B2434613F9010B884208D0013522
:1025D000092DF8D1002101316348FEF75FFA8EE73B
:1025E00001216248FEF75AFA00237AB218F9011B5A
:1025F0008A4200F00C810133092BF7D13A460121C0
:10260000E9E7A7F1140253425341059308AD0023B3
:1026100003F10108EB68A3BB95F900B0584609F037
:10262000D9FBD5F804A020B1D0F80090B9F1000F83
:102630005ED1BAF1000F19D14FF461434FF0010A96
:102640006B60AB680BB90323AB600023D5F8049033
:102650005846029319462A7ACDE900921A4609F0A3
:102660003EFCE86028B94146414891E74FF0000A36
:10267000E7E74A464146BAF1000F37D03D48FEF73A
:10268000CDF9B8F1020F05F110054FF00103BFD1EC
:10269000059BDDF83C800B9D53B13748FEF78AF966
:1026A000D8F800301B6A1BB12A4634494046984787
:1026B000049B002B4ED03249324B142F18BF1946C1
:1026C0003148FEF7EBF9142F09D1049B03B936B159
:1026D0002B68DB691BB132462C4928469847002CF1
:1026E00066D100224146284637F056FA2848C6E708
:1026F000C5F80C90BAF1000F25D041462548524646
:10270000FEF78CF95146484603F046F8D5F808A084
:10271000BAF1000F0FD099F8042092450BD0534620
:1027200041461D48FEF77AF9D9F800305FFA8AF180
:1027300048469B699847D9F82C30002BA1D000233C
:10274000C9F82C309DE7D9F8082041461348FEF718
:1027500065F9DBE70B49B3E7744F0120CD0A0608A2
:10276000E4060608CC06060828080608FD06060842
:102770000907060825070608DC0706089957010817
:10278000AE06060859130608050806086155010833
:102790004907060865070608B707060892070608EE
:1027A000C6060608F0030608BB06060872500508B0
:1027B0001C4F0026DFF874904FF0030A05F0D2FC9E
:1027C000052006F0A5F999F89035B34289D917F894
:1027D00001BBBBF1000F15D0584606F0C9FA0446FC
:1027E00080B1584605F0DCFB08B1A0F806A0012135
:1027F0000490F8F7A1F8A379049813F0010F03D01F
:10280000F7F71CFB0136DEE7F7F712FBFAE73A466B
:1028100002210548FEF742F9099B002B3FF4F1AE77
:102820000023F2E670240120FD0606088C1F00201C
:102830002DE9F74F05460846FFF77EFD0B46044697
:1028400018B9334A92F8487027B9284603B0BDE852
:10285000F04FC9E42646DFF8C880DFF8C89001AA27
:10286000DFF8C4A018462B4940F0EEFC10B905F083
:1028700087FC08E056B9012201462846FFF7C6F951
:10288000421C04461BD103B0BDE8F08FFCF7F4FDF9
:102890002F28834636D80FB105F064FCBBF1060F34
:1028A00014D01D4901235FFA8BF291F89015E0B224
:1028B00005F0D6FE002759464846FEF7EFF801AA74
:1028C00014490020013640F0BFFCCFE7DAF840356C
:1028D0001B0113D5FF2C0FD0E1B22846FFF7C0F93A
:1028E000E8E701372846FFF7BBF90B4BF9B293F83D
:1028F00090258A42F5D8DDE70027F6E70748FEF77E
:1029000059F8D7E72F2241462846FEF76AFED6E758
:102910006C600120CD0A06088C1F0020F503060814
:102920004B0806083A080608744F01202DE9F04FBD
:10293000064685B008460B46FFF7FEFC044628B164
:10294000304605B0BDE8F04FFEF762BE03AA30493D
:102950001846274640F078FCA0460546DFF8C090B0
:10296000DFF8C0A0DFF8C0B05DB92A4B3A46A1B28B
:10297000186E38F039FA68BB27493046FEF731FE49
:1029800028E0B8F1000F06D0B8F1010F25D030468D
:10299000FEF73EFE1EE028463EF09CF94946024600
:1029A00001902846FCF774FC50B3019A5146284622
:1029B000FCF76EFC30B3019A59462846FCF768FCD8
:1029C00010B3019A28461549FCF762FCF0B1304675
:1029D000FFF70AFC05B0BDE8F08FBB1E2946304664
:1029E0005A425A41FFF712F9421C0446F2D003AA98
:1029F0000749002008F1010840F026FC0546B3E72E
:102A00004746F4E70127F2E70227F0E70427EEE75D
:102A1000CD0A0608744F01207708060874080608D6
:102A20006B0806086E080608710806082DE9F743CA
:102A300080460846FFF780FC0B46054628B1404615
:102A4000FEF7E6FD03B0BDE8F08301AA2D49184664
:102A50002F4640F0F9FB2E460446DFF8A8907CB9DB
:102A6000022DECD1A7F57A73B3F57A7F21D94FF413
:102A7000FA634FF47A7224494046FFF751FCE1E7CC
:102A80004DB1012D10D001AA49460020013540F07A
:102A9000DBFB0446E3E7012221464046FFF7B6F898
:102AA000431C0646EFD1CDE72046FCF7E5FC074680
:102AB000E9E7164DB8B2D5F830385B689847FF2E75
:102AC000BCEEC00A0CD1F8EE407A95F89025104B78
:102AD000A24213DC10EE101A0E48FDF7DFFFB1E73B
:102AE0000D4BF8EE407A10EE102A314603EB8603C8
:102AF0000A48C3ED137AFDF7D1FFA3E70134E3ECF5
:102B0000017AE5E7CD0A0608850906088C1F002032
:102B1000B8600120A20806086C600120950806082C
:102B2000F8B507460846FFF707FCC8B11F4B5E69BA
:102B300001363046344608F07DFF0546F0B90134D1
:102B4000192CA8BF0024204608F074FF0546A8B938
:102B5000B442F4D138461649BDE8F840FEF741BD0D
:102B60000846FCF789FC044608F064FF054628B9CE
:102B700021461048BDE8F840FDF790BF0B4B5C6163
:102B800009F072FA2A4621460B48FDF787FF182CF8
:102B900009D80A480C2101FB040090F8B806BDE8EA
:102BA000F84009F097BA0020F9E700BFA003012020
:102BB000B1080608C5080608DB080608C449050868
:102BC00038B50446114D0846FFF7B6FB68B1104B07
:102BD00093F900104B1C06D10E4B197A0E48BDE834
:102BE0003840FDF75BBFC9B2F8E70846FCF744FC84
:102BF000032804D8C0B2FDF75BFB2946E3E7204673
:102C000003220649BDE83840FEF7EBBC591306081D
:102C1000A0030120744F0120F408060804090608E7
:102C200038B50446114D0846FFF786FB68B1104BD6
:102C300093F901104B1C06D10E4B597A0E48BDE892
:102C40003840FDF72BBFC9B2F8E70846FCF714FC83
:102C5000032804D8C0B217F09FFA2946E3E72046BC
:102C600003220649BDE83840FEF7BBBC59130608ED
:102C7000A0030120744F0120F0080608FF08060891
:102C8000444B2DE9F74FDFF824A105461A7A884610
:102C90008AF800205A7A93F864308AF801200BB938
:102CA00003F02AFE00263C4CFBF780FDB1460D23C5
:102CB000394A4146734352F803B05846FCF70CFBBF
:102CC000002841D0B9F1000F01D0FDF75BFE594655
:102CD0003248FDF7A3FE002221462846FEF772FC8B
:102CE000FDF750FE237903F01803082B45D0102B75
:102CF00048D02046FDF7E1FE274A0D2303FB0623BB
:102D0000B3F80900FBF7C0FC0746D8B12046FBF733
:102D100008FB0090D7E90221024401442046FBF75A
:102D2000B9FA78B9594601901D48FDF777FE019A26
:102D3000B96828461346009A0A442146FEF750FB1C
:102D4000FDF720FE09F10109013640F262230D343E
:102D50009E42ACD10020FFF7AEF9FF238AF8003085
:102D60008AF80130B9F1000F11D142460D492846C9
:102D700003B0BDE8F04FFEF734BC0B492846FFF71F
:102D80001FFFB6E708492846FFF74AFFB1E703B03F
:102D9000BDE8F08F744F0120E06305080F060608B8
:102DA0001F090608B603060859130608A0030120E8
:102DB0002DE9F74F074608460E463DF08BFF0446C7
:102DC00020B1012825D132782A2A22D1B24E0025FD
:102DD0004FF00D0BDFF8E092B24640F26228AF48A8
:102DE000FDF7E8FD0BFB05F3484601355AF80310E3
:102DF000FDF714FE221E3146384618BF01220D365B
:102E0000FEF7E0FBFDF7BEFD4545EBD103B0BDE8A5
:102E1000F08F3D21304640F05CFB002800F0368109
:102E200001460A4611F8014D202CFAD0921B0130C0
:102E3000814610F8011B2029FAD05FFA82FA4FF080
:102E40000008DFF854B20D235246304603FB08F168
:102E50000BEB01045BF801100091FCF719FA054631
:102E6000002857D1009908463DF034FF824551D1E2
:102E7000267906F0E001402900F0CB800ED8002929
:102E800056D0202900F09D8038468549FEF7A9FBE1
:102E9000204603B0BDE8F04FFDF70FBE602900F0FB
:102EA00091808029F0D148463DF014FFE379054632
:102EB000A679DB070CD52046FBF7FCFB037801461F
:102EC00033B12A46484640F02AFB002840F0D8801B
:102ED000002D00F0D580AE42C0F0D2800D232046F8
:102EE00003FB08B393F805A0FBF7E4FB324600218F
:102EF00040F0E8F9AA452CD82A466A49484640F0ED
:102F00000EFB30B32046FBF7D5FB2A46494640F07E
:102F100065F91EE008F1010840F26223984592D15C
:102F200032466149384603B0BDE8F04FFEF759BB61
:102F300006F00703042B1CD10B460A224846FCF777
:102F4000F7F9D4F80530014683429DD32046FBF7BC
:102F5000C7FB0D23554803FB08F85BF80810FDF785
:102F60005DFD00222146384603B0BDE8F04FFEF774
:102F700029BB052B0FD101230A224846FCF7D8F9BB
:102F8000D4F8053001468342FFF67EAF5B428342B0
:102F90003FF77AAFDAE74846FCF76EFAB4F8055027
:102FA000B4F8071016F0050FAAB28BB201D02AB2FE
:102FB0000BB29042FFF668AF98423FF765AF01460B
:102FC000C4E765793A4A002602EBC505B2463346A6
:102FD00095F8A8220092009AB24202D9BAF1000FE5
:102FE00003D0002B3FF450AFB3E7D5F8A41251F84B
:102FF000260060B149460193FCF726F9019B30B9E0
:103000004FF0010A31462046FBF76AFB5346013672
:10301000E1E706F007066379013E0093009BAB42AF
:1030200097DD4846814610F8013B202BFAD0204618
:10303000FBF740FB8246042E04D8DFE806F00310BD
:1030400010161F004846FCF717FA0AF80500484614
:103050002C2140F03EFA013500F10109DEE7484637
:10306000FCF70AFA2AF81500F1E700230A220021EA
:103070004846FCF75DF94AF82500E8E70123F5E743
:1030800032460C493846FEF7ACFAFDE63146384682
:1030900003B0BDE8F04FF3E5E06305082F0906082B
:1030A0007D090608CE2A0608B60306087209060836
:1030B000C4490508420906080F0606082DE9F04F25
:1030C000914689B00C461A46002180464D46FEF7CF
:1030D000E7FF00270646DFF8E0B0B9F1000F69D03E
:1030E00029460622204640F0C3F8002832464046D2
:1030F00013BF012100214FF0010A4FF0000AFEF733
:10310000CFFF0646287813F0E5F9079010B36879E9
:1031100013F0E0F9079B4FF461714FF0190C5B79E4
:10312000EA780793AB781CFB021295F801E01CFBD0
:103130000313297900B14079CDF804E0CDE90232DA
:10314000079B5A46CDE90410009351463B46404642
:10315000FDF74CFC207813F0BDF9079010B36079AF
:1031600013F0B8F9079B4FF461714FF0190C5B79BC
:10317000E2780793A3781CFB021294F801E01CFB91
:103180000313217900B14079CDF804E0CDE9023292
:10319000079B5A46CDE90410009351463B464046F2
:1031A000FDF7F4FB013706340635142F95D109B02D
:1031B000BDE8F08FCA46CDE78B0906082DE9F0413E
:1031C000064686B008460F46FFF7B6F8054638B102
:1031D00000235C4901201A4606B0BDE8F0416DE7C6
:1031E0000846FCF749F91328044600F3A280062696
:1031F0008DF81750544D4643781CFBF77FF907466E
:1032000070B1FCF739F9C0B213F078F940B1AB19DD
:10321000027983F8E8259DF8173001338DF81730CF
:103220003846FBF76BF9074668B1FCF725F90D281E
:1032300009D8062303FB045383F8E9059DF81730EA
:1032400001338DF81730DFF8FC80B11C0DF1170247
:1032500038464144FCF714F9FBF750F9074668B1CA
:10326000FCF70AF9012809D8062303FB045383F865
:10327000EC059DF8173001338DF817303846FBF711
:103280003DF980B1FCF7F8F8C0B213F037F950B14E
:103290000623027903FB045383F8ED259DF81730CC
:1032A00001338DF817309DF817200623042A2FD1FB
:1032B00003FB04530022A3F8EC2519F0EBFE0623D0
:1032C0004FF4617603FB045595F8E80513F002F915
:1032D00095F8EB2595F8EA751923804695F8ED05E4
:1032E00013FB076713FB026613F0F4F843792146DA
:1032F00098F80520039395F8EC3514480097CDE92C
:10330000016395F8E935FDF7C9FB06B0BDE8F0812A
:10331000052A05D103FB0453002283F8ED25CCE7F1
:10332000062ACAD0002308EB060248F8063093802C
:10333000C3E713232A460649304606B0BDE8F041EC
:10334000FEF7EEBF5C550120744F01208B09060883
:10335000A40906082DE9F04F174689B01A460C4615
:10336000002181463D46FEF79BFE3A4E07F16C0375
:103370008046DFF8E8B0079394F904100023364A3A
:1033800092F90800884260D001330C32092BF7D142
:103390000C35079B0C349D42EED109B0BDE8F08F8F
:1033A00029460C2220463FF063FF0028424648464B
:1033B00013BF012100214FF0010A4FF0000AFEF770
:1033C0006FFEEA7995F90430804606EB8202514699
:1033D0004846D2F8E02404922A7A06EB8202D2F818
:1033E000E0240392AA7906EB8202D2F8E02402924A
:1033F0006A7906EB8202D2F8E02401922A680092F0
:103400005A46FDF7F3FAE279514694F904304846FA
:1034100006EB8202D2F8E0240492227A06EB8202C2
:10342000D2F8E0240392A27906EB8202D2F8E024DB
:103430000292627906EB8202D2F8E02401922268BD
:1034400000925A46FDF7A2FAA2E7002FA8D1BA4689
:10345000D9E700BFC449050844540120AA09060859
:103460002DE9F04707468AB00846FEF765FF044697
:1034700038B10023544901201A460AB0BDE8F0478C
:1034800068E70DF11C0807904E1CC8E901000846CA
:10349000FBF7F2FF4C4B40B21A4693F904108142FD
:1034A00000F08A8001340C33092CF6D10024254623
:1034B0003046FBF723F8064638B1013500230A22CF
:1034C000EDB21946FBF734FF07904FF00009DFF823
:1034D00000A13046FBF712F8064640B3FBF7CCFFDD
:1034E0003A49002251F804CBD3B2604503D00132EF
:1034F000102AF7D100230AEB8302D2F8E02490428D
:1035000015D1B9F1020F1FD0B9F1030F21D05A1E06
:10351000B9F1010FD2B212D00B2A03D88DF82130A5
:103520000135EDB209F10109B9F1040FD1D1052D31
:1035300015D838460AB0BDE8F047FEF769B8042A46
:10354000F0D88DF82230EBE7052BEBD88DF824303E
:10355000E6E79A1E0D2AE5D88DF82330E0E798E8D3
:1035600007001B4B84E807009DF82320002103EB94
:1035700082020846D2F8E02404929DF8242003EB4E
:103580008202D2F8E02403929DF8222003EB82020B
:10359000D2F8E02402929DF8212003EB82030D4A29
:1035A000D3F8E0340193079B00939DF92030FDF799
:1035B000EDF90AB0BDE8F0870C2301258DF8200055
:1035C00003FB042474E700BF80530120A44E0508C8
:1035D000C4490508AA0906082DE9F04F8BB00C462E
:1035E0000021074608921A46FEF75AFD0026089D5C
:1035F0004FF019094FF46178DFF8A4B00990089BE7
:10360000002B49D029460A2220463FF031FE0028EF
:10361000099A384613BF012100214FF0010A4FF0EB
:10362000000AFEF73DFD2A8909903346069251466D
:10363000EA88384605922A790492EA780392AA78B1
:1036400019FB028202926A7819FB028201922A789F
:1036500000925A46FDF7CAF922893346013651468F
:1036600006923846E2880A35059222790492E27879
:103670000392A27819FB02820292627819FB0282FD
:10368000019214F80A2B00925A46FDF77FF91E2E7C
:10369000B5D10BB0BDE8F08FDDF820A0DCE700BFAE
:1036A000C70906082DE9F04380468BB008460F464F
:1036B000FEF742FE044638B10023654901201A4650
:1036C0000BB0BDE8F04387E70846FBF7D5FE1D28A1
:1036D000054600F3B3800A268DF827404643781C40
:1036E000FAF70CFF044630B1FBF7C6FE9DF8273011
:1036F00001338DF827302046564CFAF7FFFE074677
:1037000068B1FBF7B9FE0D2809D80A2303FB05436E
:1037100083F86C009DF8273001338DF82730DFF8EF
:103720003091711C0DF1270238464944FBF7A8FE81
:10373000FAF7E4FE074668B1FBF79EFE222809D897
:103740000A2303FB054383F86F009DF827300133FC
:103750008DF827303846FAF7D1FE074668B1FBF7F7
:103760008BFE0D2809D80A2303FB054383F870005C
:103770009DF8273001338DF827309DF82730062B30
:103780000CD0002309EB0602404649F8063053608E
:103790001381FDF73DFF0BB0BDE8F0830A2600233F
:1037A000384606FB0546A6F87230A6F87430FAF7DC
:1037B000A5FE074640B1FBF75FFE9DF82730A6F84F
:1037C000720001338DF827303846FAF797FE58B16A
:1037D000FBF752FE0A2303FB0543A3F874009DF890
:1037E000273001338DF827301B4B4FF0FF324FF459
:1037F00061705A600A2202FB0542B2F874300693E7
:10380000B2F87230059392F87030049392F86F30EA
:103810000393192392F86E1013FB0101029192F8A1
:103820006D1013FB010300210193084692F86C30E0
:103830000A4A00932B46FDF7A9F8ACE71D23224660
:10384000074940460BB0BDE8F043FEF769BD00BF35
:10385000D86001206C600120A0030120C709060880
:10386000A40906082DE9F04F804691461F460C46F4
:1038700016464FF0000BDFF820A12DED088B95B018
:1038800094ED008AB5EE408AF1EE10FA7DD0D4EDC9
:10389000019A94ED029AD4ED038AB9F1000F49D050
:1038A000D6ED00BA96ED01BAB4EE6B8AD6ED02AA57
:1038B00096ED03AAF1EE10FA6CD1F4EE4B9AF1EE0C
:1038C00010FA67D1B4EE6A9AF1EE10FA62D1F4EE12
:1038D0004A8AF1EE10FA0CBF012100213A460D464A
:1038E000404681F00101FEF7DBFBB0EE6B0A0746B4
:1038F00011A8FAF70FFEB0EE4B0A07900EA8FAF7E0
:1039000009FEB0EE6A0A06900BA8FAF703FEB0EEC5
:103910004A0A059008A8FAF7FDFD0599069A079B43
:1039200003904046029129460192524600935B461D
:10393000FDF75CF8B0EE480A11A8FAF7EBFDB0EE1F
:10394000690A05460EA8FAF7E5FDB0EE490A0690A9
:103950000BA8FAF7DFFDB0EE680A059008A8FAF7A1
:10396000D9FD069B059A00210390404602925246DB
:1039700010341036CDE900535B460BF1010BFDF717
:1039800005F8BBF1080F7FF47BAF15B0BDEC088BD9
:10399000BDE8F08F0021A1E7EA0906082DE9F74FFD
:1039A00007460D46DFF8A8A1DFF8A8B12846FEF7C4
:1039B000C3FC064638B100235D4901201A4603B016
:1039C000BDE8F04F4EE7052251462846FBF760FC64
:1039D000A0B9584B0022C3F89821C3F8A821C3F816
:1039E000B821C3F8C821C3F8D821C3F8E821C3F827
:1039F000F821C3F8082203B0BDE8F08F04224E4935
:103A00002846FBF745FC04462846002C44D1FAF72B
:103A100075FD80460028EED03DF05CF9474BC2B200
:103A200053F8049BB9F1000F07D12A4644493846A0
:103A300003B0BDE8F04FFDF7D4BD49464046013420
:103A4000CDE90023FBF724FC0646DDE9002300282E
:103A5000E6D1374A034600211546013342F8101BD0
:103A6000082BFAD10BEBC404D4F8BCC0BCF1000F96
:103A700003D094F8B8E0764505DB49463148324D2D
:103A8000FDF70CF892E70CEB061305EB0614013674
:103A90000FCB84E80F00EEE7FBF7EEFC07280446A7
:103AA0003DD82846FAF72AFD064658B3FAF704FB34
:103AB000204B012503EB041383ED660A3046FAF729
:103AC0001DFD064638B1FAF7F7FA1A4B013503EB3C
:103AD000041383ED670A3046FAF710FD064638B145
:103AE000FAF7EAFA134B013503EB041383ED680A86
:103AF0003046FAF703FD38B9384603B0BDE8F04F59
:103B0000FDF786BD0546D9E7FAF7D6FA0948032D31
:103B100000EB041484ED690A3FF44DAFECE7072392
:103B200032460A49384603B0BDE8F04FFEF7F8BB0D
:103B3000046201206C600120FE090608005005089F
:103B4000B6030608030A060859130608A40906085E
:103B5000C6060608C44905082DE9F74F92460C46EB
:103B60001A46002181465646FEF79AFA00258046FD
:103B7000DFF864B0BAF1000F2CD0314604222046A1
:103B80003FF076FB00284246484613BF0121002142
:103B900001270027FEF784FA738880465A4601936E
:103BA00039463AF82530484600932B46FCF71EFF6D
:103BB00063885A46394648460193043634F8043B34
:103BC00000932B460135FCF7E1FE042DD2D103B062
:103BD000BDE8F08F5746EBE70D0A06082DE9F341E3
:103BE00005460846FEF7A8FB0C46074638B10023F9
:103BF000334901201A4602B0BDE8F041ACE7314933
:103C00002046FBF721FB034668B92D4A4FF47A7032
:103C10004FF4FA610133108051800432042BF9D142
:103C200002B0BDE8F0812046FBF726FC03280646DB
:103C300041D82046FAF762FC074670B1FBF71CFC3E
:103C40004FF0010804463846FAF758FC48B92846B0
:103C500002B0BDE8F041FDF7DBBC40F2EE24804647
:103C6000F1E7FBF709FCB8F1000FF0D0A4F2EE2267
:103C700040F2DC539A4203D8A0F2EE229A420AD9CB
:103C800040F6CA0340F2EE220F49284602B0BDE8D2
:103C9000F041FEF745BB0D4B00210D4A03EB8603B7
:103CA000A3F81842A3F81A023346CDE900400846AB
:103CB000FCF76CFEB4E703233A460649E5E700BF8C
:103CC00084620120C60606081E0A06086C600120F0
:103CD0000D0A0608A60606082DE9F04F8FB08946A2
:103CE000174600211A4606460024FEF7D9F90DF1C1
:103CF000240B0546DFF86CA059F82430594602A879
:103D0000029335F0F9FE57B357F824303046029A43
:103D1000039393422A4613BF012100214FF001086B
:103D20004FF00008FEF7BCF904A9054603A835F0DA
:103D3000E3FE04A923465246009130464146FCF773
:103D400055FE23460134524641463046CDF800B078
:103D5000FCF71CFE202CCFD10FB0BDE8F08FB84689
:103D6000EFE700BF2C0A0608F0B5074689B0084601
:103D70000E46FEF7E1FA054638B100231949012045
:103D80001A4609B0BDE8F040A6E70846FBF774FB09
:103D90001F2804461DD83046FAF7B0FB01462046DE
:103DA0002BF090FE78B103AE0E48314600EB840054
:103DB00035F0A2FE23460C4A294628460096FCF719
:103DC000E5FD09B0F0BD384609B0BDE8F040FEF7AA
:103DD0000BBA1F232A460549384609B0BDE8F04012
:103DE000FEF79EBA946201202C0A0608A409060870
:103DF0002DE9F04F924685B00C461A4600218146C7
:103E00005546FEF74DF900268046DFF86CB0BAF152
:103E1000000F2FD02946042220463FF029FA00281F
:103E20004246484613BF0121002101270027FEF723
:103E300037F9EB7880465A4602933946AB784846C4
:103E400001932B8800933346FCF7D0FDE3785A4664
:103E50003946484602930435A378019334F8043B6D
:103E6000009333460136FCF791FD102ECFD105B0FB
:103E7000BDE8F08F5746E9E7360A0608F0B5074671
:103E800085B008460E46FEF757FA054638B10023BE
:103E90001C4901201A4605B0BDE8F040A8E70846D5
:103EA000FBF7EAFA0F28044623DC3046FAF726FB34
:103EB000014620462BF07EFDA8B104F12002124BF2
:103EC0002946284603EB820393F82B22029293F8AB
:103ED0002A220192B3F828320C4A00932346FCF7B9
:103EE00055FD05B0F0BD384605B0BDE8F040FEF721
:103EF0007BB90F232A460649384605B0BDE8F04095
:103F0000FEF70EBA146301206C600120360A060821
:103F1000A40906082DE9F04F87B014461A46054655
:103F200003910021FEF7BCF84FF000080646DFF8C9
:103F300020B106234FF0000903FB08F7C037039BAD
:103F4000DB5D0493002C7FD0E35D2846049A059343
:103F50009A42324613BF012100214FF0010A4FF06F
:103F6000000AFEF79DF8059B06465A46514628462C
:103F7000CDE900934346FCF739FD049B5A46514670
:103F800028460137CDE9009309F101094346FCF7C2
:103F9000FDFCB9F1060FD2D108F10108B8F1060F06
:103FA000C7D1E427DFF8A8B0039BA7F1E40913F811
:103FB00007A0002C4AD0E35D324628469A45049378
:103FC00013BF012100214FF001084FF00008FEF758
:103FD00067F8049B06465A4641462846CDE90093B9
:103FE0000623FCF703FD01370623194A41462846FC
:103FF000CDE9009AFCF7CAFCEF2FD5D1039B93F8CB
:10400000EF70ACB194F8EF8032462846474513BFB5
:104010000121002101240024FEF742F800230C4A6C
:104020002146009328460723CDF80480FCF7DEFCE8
:104030000023074A21462846009307230197FCF7EF
:10404000A5FC07B0BDE8F08FA24696E7A046CAE7F8
:10405000480A0608F0B5054687B008460B46FEF745
:104060006BF9044638B100231C4901201A4607B0F9
:10407000BDE8F0404EE703AE194F02AA18491846B2
:104080003FF0E2F8B8B1032C04D12846FDF7C0FA9E
:1040900007B0F0BDFBF7F0F902AA46F8040B394669
:1040A000002001343FF0D0F8ECE7324621460D48BD
:1040B000FCF7F4FCECE7032CE7D1059BDDE90346B4
:1040C0001A4601933146E0B22BF0BEFC019B00285A
:1040D000EBD12846FEF788F8DAE700BF94620120AA
:1040E000CD0A0608480A06082DE9F04F0F46164685
:1040F00089B04FF00009B8463446DFF83CB11A46A3
:1041000000210546FDF7CCFF0790002E7CD021460C
:104110000C2240463FF0ACF80028079A284613BF0F
:10412000012100214FF0010A4FF0000AFDF7B8FF0E
:1041300094F90B2007904B460492514694F90A20BB
:1041400028460392B4F908200292B4F9062001929D
:10415000B4F9042000925A46FCF748FC98F90B2069
:104160004B4609F1010951460492284698F90A2064
:104170000C3408F10C08039238F9042C029238F937
:10418000062C019238F9082C00925A46FCF7FEFBE7
:10419000B9F1080FB9D10024DFF8A0900C2303FB7C
:1041A00004FA9EB34FF00008012356F80A2003FAE0
:1041B00008FB57F80A3053403BEA030314BF0121C0
:1041C000002112EA0B0F08D023464A462846CDF8B4
:1041D00000800791FCF70AFC079957F80A301BEAA0
:1041E000030F06D023464A462846CDF80080FCF748
:1041F000CDFB08F10108B8F10E0FD5D10134082C20
:10420000CCD109B0BDE8F08FB246A7E7B046012394
:1042100057F80A2003FA08F3134207D023464A4608
:1042200001212846CDF80080FCF7B0FB08F1010819
:10423000B8F10E0FEBD1E1E75C0A0608740A060834
:10424000F0B506468BB008460D46FEF775F80446F5
:1042500020B300233F4901201A460BB0BDE8F040CF
:1042600042E72D2B03D0A3F13002092A4BD8052CAD
:1042700005DD30460BB0BDE8F040FDF7C9B9284672
:10428000FBF7FAF80AAB621C03EB440424F80C0CAD
:1042900015F8013F303B092BFAD914462B78002B37
:1042A000DFD1062CE5D1BDF81C20BDF91C30072A52
:1042B000DFD8BDF91E10A1F5FA7292B2B2F5FA6F0D
:1042C0001AD8BDF92040A4F5FA7292B2B2F5FA6F8D
:1042D00012D8BDF92270B9420EDCBC420CDBA142FF
:1042E0000ADCBDF924C00CF1640292B2C82A03D8DA
:1042F000BDF92650112D11DD174930460BB0BDE830
:10430000F040FDF76EB9202B02D101352246C4E7FB
:1043100030460BB0BDE8F040FDF766BF0C200F4AF9
:104320006DB200FB0322A2F81C13A2F81E43A2F8F0
:10433000207382F822C382F8235300910021084A97
:104340000846CDE903C5CDE90147FCF71FFB0BB0DB
:10435000F0BD00BF84630120890A06086C6001205B
:104360005C0A06082DE9F04F89468DB016460021FB
:104370001A4607460024FDF793FEDFF8DCA0054649
:10438000C4EBC40309EB030259F80300918840F31E
:10439000074892790890ADF824108DF82620B8F1DE
:1043A000000F53D0002E54D0F218F0589188937912
:1043B00007220A9008A8ADF82C100AA98DF82E3013
:1043C0003EF056FF00282A46384613BF012100213F
:1043D0004FF0010B4FF0000BFDF762FE9DF82E3001
:1043E00005465246069359469DF92D3038460593A9
:1043F0009DF92C3004939DF82B3003939DF92A30BE
:1044000002939DF8293001939DF8283000932346AC
:10441000FCF7ECFA9DF8263052465946384606938A
:104420009DF9253005939DF9243004939DF82330A0
:10443000CDE902839DF8213001939DF8203000934F
:1044400023460134FCF7A2FA102C99D10DB0BDE837
:10445000F08FB346DEE700BF9F0A06082DE9F04F54
:1044600006468DB00D469C4FDFF8A082DFF8A09283
:1044700028463CF02FFC034630B9024697490120FC
:104480000DB0BDE8F04F6DE7052239462846FAF732
:10449000FFFE0446C8B9924D0146702205F55E70D4
:1044A0003EF010FFC5F81843C5F82443C5F8304363
:1044B000C5F83C43C5F84843C5F85443C5F86043C4
:1044C000C5F86C430DB0BDE8F08F04224146284684
:1044D000FAF7DEFE044638BB2846FAF70FF88246A4
:1044E0000028EFD03CF0F6FBDFF828B202465BF87C
:1044F000041B39B92A467B4930460DB0BDE8F04F60
:10450000FDF76FB85046CDE90012FAF7C1FE019AE7
:1045100040B92046744D1DF031FA00994846FCF729
:10452000BDFAA5E70134E2E7072270492846FAF709
:10453000AFFE074600287AD1202128463EF0C9FF69
:10454000044670BB6A4D6B48FCF768FA214601349B
:104550002846FCF763FA0E2CF8D10024DFF8B89156
:10456000654FFCF70FFADFF8B4810C260025DFF861
:10457000B0A1214666434846FCF750FA0123F259A0
:104580005E48AB400135134214BF41465146FCF72B
:1045900045FA0E2DF2D10134FCF7F4F9082CE4D1E0
:1045A00090E704AC564D03AA55493EF04DFE002855
:1045B00048D0022F11D1049A072A07D805990D294E
:1045C00004D80378722B13D06E2B22D0082300223C
:1045D0004C493046FDF7A4FE74E7FAF74DFF03AAF5
:1045E00044F8040B2946002001373EF02DFEDEE79B
:1045F0000C203B4B00FB0233012000FA01F1D3F801
:1046000018030843C3F8180338493046FFF726FF5C
:1046100058E7334B0C2000FB0233012202FA01F170
:10462000D3F8182322EA0102C3F81823ECE728463E
:10463000002404AD324F03AA31493EF005FEA8B173
:10464000082C03D13046FCF7E3FF3BE7FAF714FFF1
:1046500003AA45F8040B3946002001343EF0F4FD6E
:10466000EDE729493046FCF7BCFF2BE7082CE9D1E0
:10467000049B0F2BF5D8DDF814E0BEF1070FF0D83E
:10468000DDF818C0BCF10D0FEBD8079F07F16402ED
:10469000C82AE6D8089DFF2DE3D809986428E0D8F9
:1046A0000A996429DDD88842DBDA0B9C032CD8D820
:1046B000C3EBC3020A4B134483F87D1383F878E3FA
:1046C000094983F879C383F87A7383F87B5383F8B5
:1046D0007C0383F87E4398E7C6060608E46301205E
:1046E0006C600120B603060859130608BC0A0608C8
:1046F000C40A0608F510060884630120C90A0608E2
:10470000CD0A0608CF0A0608890A0608FE09060827
:10471000030A060800500508A8FC0508870A0608D1
:10472000BE1306082DE9F04F89B000260C46002183
:1047300007921A460746B246FDF7B2FC4FF0190938
:10474000079D4FF46178DFF894B00690079B3BB368
:104750002946062220463EF08BFD0028069A384660
:1047600013BF012100214FF0010A4FF0000AFDF7AD
:1047700097FC6A790690334619FB02825146384607
:1047800005922A7919FB02820492EA780392AA78A8
:1047900002926A7801922A7800925A46FCF726F92A
:1047A000627933460136514619FB02823846063596
:1047B0000592227919FB02820492E2780392A27890
:1047C00002926278019214F8062B00925A46FCF786
:1047D000DDF80A2EBAD109B0BDE8F08FD50A060877
:1047E0002DE9F04F074689B008468B46FDF7A4FD3A
:1047F000044638B10023544901201A4609B0BDE8E7
:10480000F04F8FE7514B084693F808A793F80997A4
:1048100093F8F287FAF730FE0928054600F38B80FB
:1048200006268DF81F404A4C46430BF10100F9F76C
:1048300065FE834658B1FAF71FFE0D2807D8A31965
:1048400083F8E8039DF81F3001338DF81F30584678
:10485000F9F754FE834668B1FAF70EFE824509D394
:10486000062303FB054383F8E9039DF81F3001335A
:104870008DF81F305846F9F741FE824668B1FAF7C5
:10488000FBFD484509D8062303FB054383F8EA03EB
:104890009DF81F3001338DF81F305046F9F72EFE7A
:1048A000814668B1FAF7E8FD804509D3062303FB8A
:1048B000054383F8EB039DF81F3001338DF81F305B
:1048C000DFF88480311D0DF11F0248464144FAF79C
:1048D000D7FD9DF81F20062A0BD0002308EB060207
:1048E000384648F806309380FCF792FE09B0BDE8E0
:1048F000F08F02FB05424FF46170192392F8ED131B
:1049000013FB0101059192F8EC1313FB0103002145
:104910000493084692F8EB33039392F8EA33029338
:1049200092F8E933019392F8E8330A4A00932B4650
:10493000FCF72CF8DAE7092322460749384609B084
:10494000BDE8F04FFDF7ECBC54640120744F01202A
:104950006C600120D50A0608A40906082DE9F04F6D
:10496000144689B00F461A4600210646FDF798FB0B
:104970000546002C00F0D58022783B789A4202460A
:1049800030460DBF4FF001084FF000080121002113
:10499000FDF786FB23780546994A41463046FCF7E9
:1049A00025F83B784146964A3046FBF7EFFF002C4E
:1049B00000F0B980627830467B789A422A460DBF73
:1049C0004FF001084FF0000801210021FDF768FBBE
:1049D000637805468B4A41463046FCF707F87B78FA
:1049E0004146884A3046FBF7D1FF07F1CA0304F17C
:1049F000CA0B4FF0020904934FF0000A822305937B
:104A00003B78534500F39180002C00F0F28097F83A
:104A1000EA30304694F8EA209A422A460DBF4FF019
:104A200001084FF0000801210021FDF739FB94F83F
:104A3000EA300546744A41463046FBF7D7FF97F8FF
:104A4000EA304146704A304607F1EC09FBF79EFF19
:104A5000002C00F0D08004F1EC034A4604F1FC0184
:104A60004FF001089A4633F802CB32F8020B844526
:104A700018BF4FF000088B42F5D188F001012A469B
:104A80003046C9B2FDF70CFB082105465046FAF73F
:104A90004DFB5E4A034641463046FBF7A7FF97F8B9
:104AA000EA104846FAF742FB584A03464146304668
:104AB000FBF76CFF002C00F0A0804FF0FC094FF0DA
:104AC000010807EB090104EB0900FAF7BDFB09F146
:104AD0000409002818BF4FF00008B9F58E7FF0D107
:104AE00088F001012A463046C9B2FDF7D9FA0821FB
:104AF00004F1FC00F9F794FD454A0346414630466F
:104B0000FBF774FF97F8EA1007F1FC00F9F788FD4E
:104B10003F4A03464146304609B0BDE8F04FFBF737
:104B200035BFA0463DE7A04659E7059B3B440693A9
:104B3000002C5CD0059B0698234419460793FAF78E
:104B400083FB049B1A789BF800309A424CD1B0FA50
:104B500080F84FEA58184B4609F11002F85AE15A0A
:104B60000233884218BF4FF000089342F6D188F014
:104B700001012A463046C9B2FDF792FA627804EB89
:104B8000090105469BF81800FAF7A2FA02909BF873
:104B9000003041461F4A30460193079B00930AF1BB
:104BA0000103FBF723FF049B07EB09017A780AF165
:104BB000010A187E0BF1010B0793FAF789FA079B9C
:104BC0004146049A09F11009029030461B780132DF
:104BD0000193069B0492009353460E4AFBF7D6FEC0
:104BE000059B093305930BE74FF00008B3E7A04698
:104BF000D9E7A04623E7A04651E7A04682E700BFD9
:104C0000EE0A0608000B06082E0B0608460B0608DF
:104C10005D0B0608150B06082DE9F04F8FB0044612
:104C20000846B04902AA3EF00FFB064640B90346CB
:104C30000246AD494120FFF791FE0FB0BDE8F08F6D
:104C4000AA49FAF701FB074620BB02AAA5493EF094
:104C5000FBFAFAF711FC0828054606D908233A465C
:104C6000A3492046FDF75CFBE7E7A24C94F8083720
:104C7000834202DC84F80857DFE7064604F5E16763
:104C80003146384624F040FF013694F80837B342E5
:104C9000F6DCEFE798493046FAF7D6FA0546E0B970
:104CA00002AA90493EF0D0FAFAF7E6FB0828064639
:104CB00003D908232A469149D3E78E4C94F8093743
:104CC000834202DC84F80967B7E72846013531469C
:104CD00034F0EAFE082DF8D1F4E789493046FAF7B6
:104CE000B3FA074600BB02AA7E493EF0ADFA00289F
:104CF000A3D0FAF7C1FB0828054603D908233A4692
:104D00008049AEE77B4C94F8F237834209DD0146D7
:104D100004F5E16024F042FF294604F5E16024F047
:104D20004BFF84F8F25788E777493046FAF78CFA58
:104D3000054618BB06AE6F4BDFF8A8910146B0469A
:104D40001022304693F8F2773EF0BCFABD4202AA38
:104D500080F20E81494600203EF076FA10B93A46BC
:104D60006A490EE1FAF788FB013528F8020BEDE7F6
:104D7000674C96E80F0084E80F005EE7654930460F
:104D8000FAF762FA054600283BD15A4B0DF1180894
:104D9000074693F8F29746464F4502AA51494FF00D
:104DA000000080F2F2803EF04FFA014610B94A4608
:104DB0005949E6E0B2464FF0000B032230463EF080
:104DC000C2FB30463BF086FF584502D80137043617
:104DD000E2E79AF800000BF1010BFAF72FFA0AF854
:104DE000010BEEE74A464D49CBE0414620460135EE
:104DF000043408F10408032224F070FEAF42F4D119
:104E00001BE747493046FAF71FFA0546002840F0ED
:104E1000AC80384F02AA334997F808873EF014FA5D
:104E200000283FF40AAFFAF727FB461E01D4B0452D
:104E300003DC434601223B4913E72A4902AA00202A
:104E40003EF002FA014600283FF4F7AE4FF00008AA
:104E50000DF10C09082203A88DF81480CDE9038810
:104E60003EF071FB03A83BF035FF40451CD802AA79
:104E70001C4900203EF0E8F900283FF4DEAE90F82F
:104E800000A04FF0000897F80997DFF8A8B04D454B
:104E900002AA14494FF000007EDA3EF0D5F902462E
:104EA00058B94A4620496CE099F8000008F1010819
:104EB000FAF7C4F909F8010BD4E7002D40D11378B3
:104EC000303B092B3CD919490192FAF7BDF9019AF7
:104ED00090B310465946FAF7B7F9019A002838D02E
:104EE00013494EE0CD0A06087C560120740B0608D3
:104EF0007A0B0608744F0120850B06088E0B0608F6
:104F00009C0B0608A80B0608BA0B0608A90C060895
:104F100068570120E40B0608C90C0608F00B0608C8
:104F20000E0C0608130C0608E90C06083BFC0508E5
:104F3000260C06081F0C06084FF001084FF0FF353D
:104F400010460192FAF798FA0028019A03DA2149EB
:104F500017E0A846F2E70EAB03EB4503013523F853
:104F6000200C94E74A461C490BE032461B4908E0F6
:104F70001B4900203EF068F900283FF4F9AE3A469C
:104F800018492046FCF72DFB57E63EF05DF9002856
:104F90007FF428AF144C31E73EF056F90028E1D1F8
:104FA00006EBC600114C082203A982303744204486
:104FB00024F094FD5046FAF741F987F8D20704EB44
:104FC000061006A96A0002303EF008F987F8EA8761
:104FD00033E600BF5B0C0608700C0608930C06084D
:104FE000CD0A0608C60B0608785701207C5601201A
:104FF0002DE9F04F0F46914689B0002187EA090953
:105000009846139A06460025FDF74AF86FEA090309
:105010000446DFF880900693284606F0F9FC129BC0
:10502000184230D0069BDFF870B0034014BF4FF039
:10503000010A4FF0000A049310EA0703284614BF40
:105040004A465A460593079206F0F4FC4346079AEF
:105050005146039000903046FBF7C8FC049B224663
:105060003046B3FA83F14909FDF71AF8039B059A14
:105070000446009351464346002A14BF5A464A4606
:105080003046FBF783FC0135182DC5D109B0BDE8CA
:10509000F08F00BFF80906080E0D060837B5044664
:1050A000084601913BF016FE01990546024620464E
:1050B000FAF7EEF870B9625D1046FAF7A9F800B990
:1050C00032B901352C44204601340378202BFAD024
:1050D00003B030BD0020FBE70329F0B5054685B0DD
:1050E0000C46164614D80B4F3970FBF74BFC0A4997
:1050F0002846FDF765FD2246084901A8F9F78EFF0D
:1051000001AB324608212846FCF7F8FFFF233B702D
:1051100005B0F0BDA003012059130608F4080608E5
:105120000329F0B5054685B00C46164614D80B4F3A
:105130007970FBF727FC0A492846FDF771FD2246E6
:1051400008496846F9F76AFF6B463246102128463F
:10515000FCF7D4FFFF237B7005B0F0BDA003012056
:1051600059130608F008060810B5114B86B011490E
:1051700004460493104B11480393114B114A0293B8
:10518000114B0193114B0093114BFBF747FCFBF7BD
:10519000F9FB10491048FBF781FC3CB10F4A10495C
:1051A000104806B0BDE81040FBF778BC06B010BD53
:1051B000550D06081F0D06085A0D06082A0D06088B
:1051C000640D0608150D06086D0D0608790D060814
:1051D000834F01207F0D0608870D060850B705088C
:1051E00048B70508980D06080120BDE72DE9F04FE6
:1051F0003E4C87B00A4600210646FCF751FF059059
:105200003B4A2378608802EB8303D3F8F4A8F9F7CC
:105210003BFA8368C1680493364B93F86420002AF4
:105220004BD0DDF810800491002721796279049B2E
:1052300007FB012213F80290B8F1000F3FD018F8D5
:1052400002504D45059A304607F1010713BF012171
:1052500000214FF0010B4FF0000BFCF721FF0590F0
:105260007DB305F00F022D09534659464035029291
:105270003046214ACDE90075FBF7B8FBB9F1000FC4
:105280002AD009F00F024FEA1919534659460292E3
:1052900009F140023046CDE90072174AFBF776FB70
:1052A000A279012A38BF0122BA42BEDC0834134B6E
:1052B000A342A5D107B0BDE8F08F9046B4E74546BC
:1052C000BFE7B8F1000FD9D053460D4A59463046D2
:1052D0000097FBF78BFBD1E77306E1D45346084AEE
:1052E000594630460097FBF751FBD9E7A85105080E
:1052F000C4490508744F0120C50D0608B8520508B9
:10530000DB0D060838B50C4B0C4603EBC0050B480B
:1053100095F8E42703EB8203D3F8F418FBF77EFB40
:1053200095F8EA3733B1611C0548C9B2BDE8384089
:10533000FBF774BB38BD00BFC4490508F41006086C
:10534000A7FC050873B50E4611490546F9F77CFF21
:1053500018B93070012002B070BD2C78602C8CBF61
:10536000613C413C072C10D8013501230A2201A9D8
:105370002846F9F7DDFF019B9D4206D00F2804D88F
:10538000013440EA04143470E4E70020E3E700BF8E
:10539000D10E060802460846531C05D1044B1A6874
:1053A0001B790A600B7170470249F9F737BE00BFDD
:1053B000D10E0608A8FC050808B504460848FBF706
:1053C000D9FAFBF7BBFA074B186E06F001FE03F0A3
:1053D00077F8012C01D135F03FFF72B6F7F73CF8B2
:1053E000F40D0608744F012010B5044608460B461C
:1053F000FCF7A2FF28B9032208491846F9F748FF2D
:1054000028B90748FBF7DCFA0120FFF7D5FF204653
:105410000449BDE81040FCF7E4B800BF000E0608E0
:10542000040E0608DD0506082DE9F74F4FF0000BC6
:10543000064601AA08462E495D463DF005FF0127B4
:105440000446DFF8BC80DFF8BC90DFF8A4A01CBBEA
:10545000BBF1000F28D1274C002D44D02946264807
:10546000FBF71CFB94F864300BB901F045FAF9F72F
:105470009DF9002384F86D30FBF746FA15B12846F4
:10548000FCF719FE9FB13046FCF7D0FD78B1FBF771
:10549000ADF80020FFF790FFBBF1000F0AD02046C7
:1054A000F9F7EAFF85B2C5B93046FCF79DFE03B0B7
:1054B000BDE8F08F41462046F9F70EFF80B9494616
:1054C0002046F9F709FF0028EED05F4601AA5146B1
:1054D00000203DF0B9FE0446B9E74FF0000BF5E7B8
:1054E0004FF0010BF2E70548FBF76AFABFE700BF90
:1054F000CD0A0608744F01202F0E0608520E06082A
:10550000260E0608AE1106080948002408B5FBF768
:1055100057FAFBF713FA074B83F8A648C3F8A849D4
:1055200083F8AC491AF08EFC2046FFF745FF00BF18
:10553000680E06086C60012008B5FCF777FD50B1D5
:10554000054B01229A75FBF751F80448FBF738FA2E
:105550000020FFF731FF08BD744F01208F0E0608B1
:1055600010B50C4628B1C943013801F0010102F021
:105570001DFEE30702D472B6F6F76EFF10BD00BF42
:10558000224BB0F5FA6F1A680346A8BF4FF4FA63CE
:10559000B3F57A7FB8BF4FF47A73D20416D540F2D0
:1055A000DC52904215D040F2DB5207EE903A904226
:1055B000F8EE677A1FD8DFED166A9FED167A77EE60
:1055C000E67A9FED150AA7EE870A7047B0F57A7F55
:1055D00002D89FED120A704707EE903ADFED106A8D
:1055E0009FED107AF8EE677A9FED0F0A77EEE67A74
:1055F000A7EE870A7047DFED0D6A9FED0D7A77EE13
:10560000E67A9FED0C0AA7EE870A7047B454012092
:1056100000007A44D62000C000E082440000000070
:1056200000407A44661000400000404200A0BB44A5
:10563000D62000400000834410B584464FEA810E16
:10564000102312F4004F4FEA420214BF0E24072425
:10565000013B92B2CCF80040F444F2D100EB81124D
:105660008C010351122042F8213010BD10B5844640
:105670004FEA810E0424130B013C4FEA021203EBA4
:10568000430392B203F11803CCF80030F444F2D192
:1056900000EB01130A018450062043F8214010BD9D
:1056A000704700BF704700BF034B00EB400003EBA7
:1056B000C000407C704700BF3C0700202DE9FF4739
:1056C0001E46C368044689469246BDF83070DDF830
:1056D00034804BB3CBB20D2B24D81A4AD556BAF12D
:1056E000FF3F23D023683146174A3846CDE9005A98
:1056F000C04752465FFA89F12079F4F7B9FB0246B8
:1057000000B10288D3B2314638460393C2F3032373
:10571000120B02932368CDE900520C4AC04704B033
:10572000BDE8F0870025DAE74D1CD8E77B06F6D404
:1057300023683146064A3846C4460C9504B0BDE895
:10574000F04760472CB70508960E0608A30E06081A
:10575000C70E060800233E22437002708370C37098
:10576000704700BF704700BF00207047704700BF00
:105770000020704701207047704700BF704700BF8E
:10578000704700BF704700BF9FED010A704700BF20
:10579000000000000020704703681B691847094B90
:1057A000002230B593F9004001325D7804330119CD
:1057B000062ACD7213F8025C055513F8014C8C755E
:1057C000F0D130BDDC820508002383700370C37004
:1057D00043707047D0F8FC304BB1D0F88C31D0F822
:1057E00014211B685B689A4205D3D01A7047D0E930
:1057F00007239A42F9D2C0681044C01A704700BF0C
:10580000D0E9091291420ED38A1AD0F80011036927
:1058100081B1D0F88811013B096849680A44934274
:105820000BD9981A7047036919448A1AD0F80011E5
:105830000029EED1013B981A70470020704700BF45
:10584000D0F8003113B190F8A4017047D0E90903F2
:10585000181AB0FA80F04009704700BFD0F8FC2059
:10586000034610B472B1D0F81421C1685C69881A7B
:10587000013A205C08BF0A465DF8044BC0B2C3F889
:1058800014217047006A5C69411C205CDC68C0B26E
:10589000A14238BF0A465DF8044B1A62704700BF48
:1058A000D0F8A83103B11847704700BFF8B590F899
:1058B000BD31012B1CD0002A164619DD05460F46C6
:1058C0000269436AD41AA8693946B4421844A8BF89
:1058D00034462246361B3DF081FC686A2A6927441B
:1058E0000444002EB4FBF2F302FB13436B62E9DCC9
:1058F000F8BD00BF0023084901E0152B09D003EBD8
:105900004302013311F802C00A448445F5D1104620
:1059100070470020704700BF4822012008B3B1FA49
:1059200081F35B09E9B14FF0100C10B50E4C4FF04C
:10593000010E224604E001334E2B10D092F804C031
:10594000604502F11C02F6D10EF1010C71455FFABF
:105950008CFEF0D1C3EBC30304EB830010BD002029
:1059600010BD0020704700BF9C4005082DE9F041A4
:105970001E4688B0030990460E9F00F00F04403386
:1059800049B30793FFF7CAFFC2790546079B414613
:105990003046CDE90042144AB847C8B12868F4F748
:1059A00003FCA9796A7911F0020FDFF84CC04FEAC5
:1059B00092020E49ED7908BF61460132079B0094BF
:1059C000CDE90102CDE90315094A00213046B84767
:1059D00008B0BDE8F081074A41463046BC460E9407
:1059E00008B0BDE8F0416047D60E0608FAFC05088D
:1059F000E80E06080A0F06085913060870B5094C88
:105A0000236873B10546002606E099681A681E737C
:105A100021609047236823B15A681846AA1A002AC1
:105A2000F3DA70BDC077012070B5204C2378012BCC
:105A300000D070BD1E4B1B68002BFAD01D4D2B688B
:105A400028465B6898470028F3D01B4B1B4E1A680A
:105A5000338892889A4219D3194900222846096846
:105A60004968EA622A6803FB01F1D36898473388E2
:105A7000144A013352683380002ADAD011689388BF
:105A80004A69134218BF1B048B6170BD0D4B002285
:105A90005B682270002BCCD00B491A6809789B8870
:105AA000890748BF1B04936170BD00BF58280120BF
:105AB0004C1B0120501B012050280120562801209A
:105AC000482801208C1B0120981B01202DE9F04162
:105AD000154686B0884619466A1CBDF830600D9F91
:105AE00023D0030900F00F04174A30464033CDE9B4
:105AF00000450593B847A8B12A4698F80510D8F88C
:105B00000000F4F7FDF968B1028801783046059B82
:105B10000391C2F30321120B02910021CDE900424F
:105B20000A4AB84706B0BDE8F0817306FAD4030903
:105B300000F00F00064ABC460C904033304606B0D9
:105B4000BDE8F041604700BF1C0F06082E0F060895
:105B5000570F06082DE9F04F704D0A460021824686
:105B600005F1800B2DED028B8BB0FCF799FA814685
:105B700000266B4B1C78AB7AB34200F39180103552
:105B8000AB45F5D140F21620F8F77EFDD0E902537F
:105B90000CB12C461D460DF1100B002715220021DB
:105BA00058463DF08FFB2E78002E41D06978304664
:105BB000FFF7B4FE95F9023008EE100A5A1C029362
:105BC00053425341002C00F0A580002214F802C07B
:105BD000A018B44540F09A8090F90280029A42459C
:105BE00040F0928042788A4208BF0123012203F0EC
:105BF00001030BF807204A4683F001015046039346
:105C0000FCF74EFA039B81464CB1464A18EE101A37
:105C10003046CDE900A24246FFF758FF039B424AB7
:105C200018EE101A3046CDE900A2029AFFF74EFF97
:105C300001370335152FB6D16CB304F13F06394F48
:105C4000DFF8E4801BF8013B02930BBB2078F8B12E
:105C500094F9022001321BD06178FFF75FFE054600
:105C60004A4601215046FCF71BFA94F90220029B98
:105C7000294681462078CDE900A7FFF727FF207845
:105C8000029B4FF0FF322946CDE900A8FFF71EFF27
:105C90000334B442D6D10BB0BDEC028BBDE8F08F1B
:105CA000E888F8F7F1FCD0E902230CB114461A4653
:105CB000297A6B7A06FB013312F903800CB3E7569D
:105CC000B8454A4650460DBF01230023012100215B
:105CD0000293FCF7E5F9029B814644B1114A314633
:105CE0002846CDE900A23A46FFF7E8FC029B0E4A9F
:105CF000314628460136CDE900A24246FFF7DEFCD8
:105D000037E74FF0FF37DBE700236FE703323F2A27
:105D10007FF45CAF4FF0FF386DE700BFD003012088
:105D2000D84F0120ED0901088D0901082DE9F04F38
:105D300007468BB040F216200391F8F7A5FC039AB2
:105D4000044600213846FCF7ABF93F4A0646D4E941
:105D5000025314780CB12C461D461522002104A8CC
:105D60003DF0B0FA05F13F03039395F80090B9F1C7
:105D7000000F30D095F801A0002C63D022460023FC
:105D80001178494557D1283392F8018001226B449C
:105D900003F8182CD0453246384613BF01210021A4
:105DA0004FF0010B4FF0000BFCF77AF9064654B1A7
:105DB000B8F1000F07D0254B5A464146484600939C
:105DC0003B46FFF7D3FD224B5A46514648460093C7
:105DD0003B46FFF7CBFD0335039B9D42C5D13CB34A
:105DE000651C0DF110084034DFF86090DFF860A00A
:105DF00018F8013BCBB915F8013CB3B116B13046E8
:105E0000FAF7DEFD29783B4615F8010C0022CDF8A3
:105E100000900026FFF7AAFD002215F8010C3B4672
:105E20001146CDF800A0FFF7A1FD0335A542DFD153
:105E30000BB0BDE8F08F01330332152BA0D14FF02A
:105E40000008A7E7A046A5E7D84F0120ED09010803
:105E50008D09010810B501311446FFF75FFD28B91F
:105E6000064B1A681B792260237110BDC279204647
:105E70000349BDE81040F9F7D1B800BFD10E0608BC
:105E8000E30E060808B5294B1B68DB041ED5B5EEEA
:105E9000400AF1EE10FA26D0DFED257AB4EEE70ADB
:105EA000F1EE10FA1FD49FED237AB4EEC70AF1EE9B
:105EB00010FA2AD870EE677A9FED1F7A9FED1F0ABD
:105EC000A7EE870A3CF012FC80B208BDDFED187A1D
:105ED000B4EEE70AF1EE10FA0BDA9FED190A3CF086
:105EE00005FC80B208BD9FED170A3CF0FFFB80B2B5
:105EF00008BD70EE677A9FED147A9FED140AA7EE45
:105F0000870A3CF0F3FB80B208BDDFED117ADFEDCC
:105F1000116A70EE677A9FED107AA7EEA67AB0EE5E
:105F2000470A3CF0E3FB80B208BD00BFB454012037
:105F30000000404200E0824466BEFFBE0060BB44F9
:105F400000007A440080BB4438DFFF3E00407A44C2
:105F50000000834466BEFF3E00A0BB446D4B1B782F
:105F60002DE9F04F87B0002B00F0CE806A4D4FF046
:105F700000086A48A968FAF791FD69686848FAF765
:105F80008DFD684B6848DFF8D8A1D3E90031C91A04
:105F9000664B1A68B1FBF2F2FAF780FDFAF7F2FCF1
:105FA0006348FAF707FD6348FAF704FD624B5FFAAE
:105FB00088F41B78A34221D8604C0025604FFAF783
:105FC000E1FC2646013556F8041B3846FAF726FD53
:105FD000162DF7D101255A4EFAF7D4FC23466168F5
:105FE000013530461B680434C91AFAF717FD162D1F
:105FF000F4D107B0BDE8F04FFAF7C4BC514B1426FA
:106000004FF03C0B671C03EB840306FB045693ED37
:10601000000A3CF06BFB96F81EE081B2B6F80E90D9
:106020001EF0010F80B214BF52222D221EF0020F6B
:106030000490504614BF54232D231EF0040F07EE86
:10604000903A14BF56232D231EF0080F009317EE2D
:10605000903A14BF4FF0430C4FF02D0C1EF0800F00
:10606000CDF804C014BF4FF0530E4FF02D0EB1FB0E
:10607000FBF10591642101FB09F1CDE902E139460B
:10608000FAF7CCFCB37FDB073AD55C232E4A634397
:10609000D118D05891ED010A70B1B8EE400ADFED89
:1060A0002B7A20EE270A07EE900AF8EE677A80EE48
:1060B000270A3CF01BFB00B2642290FBF2F102FBCA
:1060C00011022348FAF7AAFC1421224808F101081A
:1060D00001FB075701FB0454F988628A0491218B64
:1060E00002F0030392080391E18A0291A18B0191CE
:1060F000A18A009119214B43218AFAF7CFFC55E779
:106100001548FAF737FCDFE7144807B0BDE8F04F51
:10611000FAF750BCC8010020FC0C00206B0F0608E9
:106120007B0F0608D4160020920F0608641C01207D
:10613000BF0F06081B1006081C250020A80D002014
:10614000CB10060844560020040E002000401C46D8
:1061500094100608A9100608A0100608CF1006081B
:10616000771006082DE9F84F06460C461E4D3A27D3
:106170004FF00008DFF87890DFF878A02046FCF7B1
:10618000DBF8D5F800B048B921465846F9F7A4F82D
:1061900020B921466868F9F79FF880B15846FAF7A8
:1061A000E9FB696811B15046FAF738FCA96811B1EA
:1061B0004846FAF733FC4FF00108FAF7E3FB013FDA
:1061C00005F11005DAD12046FCF7B6F848B9B8F168
:1061D000000F06D1224630460449BDE8F84FFBF7D0
:1061E00000BABDE8F88F00BFF4820508F710060872
:1061F000F1100608EB10060870B504680546236A1E
:106200001B6943B1236AD0F894001B6998470128A1
:106210002AD002280DD0236ADA699AB9586958B38E
:1062200099692162BDE87040C3E905223DF00CBACE
:106230002362236ADA691433002AF9D1236ADA69FE
:10624000002AEBD0216A143394F824200E7B2362B9
:10625000F6B2DAB996B92846F3F762FD284601216D
:10626000BDE87040F3F7DCBC236A01462846143BC6
:106270002362F3F7D5FCCEE7206270BDAB68002B3C
:10628000E9D09A88196812048A61E4E70021284657
:10629000F3F7C6FC002384F82430002EDBD0EDE7B2
:1062A00038B58569002D3DD02C68236A1B7B5BBB0C
:1062B00020463AF081FC236A5B680BB3236A5A6874
:1062C000236A22F01F025B68216A886803F01F01BD
:1062D00000F11F03194421F01F01BFF34F8F002964
:1062E0000ADD02F1200311440F488B42C0F85C2202
:1062F0001A4603F12003F8D1BFF34F8FBFF36F8F1E
:106300002846BDE8384077E7AB68002BD0D01A6844
:1063100020469B8893613AF04FFC236A5B68002B10
:10632000CCD1EDE738BD00BF00ED00E038B58469A1
:1063300004B938BD256828463AF03EFC2B6A1B7B21
:106340001BB92046BDE8384056E7A368002BF8D0BB
:106350001A6820469B889361BDE838404CE700BF2F
:106360008160F5F7FBBB00BF0171F5F7F7BB00BF1C
:1063700038B5D0F8A83104460D460BB19847B8B1EE
:10638000636AA269D554636A21690133D4F8002194
:106390008B4228BF0023636222B12046BDE838400B
:1063A000F5F78EBDD4F82021136843F08003136005
:1063B00038BD00BF90F8BD21012A0AD0D0F80021D5
:1063C0000AB1F5F77DBDD0F82021136843F08003B2
:1063D000136070472DE9F84FAD4C80462379DB07F9
:1063E0002DED028B6BD5AB4B6579AB4E1F88012D24
:1063F00056D0022D35D0002D3ED094ED068AF37B89
:1064000033B1B38923B1A54B1B78002B40F0CB806F
:10641000A279337A632B06D8022D00F0DD80217C2F
:10642000002940F0ED8095429D4BB0EE487ADFEDBB
:106430009D6A38BF1546B27B1D70D4E90A31E3620C
:106440005B1A07FB03F307EE903AF8EEE77AA7EE44
:10645000A67A84ED067A002A5FD1BDEC028BBDE8F6
:10646000F88F6389BB42C8D28F4B012594ED068A11
:106470001B686571E361C2E7A389BB4219D38A4BEC
:10648000E1691A68F37D521A03EB830303EB83037C
:10649000B2EB830FB1DB012594ED068A6571AEE79F
:1064A000E389BB4280F086802389BB4201D200256C
:1064B00065717D4B94ED068A1B68E3619FE7657902
:1064C000DFF8D091EB1E012B32D9B9F80800C0F3E8
:1064D0000B003BF02BF9092840F3A7806E4EB9F86A
:1064E0000070F3889F4203D33288BA42BFF47FAF73
:1064F000B7EB430F3FF77BAF0323DFED6C7A674ABF
:106500006371B0EE678AA3710023C4ED067A13703D
:1065100023816381A381E3817EE0012D7ED0022D62
:106520009BD10720BDEC028BBDE8F84F05F0D2BD32
:10653000594EB9F80070F3889F4202D33288BA42AC
:1065400002D2B7EB430F63DDB9F80800C0F30B00CC
:106550003BF0ECF8092873DD0022357D6271A271F1
:10656000002D70D04D4B1D702B46154699B2B28848
:10657000738812FB01F213FB01F3717C92B29BB2A0
:106580008A422281638140F2B980521A92B28B42D0
:10659000A28140F2B1805B1A9BB2E38164236374F1
:1065A0000023636123E712F031FF002841D102226A
:1065B000A2712EE73C4BE1691A68337E521A03EB55
:1065C000830303EB8303B2EB830FFFF616AF0225C1
:1065D00094ED068A657112E7207C88B90121C4F820
:1065E000148080462174C3F16403314908FB03F32E
:1065F00081FB0301DB17A3EBA1536433637412E740
:1066000060692C49A8EB00088845ECDB63740AE755
:10661000032D7AD194ED068A0325F0E6BDEC028BBA
:106620000820BDE8F84F05F055BDB9F800701A4EC6
:10663000DDE6337C83422CBF01220022A271E8E612
:10664000032DE7D0D9E632881B4BDFF850A01B683A
:10665000B7FBF2F2013293F96C10082A28BF082226
:10666000D3B28AF80030002980D091423FF47EAF47
:10667000124991F800E00EF1010101F003018E458D
:106680003FF474AF4FF0FF3C4FF0A40B22E000BF8B
:10669000C0770120F05F0120B8540120EF5F012096
:1066A000EE5F0120ACC52737841B012000000000ED
:1066B0006BCA5F6B80969800745301207C4F012059
:1066C00018B93CEA2C0C28BF8C46013101F00301BB
:1066D0008E4515D012480BFB010090F96C008242E8
:1066E000EED18C465FFA8CF0F9F7E2FD9AF80030B3
:1066F000B9F80070657939E700234EE7002246E7D4
:10670000BCF1FF3F3FF432AFECE7B9F80800C0F34B
:106710000B003BF00BF809283FF7E1AE6DE600BF38
:10672000B45001202DE9F047694CA36820469847F2
:10673000002869D0B4F90E3004F14805A17D06EEB9
:10674000903AB4F91030092907EE103AB4F9123032
:10675000F8EEE66A07EE903AB8EEC77A4FF001031A
:10676000F8EEE77AC4ED126A84F8543084ED137AB7
:10677000C4ED147A4AD0574F28461CF07DFABB8DE1
:10678000002B4CD1544B1B685B0770D4BB6AD4ED13
:10679000127AB3F90220D4ED135A06EE102AB3F997
:1067A0000420B3F9003007EE102AB8EEC66A00EEF6
:1067B000103AD4ED146AB8EEC77A484DB8EEC00A64
:1067C0003B8835EEC66A464E36EEC77A05F10808B4
:1067D00037EEC00A84ED136A84ED147A84ED120A50
:1067E00053B9A84506F10C0605ED010A0CD03B880B
:1067F000B5EC010A002BF4D030460C363CF018FF03
:10680000A84505ED010AF2D1BDE8F087314F04F14A
:10681000200128461CF0F4F9BB8D002BB2D0D7F82C
:1068200028C02846DFED2F6A00252F49ACF102026F
:106830000CF10406B3F5C87F1CD0D1ED007AB8EE98
:10684000E77AD0ED007AE0EC016A77EE877AFDEE28
:10685000E77AE1EC017A22F8025FB242EAD1012B39
:106860000CD0013BBB851C4B1B685B078ED533F0FE
:1068700033F88BE7B0EE667A0D60E2E71B48DFF88D
:1068800074E0816BB4F80C80C831194E8EFB01A9FD
:10689000C917D0E90C20C1EBE911C832C830A1EB0F
:1068A0000801ACF804108EFB0281D217C2EBE11292
:1068B000ACF800208EFB002EC017C0EBEE10ACF839
:1068C0000200B581F5817381F9F7C6FEBB8DC8E77B
:1068D000AC26002078260020B4540120F8260020A1
:1068E0007C26002000000000F0770120C077012006
:1068F000085501201F85EB5138B5074C074DAC42B8
:1069000003D3074B01221A7038BDA288D4E90210C4
:106910003CF064FC1C34F2E7B08206088C8B06085D
:10692000D84F01202DE9F04F0C4695B0054634496B
:1069300020461746FEF7B2FB064600284FD13149E4
:106940002046FEF7ABFB064600284AD12E492046DA
:10695000FEF7A4FB0646002845D12C492046FEF749
:106960009DFB0646002840D120462949FEF796FBAC
:106970000028064612BF0824264601240FB144F021
:10698000100424493046FEF789FB80B344F020040C
:10699000214B1B780BB9FFF7AFFFF7F707FF14F098
:1069A000090F00F047831D48FAF70AF80020FEF7A8
:1069B000DBFB14F4807306933CD11948FAF700F816
:1069C0001848F9F7F7FF04F01803182B05D11648FB
:1069D000F9F7F6FF1548F9F7EDFF01232BE0012445
:1069E000CCE70224CAE70424C8E78124C6E710499B
:1069F0003046FEF753FB0028CAD044F48074C7E742
:106A00002A11060831110608391106083F11060837
:106A100048110608490E0608D84F012051110608F2
:106A200059110608711106087D110608A5110608FE
:106A30004C11060800230593F9F7A4FFBC4904F0A4
:106A40001008BC48FAF72AF8BB49BC48FAF726F800
:106A500004F48473082B07D1B9492846FAF7F4F8EF
:106A6000B7492846FAF7E8FE14F0800308930CD1E2
:106A7000B44B204613F83C2F002AB34A06BF01212D
:106A800013460021B14AF9F781FFB1492046FEF7CC
:106A9000ADFBB0492046FFF749F9AF492046FFF763
:106AA00059F8AE4BD3F800B0AD4B1B680493B8F166
:106AB000000F40F0FD814646AA48F9F781FFAA4B36
:106AC0004FF00009DFF864A307930393049B6BEA7C
:106AD00003030A93039B53F8047B0393002F40F0B6
:106AE000E981049BDFF848A363EA0B030993079B42
:106AF00053F8042B03920793002A40F005829B4B26
:106B000020469B4A9B49FCF725FC089B002B40F044
:106B1000A382DFF820A32046DFF81CB39AF80020F8
:106B20009BF80030DFF814939A42934A13BF012177
:106B3000002101270027FBF7B3FA9BF80030394604
:106B40000646013B8D4A204659F82330F9F74EFF9F
:106B50009AF8003039468A4F013B884A204659F856
:106B60002330F9F713FFD7ED007A864A2046F5EE79
:106B7000407AF1EE10FA0CBF01210021F9F706FF6F
:106B800033463A4680492046FCF76CFE7F4B804AEC
:106B900020468049FDF7A8FAB8F1000F05D07E4BDA
:106BA00093F90230002B00F0DF817C48F9F708FFF1
:106BB0007B48F9F7FFFE0023774A20467949FDF725
:106BC000D1FB794B6FF07F42784F794E204601938D
:106BD00000923A683168FEF70BFA40F20222754BD8
:106BE000204600920193BA68B168FEF701FAB8F145
:106BF000000F40F0BB817048F9F7E2FE42466F4853
:106C000008266F490127DFF838C210F8013B11F858
:106C1000019B03F1500EEE440EF8209C1CF801EB92
:106C20000EF1500AEA440AF8109C2FB1A3EB0E0EA5
:106C3000DEF1000747EB0E07013EE6D187F00101C8
:106C400020468DF83860FBF72BFA10AB5D4A3946C9
:106C500020468DF84860F9F7C9FE0CAB594A394611
:106C60002046F9F793FE584B584A20465849FDF7FD
:106C700033F8584B584A20465849FDF7B9F8584B55
:106C8000524A20465249FDF745F9564B564A20468E
:106C90005649FCF713FA564B564A20465649FCF71C
:106CA0009BFC564B564A20465649FCF755FF564B1F
:106CB000564A20465649FDF751FE564B564A204645
:106CC0005649FDF72FFDB8F1000F40F051815448AF
:106CD000F9F776FE534F4FF0000BDFF8688141461D
:106CE000022238463CF0C4FA002897F800A020465B
:106CF00014BF01210021039A0CBF4FF001094FF08E
:106D00000009FBF7CDF9BAF1020F039040F033818F
:106D100098F801204FF0190A40F2EE234946204628
:106D20001AFB0232404B019298F800208CE000BF21
:106D3000B511060808030608C3110608260306084D
:106D400059130608C0770120CE2A0608C811060884
:106D5000D5110608DF110608CFFE050810760120C0
:106D6000B05401200B110608844F0508FC110608D9
:106D700080530120BC710120191106080312060876
:106D8000046201200C1206084C740120CF0A060888
:106D900084630120946A0120E46301201311060832
:106DA0001B120608206A012028120608F05501204F
:106DB000987601202F1206081F1106085073012033
:106DC00014FC050869060608E00306089462012021
:106DD000F86A01203B12060814630120786B012039
:106DE00036120608411206085C550120F86D012094
:106DF00045120608D8600120006C01204E120608DA
:106E000084620120EC6B0120561206087C5601209A
:106E1000307201205F1206085464012010750120B1
:106E200023110608306D012024CC0508E511060861
:106E3000F111060840770120785301200050050821
:106E400018550120906001209A5C5B460092864AAA
:106E5000F9F7CCFD7A7840F2EE21844B20461AFBFC
:106E60000212494601923A789A5C5B4600927E4A49
:106E7000F9F78CFD0BF1010B023708F10208BBF1A9
:106E8000120F7FF42CAF7A4B224600212846FBF7E5
:106E900035F9230700F18580764E22462846317861
:106EA000FEF71AF9224671782846FEF739F9B7E05D
:106EB000714E04E63B7823B301230A9A204603FA75
:106EC00009F31A400B930CBF0121002109923246AD
:106ED000FBF7E6F8049B0646204663EA0B020B9B91
:106EE0001A423B46524614BF01210021F9F77EFDAC
:106EF00009993B4652460039204618BF0121F9F74F
:106F000045FD09F10109E5E5039B1B7853B34FF0FB
:106F10000109049B09FA07F913EA090F0BD06BEA80
:106F200003035246204613EA090F039B14BF0121B5
:106F30000021F9F75BFD1BEA090F13D0099B3246CC
:106F4000204613EA09090CBF01210021FBF7A8F82C
:106F5000B9F100010646039B524618BF01212046A5
:106F6000F9F714FD0137C2E5444B25E6444A46E6ED
:106F7000444B0393AEE698F8002049463B4B20462D
:106F80009A5C5B460092404AF9F730FD3A78374BFD
:106F9000494620469A5C5B4600923B4AF9F7F6FC6C
:106FA00068E70027F9B2013722462846FEF794F831
:106FB000042FF7D12F4FDFF8F4803B7888F80030AA
:106FC000069B33B93148F9F7FBFC31492846FBF7FA
:106FD000F7FDFF2388F80030F1B20136224628463B
:106FE000FEF79EF8042EF7D17B782A4C2370069B7F
:106FF000A3B92948F9F7E4FC25492846FBF710FE18
:107000002648F9F7DDFC2648F9F7B4FCFF23237086
:10701000002015B0BDE8F04FFBF74DB8FF232370FB
:10702000059B002BF4D01F48F9F7CAFC1E48F9F75E
:10703000C1FCEDE7A10706D50E4B2246284619787C
:10704000FEF74AF8E4E76207E2D50A4B22462846F3
:107050005978FEF765F8DBE7054B224618212846EC
:10706000FBF74CF8DCE700BF8906060824CC0508CE
:107070002A110608887701200B110608131106084B
:107080001F11060823110608990606086312060850
:1070900059130608A103012086120608AD1206083E
:1070A000B0110608C0120608D6120608A003012077
:1070B000002237E4012235E4224B30B583B09A79BF
:1070C00001906AB393F82630DFED1F6A07EE903A1D
:1070D0001E4B1F4CF8EEE77A1D7886EEA77A84EDFA
:1070E000187ADDB11B4BDDED017AB3F86A30F8EEAA
:1070F000670ADFED197A00EE103A60EEA70AB8EEE3
:10710000400AF7F797FB04F12003002103EBC502C7
:107110001960083303ED010A9A42F9D103B030BD7A
:107120000E4A12681201F9D593F82630DFED066A8F
:1071300007EE903A064BF8EEE77A86EEA77A83EDF3
:10714000187AEBE768240120555555401C2500208E
:1071500044560020C0770120BD378635B454012045
:10716000A54B1B78002B00F0B2802DE9F04FA34D0A
:1071700083B095F80491B9F1010F02D003B0BDE8D6
:10718000F08F9F4B9F4C1B6893F83470002F6ED08C
:107190009D4B0022DFED9D6AA64694ED187A90463D
:1071A00093F800B040F6FF7A67EE266A9FED986A82
:1071B0002B46984E019200941CE000F47061B1F5EA
:1071C000006F00F0B38000F29380B1F5806F00F0A3
:1071D000DB80B1F5C06F7BD1C0B24CF0080C988257
:1071E00083F81EC0013214330EF1040E0236D2B2FF
:1071F000BA422AD093F81EC09889BCF1010FDCD1A5
:10720000504500F0D080C0F30801400A01FA00F0B8
:1072100081B2002900F0BF807F4C80B2BBF12D0FFE
:1072200004EB5101B1FBF0F000F0D7804FF6FF7195
:107230008842D7D007EE900A0199F8EEE77A014428
:1072400080B2019167EEA67AB3E0009CB8F1000F1E
:107250000DD0DDED017AB8EE677A07EE908AF8EE90
:10726000677A27EE267AC7EE276AC4ED196ADFF837
:10727000B4A16A4A9AF80030A26613B3684E002798
:10728000DFF8788106F14C09B8F80E30304694EDFD
:10729000180A013707EE903A08F114080836F8EE9C
:1072A000E77A27EE800A3CF0BFF99AF80030D4ED77
:1072B0001A7ABB42A9EC010A87FEC00A84ED1A0AB9
:1072C000E2DC022385F8043103B0BDE8F08F70479B
:1072D000B1F5007F31D14CF0020CC1B283F81EC071
:1072E00093F81FC019828C45BFF47CAFD87779E73B
:1072F000B1F5406F13D0B1F5606F06D1C0B26CF03C
:107300007F0C988383F81EC06CE7B1F5206F14D111
:10731000C0B24CF0200C188383F81EC062E7C0B2E4
:107320004CF0400C588383F81EC05BE7C0B24CF0B1
:10733000100CD88283F81EC054E7504546D0C0F3E5
:107340000801400A01FA00F081B221B3324C80B248
:10735000BBF12D0F04EB5101B1FBF0F049D04FF61A
:10736000FF7188423FF43EAF07EE900A0199F8EEB4
:10737000E77A014480B2019167EEA67A4CF0010CE5
:10738000D88183F81EC017E0C0B24CF0040C5882BC
:1073900083F81EC026E7BBF12D0F7FF423AF4FF01B
:1073A000FF3131801EE7BBF12D0FF0EE467A08D099
:1073B0000020D88183F81E9008F10108CEED007AF4
:1073C00010E74FF0000100203180F2E7BBF12D0FF4
:1073D000F0EE467A08D00020D0E74FF6FF713080FB
:1073E00088423FF4FFAE25E74FF0000100203180D6
:1073F000C4E73080B3E700BFC8010020FC0C0020C8
:10740000BC27002044560020E51B012000007042EC
:1074100000000000E81B0120C0270900FFFF7F7F5C
:10742000645600201C25002070B41A4C1A4BA4FB93
:1074300002425209A3FB0243DB0803EB8303A2EBE6
:10744000430390F858205FFA83FC62451ED09A00EF
:10745000046800EB830346689D68641B04601D6B31
:10746000751B456000259D601D6380F858C083181A
:10747000013404609A6801329A6029B94268013285
:1074800042601A6B01321A6370BC704704689A003C
:10749000EDE700BF1F85EB51CDCCCCCC10B5437BC5
:1074A00004468268581C6073D154627B237B9342EC
:1074B00000D802B910BD2368D4E901019847002320
:1074C000637310BD427B42B1036810B50446D0E936
:1074D000010198470023637310BD7047084B0246B3
:1074E00002201968B2EB910F4FEA910307D25B08B3
:1074F00040009A4280B202D2FF28F8D97047704704
:10750000DC1B01200139032930D81E4B01EB810C13
:10751000024610B403F16C0403EBCC0304EBCC047F
:107520004FF0010C046003F16C0480F888C093F8FC
:107530006C0002281CD0C9B21348C1EB011150F8ED
:107540003110196771B10221604683F86C104FF455
:107550008071A18102F110014C325DF8044BC3E946
:107560002112704700205DF8044B704700207047DF
:1075700093F8792060465DF8044B624483F87920E3
:10758000704700BFC077012088220120954B2DE96C
:10759000F04FDFF864B285B04FF001094FF0000AF8
:1075A0001D469BF80030022B0CD00AF1010A09F1AC
:1075B00001090BF1280B0535BAF1040FF1D105B023
:1075C000BDE8F08F95F90320511C00F0E680D2B29F
:1075D00001924FF00C0C4FF008085FFA8AF1AE46AA
:1075E000012A50B225D800247F4D1CFB008723467A
:1075F00034B10133172B1CD015F81C4F002CF8D1D7
:107600006E788E42F5D1EE59002EF2D0774D6F682C
:1076100001342435BE4214D0102CF8D1734B13F82A
:10762000083C33B9714B4FF0140003F8079C03F882
:10763000080C0132019BD2B29A42D1D9754600247E
:1076400029E0E4B2694D671E07EBC70605EB860625
:10765000357F039506F11C050295039D002DE8D1A9
:10766000C3EBC303029A00EB400075469B009646AD
:107670005D4A07F0070703EB800386F81D9020465C
:1076800037721344CBF81060DB68F36014238EF874
:107690000030F2F743FD95F904104B1C00F0968082
:1076A000C9B201914FF008085FFA8AF301294FFA35
:1076B00081FC20D80C224C4812FB0C86002201329F
:1076C000172A18D010F81C7F012FF8D147789F4255
:1076D000F5D18759002FF2D0BE460026434F786877
:1076E00001362437864526D0102EF8D13F4A12F8AD
:1076F000082C002A6ED00131019AC9B29142D5D925
:10770000002C46D02423394A601E002603FB0020AB
:10771000CBF81460CBF81000F2F75CFA5846F2F799
:107720002DFA3346324620463149F2F70BFD01234C
:107730008BF80C3039E7F0B22C4F00F1FF3E03908C
:107740000EEBCE0007EB800000F11C06077F0296CF
:10775000002FD0D103466046039E0EF0070E9C46D4
:10776000C2EBC20300EB40001F4A9B008CF808E00C
:107770008CF81D9003EB80033046CBF814C0134403
:10778000029ADB68CCF80C3013231370F2F7C6FCB6
:107790003CB90023CBE9043307E70123002201931E
:1077A00017E7DBF81400F2F715FADBF81000F2F730
:1077B00011FA5846F2F7E2F93B463A4630460D498F
:1077C000F2F7C0FC01238BF80C30EEE60123002118
:1077D000019367E7054A4FF0130002F8079C02F88F
:1077E000080C88E7F8640120A03B05088000012010
:1077F0002D630108A16201082C78012030B40568CE
:10780000EFF3118C102383F3128803681B6AEBB12A
:107810008B6804460A461BB1D3691432002BFBD196
:107820002B6A6BB1986838B9934209D0186828B1AF
:107830005B6898680028F7D01433F3E7C3E9004188
:107840005FFA8CFC8CF3118830BC70475FFA8CFCBB
:1078500029628CF3118830BC3BF0F6BE30B593B092
:10786000002304468DF807100DF106018DF806205F
:107870000DF1070501228DF8183003958DF82C20A5
:107880008DF840201193CDE9073103A9CDE90432E9
:10789000CDE90932CDE90C33CDE90E33FFF7AEFF68
:1078A0002268136A002BFCD113B030BD2DE9F04FD4
:1078B000066887B03578012D0AD0022D03D1336ACE
:1078C000002B00F097800024204607B0BDE8F08F21
:1078D00096F9046014460279032E8DF81740D4BF40
:1078E00000240124B6F1FF3F08BF44F00104002C3E
:1078F000E9D1DFF810A206EB46038C464FEA4609B1
:107900000AEB431359690029DED093F8550020286B
:1079100040F0848093F8540001287FD0DFF8E8819C
:1079200083F85450D8F8007004E0D8F80030DB1B1E
:10793000192B63D88D6915F40045F6D1B144530075
:1079400062464FF0210C4FEA4919029340230097F9
:107950000AEB090009F1140B0DF117014FEA460972
:1079600080F855C0D34480F8563001238163856583
:107970000390C3870A2385645846029934F0EEF8D1
:10798000002840F08980039DEB8F9BB2FF2B40F2D3
:1079900087806969FF235748AB874B68564A034085
:1079A000029803431A434A6009EB06030AEB4315A6
:1079B000039304E0EB8F9BB2002B00F082803A46E9
:1079C0000A2158462FF008FF40BBA96B686911F8DF
:1079D000012BAB8F8262A963013BE98F9BB2013916
:1079E000AB8789B2E987E98F89B2002BE2D1002900
:1079F000E0D01EE00124FFF731FF65E74E4420216F
:107A000000220AEB461ADAF858308AF854200B4361
:107A1000CAF858308AF855108AF85620374A138821
:107A200001339BB213804FE7D8F80020D21B0A2AFB
:107A300021D8836913F08003F6D0EB8F9BB2FF2B24
:107A40000AD943682B49029A0B402B491343194327
:107A5000FF23AB874160ADE7EB8F029A9BB2416891
:107A6000AB87DBB242EA0343224A11400B4343F0A7
:107A7000007343609EE74E44184620220AEB461AE4
:107A8000DAF858308AF854001343CAF858308AF8A4
:107A900055208AF85600C1E7039B83F85450BDE790
:107AA000039A0299D38F13489BB29387DBB2526932
:107AB00041EA0343516801400B4343F000735360B4
:107AC00072E73946584634F0B9F90028A6D16A69F8
:107AD00020260B4CD661039B51680AEB43132140CF
:107AE0000124516085F8556083F8540085F85600EC
:107AF000EAE600BF009C00FC0000FF0144220120D8
:107B000000E800FEC02001204022012010B592B004
:107B10008C46044609920DF107020A930023039252
:107B2000012203A98DF807C005928DF82C208DF84D
:107B3000402004938DF818301193CDE90733CDE937
:107B40000C33CDE90E33FFF759FE2268136A002B80
:107B5000FCD112B010BD00BF30B5056883B095F8F8
:107B600000E0BEF1010F07D0BEF1020F01D12C6A77
:107B700074B1002003B030BD844614460A4695F91E
:107B800004009CF804100094F1F74EFF03B030BDE0
:107B900041F08001FFF7BAFF0120EBE72DE9F04F3C
:107BA000066885B096F80080B8F1010F0BD0B8F1E7
:107BB000020F03D1346A002C00F0C6800026304644
:107BC00005B0BDE8F08F96F90490B9F1030FD4BF6A
:107BD00000260126B9F1FF3F08BF46F00106002E3E
:107BE000ECD11746DFF85CA209EB49021D464FEACB
:107BF000490E0AEB42125369002BE0D0044692F87A
:107C00005500202840F0B5801FFA85FC002D00F0BB
:107C1000B68092F85400012800F0AB802079824CA5
:107C200082F85480256804E02268521B192A00F269
:107C3000C5809A6912F40042F6D10EEB090B90460A
:107C40000A4643004FEA4B1B00954FF0220E40209E
:107C50000BF11401D34403930A23CBF838700AEBD9
:107C600001078BF855E003998BF856003846CBF89E
:107C70005880CBF84880ABF83EC034F0A1F84FEA0A
:107C8000490E002840F0BA80BBF83E309BB2FF2B73
:107C900040F2B780DBF81410FF236448ABF83C30A7
:107CA0004B68634A0340039803431A434A600EEB50
:107CB000090B604A4FF0FF0C07EE907A0AEB4B1865
:107CC0000399D8F8140003E027687F1B0A2F41D8D6
:107CD000836913F00403F7D0406AD8F8383018707D
:107CE000B8F83E30B8F83C00013B01389BB280B296
:107CF000A8F83E30D8F83830A8F83C000133C8F86E
:107D00003830B8F83E309BB20BB100283BD0B8F801
:107D10003E309BB2002BD4D1294617EE900A34F0A6
:107D20008DF830BBD8F814302021434C0AEB4B1AA5
:107D3000D96101265A6822405A6088F855108AF89D
:107D4000540088F856003AE741F080010126FFF719
:107D5000DDFE34E7CE4420210AEB4E1ADAF8582033
:107D60008AF854300A43CAF858208AF855108AF81D
:107D70005630324A138801339BB213801FE74FF409
:107D800000739365F5E7D8F8140003E027687F1BBC
:107D90000A2FDFD8836913F08003F7D0B8F83E309C
:107DA0009BB2FF2B1BD94368A8F83CC013400B4380
:107DB00043F0FF7343F480334360A8E7CE442021AF
:107DC00000220AEB4E1ADAF858308AF854200B4396
:107DD000CAF858308AF855108AF85620C9E7B8F81A
:107DE0003E3047689BB21740A8F83C30DBB241EA0E
:107DF00003433B4343F00073436088E78BF85480B0
:107E0000B7E7BBF83E30039A9BB2DBF81410074883
:107E1000ABF83C30DBB242EA03434A68024013430A
:107E2000074A1A434A6042E740220120009800FCBA
:107E30000024FF81009C00FC00E800FE4422012099
:107E400000240082C020012030B5002393B001221D
:107E500004468DF818300DF1070511938DF80710C1
:107E600003A90A928DF82C208DF840200395CDE9C6
:107E70000432CDE90733CDE90C33CDE90E330DF1F2
:107E80000B030993FFF7BAFC2268136A002BFCD19D
:107E90009DF80B0013B030BD036810B59B68044615
:107EA00098470122FF236273A37310BD036810B5C6
:107EB00004461B6898470121236820469B68984721
:107EC000E37B0133E37310BDF0B583B004460D4688
:107ED0001646089F0193384638F0FCFE2168284476
:107EE0003246E672A07220468E692946019BB4464E
:107EF00003B0BDE8F040604703689B6A184700BFC5
:107F000003685B6D03B11847704700BF0368DB6C03
:107F100003B11847704700BF002310B5C373044670
:107F200042748A6C016003730AB119469047236852
:107F3000012120469B689847FF2123680122A173F5
:107F4000DB6C62731BB12046BDE81040184710BDC2
:107F500070B54FF6FF7C0E4D0E4C4FF0010E0E49E2
:107F60000E4E00234CFA03F20EFA03F0013312F026
:107F7000010F03D00C60083121F8040C102BF1D153
:107F800004F58064B44202D035F802CFE9E770BD51
:107F90004C3F0508000002409424012000180240D4
:107FA00010B50409013C052C16D80D4A00F00F034A
:107FB00032F8141041FA03F212F001020ED001203F
:107FC00098400138084039F0B1FB064B064A1B5D6A
:107FD000184402EBC00010BD002010BD104610BDBB
:107FE0004C3F0508583F050894240120F8B50B4F75
:107FF00097F8343083B10A4C0025A66801353079F2
:10800000FFF7CEFF18B1217DF279F2F717F997F853
:108010003430A034AB42F0DC0120F8BDB01E0020AB
:10802000FC07002038B50C4605460078FFF7B8FF7E
:10803000611C0446C9B210B14123C171837120464D
:108040006978F2F779FCAB7820461BB1BDE838407F
:10805000F1F7EEBEBDE83840F1F7F0BE0D4B2DE96B
:10806000F04105461F6800240B4EA74201DCBDE825
:10807000F08104EB4403F05C03EB0608FFF790FF8C
:10808000854204D121464046BDE8F041CAE70134AB
:10809000EBE700BF4065012010650120054B53F858
:1080A000203033B11A689B8851690B4218BF1B04FA
:1080B000936170478C1B01200E4B012210B40E4CB3
:1080C00093F800C002FA00F354F8200003EA0C030E
:1080D00051B1003B18BF012318B1016882883BB140
:1080E0008A615DF8044B7047B3FA83F35B09F3E7E9
:1080F0001204F5E7981B01208C1B012070B5392074
:1081000086B0FFF74DFF054610B140F23E23C38015
:10811000124C4FF4007102220026236B104843F0EA
:1081200004032363236B059603F0040300930323E6
:10813000CDE9011201A9009ACDE903632FF0EEF910
:10814000A36832460E2123F07843284643F0E043EB
:10815000A36006B0BDE87040F2F73CB900380240B9
:108160000008024010B5054C23681B699847236836
:10817000002283F836209A6310BD00BFBC27002080
:1081800010B5084C236893F8352012B1DB68984786
:1081900000B910BD044A01212368126883F8361023
:1081A0009A6310BDBC270020841B01200D4A02EBFE
:1081B000C00310B593F810E193F811418EEA010C59
:1081C000644500D110BDD3F80C31C0002BB11C6840
:1081D0008E459B8808BF1B04A361104480F811C121
:1081E00010BD00BFC0770120F8B5114E0124114D1C
:1081F000522716F8010BFFF7D3FE0022202118B1F9
:10820000C4718771F2F71AF815F8010BFFF7C8FE71
:108210004FF0530C0022402120B1C47180F806C0F9
:10822000F2F70CF80134E4B2052CE2D1F8BD00BF3E
:10823000C0730120B473012003681B68184700BF96
:1082400003682DE9F0415F6A1FB13B46BDE8F0418C
:10825000184704460D46164600E023689B682046F2
:108260009847B042F9D3002E08DD2E4423682046FB
:1082700015F8011B1B689847AE42F7D1BDE8F081A5
:1082800003685B68184700BF03689B68184700BF16
:108290000368DB68184700BF03685B69184700BFC5
:1082A00003689B6A03B11847704700BF0368DB6A25
:1082B00003B11847704700BF03689B6A10B50446B6
:1082C00082B023B1CDE900129847DDE900122046C3
:1082D000FFF7B6FF2368DB6A23B1204602B0BDE892
:1082E0001040184702B010BD70B504460E46154642
:1082F000236820469B689847A842F9D32A4631460E
:108300002046BDE87040D7E7014B1868F3F754BE2C
:10831000EC1E0020014B5868F3F74EBEEC1E002007
:10832000014B9868F3F748BEEC1E0020014BD8685B
:10833000F3F742BEEC1E0020014B1869F3F73CBE78
:10834000EC1E0020014B5869F3F736BEEC1E0020EE
:10835000154B1B885BB9154A154B12781B688AB1FF
:108360007BB11A689B8800B91B0493617047114B5D
:10837000D3F840212AB150B9D3F82C21106083F8EA
:108380003D01704780F00100002BEAD1F9E7B3F816
:1083900044C10121084AD3F82C01B2FBFCF20A4186
:1083A000026083F83D117047EE640120F4640120FF
:1083B000F0640120C077012040420F0030B4EFF399
:1083C0001183102282F312880B484FF0E0210B4DED
:1083D000DBB202680A4C013202608A692A6000221C
:1083E000C4F848210A6983F31188064A13680133E7
:1083F00030BC1360704700BF841B0120601C01204B
:10840000C07701204022012010B4EFF31181102326
:1084100083F312884FF0E0229469136913F4803FCC
:108420000D4B03D00120C3F8480194690B4AC9B22F
:108430001068D3F8482181F31188094B02444FF4A6
:108440007A70196800FB01F31B1B5DF8044BB3FB4A
:10845000F1F300FB02307047C0770120841B01203C
:10846000641C0120124B5B68C3F30803F3B9EFF3FC
:108470001183DBB90F4A4FF0E02C10B40E4C136897
:10848000DCF8180011688B42F9D121688842F6D8CF
:108490000A4A4FF47A71146801FB04F2121AB2FB13
:1084A000F4F25DF8044B01FB03207047ACE700BF1A
:1084B00000ED00E0841B0120601C0120641C0120F1
:1084C0002DE9F0411F4C40F2DC57DFF89080236823
:1084D0001D4D1B6B98471D492368002288781C4955
:1084E00083F836209A63032898BF0F4683F8352017
:1084F000FFF7B8FF174C0646D8F80430C3F308035B
:10850000EBB9EFF31183D3B94FF0E02128688A6902
:108510002B689842FAD123689A42F7D80E4B4FF451
:108520007A71D3F800C001FB0CF39B1AB3FBFCF388
:1085300001FB0030831B9F42DED8BDE8F081FFF7CE
:1085400063FFF7E7BC270020841B0120682401207B
:10855000FCA60700601C0120641C012000ED00E067
:1085600038B51A4B05460C465B79012B29D1184BBF
:108570001B6833B30846F9F7DFFE70B92046F6F7FB
:108580007BFF00F543730446B3F5C36F08D9284653
:108590001049BDE83840F9F724B80F4BB3F94C4106
:1085A0000E48F8F70DFA0E48F8F7E4F9F8F7C6F9AF
:1085B0000C4B186803F00CFDFFF782FF2046F5F71F
:1085C00027F80948BDE83840F8F7FAB9442B0120EC
:1085D0004C1B0120E0120608C0770120F8120608A3
:1085E000F40D0608D44F0120181306082DE9F041B8
:1085F0000746DFF86880FFF735FF154C154D064636
:10860000D8F80430C3F30803F3B9EFF31183DBB9EF
:108610004FF0E02C2368DCF8181022689342F9D15F
:108620002A689142F6D80C484FF47A72D0F800C00C
:1086300002FB0CF0401AB0FBFCF002FB0300831BB2
:10864000BB42DDD3BDE8F081FFF7DEFEF7E700BFF8
:10865000841B0120601C0120641C012000ED00E04F
:108660002DE9F04F9D4C85B0267816B905B0BDE8D0
:10867000F08F04461546984603B3012BF6D1984E69
:10868000326892F836202F2D88BF42F00102002A6E
:10869000ECD13AF0B5FF0028E8D16A1E3768142AF9
:1086A00063D8DFE802F05D5D5D5D5D621F1F1F1F27
:1086B000621F1F1F62626262621F1F00884E326863
:1086C00092F836000028D1D0926B002ACED085488F
:1086D00002F6B83200682F2D98BF82422CBF0122CB
:1086E0000022D4E74FF47A7303930A230193B8F17D
:1086F000010F5AD0B8F1000FB8D17B487B4A90F8EF
:1087000000C016780CF1010202F00302B242ADD0B3
:1087100002700CEB4C02764E4FF47A70019B4FEADC
:108720004C0E06EBC2021373906021B34346A4F1D2
:10873000FF0818200A46B8FA88F800FB0C604FEAD8
:1087400058180C304146904605E039B9013300F81D
:10875000012F43450FD09C420A46F6D12A46F5E741
:10876000644B039301230193C1E74FF47A7303939E
:1087700001230193BBE797F83400002800F09E80A6
:1087800000235D4C1A4602E0904200F0978034F8D6
:108790001310013250330029F6D00EEB0C030022E7
:1087A000DB00F118F2544A6060E754494A7C012A20
:1087B00000F09080022A00F0A3800023029397F833
:1087C0003400F8B1494BA4F1FF0C18211A78BCFA17
:1087D0008CFC0C234FEA5C1C11FB0231444BE64637
:1087E00084461944002370461A4606E040B9013316
:1087F00001F8012FDAB2944504D9A2420246F5D11C
:108800002A46F4E7DFF8F0A0A04642F22830FFF74E
:10881000EDFE4FF47A70FFF7E9FE029B0BB9FB699E
:1088200098473B6A03B19847336893F83430FBB1FB
:10883000A8F1FF044FF0000B4FF00109B4FA84F4E3
:108840005846640900EB8003804529460AEB431330
:1088500083F80290BB6A01D004B9214698470BF116
:10886000010B33685FFA8BF093F834308342E9D818
:10887000BB6903B19847FB6A9847029B0BB1FB6940
:108880009847019B013B13F0FF030193C1D103986B
:10889000FFF7ACFE336893F83420002A3FF4E6AECD
:1088A00012490D2018230C78019913FB040310487A
:1088B000184405B0BDE8F04F3AF004BD0EEB0C01D2
:1088C000012342F21070C900735431443AF09CFE07
:1088D0004860CBE6CDF8088071E700BFB4600120A6
:1088E000BC270020841B0120681C01205C1C012087
:1088F000FC1B0120A0860100FC0700206824012049
:108900008B78083B18BF0123029358E72DE9F04FFD
:10891000DFF8F48183B0784AD8F8043014780191F4
:108920002BB19A88A507196858BF12048A61D8F834
:1089300000202AB19188E407156848BF0904A9619D
:1089400001386E4E6E4CC7B26E4DDFF8C0B133B118
:1089500019689B884869034218BF1B048B6132B1B8
:10896000116893884A69134218BF1B048B61012068
:10897000DDF804A0FFF7ECFC7368C3F30803002BD9
:1089800040F0AE80EFF31183002B40F0A9804FF050
:10899000E0202368816922689342FAD12A689142D3
:1089A000F7D8DBF800C04FF47A7000FB0CF2511AD4
:1089B000B1FBFCF100FB03197368C3F30803002B40
:1089C00040F08B80EFF31183002B40F086804FF056
:1089D000E02C2368DCF8180022689342F9D12A6859
:1089E0009042F6D8DBF800104FF47A7202FB01FED9
:1089F000AEEB0000B0FBF1F002FB0300A0EB0903BB
:108A0000B3F57A7FD8D3BAF1010AB5D1D8F80430DA
:108A100033B11A689B8851690B4218BF1B049361DC
:108A2000D8F8003033B11A689B8851690B4218BFDF
:108A30001B0493610020DDF804A0FFF789FC736834
:108A4000C3F30803002B4FD1EFF31183002B4BD15D
:108A50004FF0E0202368816922689342FAD12A68A6
:108A60009142F7D8DBF800C04FF47A7000FB0CF2AB
:108A7000511AB1FBFCF100FB03197368C3F308033F
:108A800043BBEFF311832BBB4FF0E02C2368DCF8E2
:108A9000180022689342F9D12A689042F6D8DBF890
:108AA00000104FF47A7202FB01FEAEEB0000B0FB47
:108AB000F1F002FB0300A0EB0903B3F57A7FDCD3EE
:108AC000BAF1010ABBD1013FFFB2FF2F10D0D8E9A4
:108AD00000233CE7FFF798FCEDE7FFF795FC8DE7F7
:108AE000FFF792FC814667E7FFF78EFC8146C4E7FB
:108AF00003B0BDE8F08F00BF981B012000ED00E03F
:108B0000841B0120601C01208C1B0120641C01209F
:108B10002DE9F843284F451E284C294EDFF8A48044
:108B20007B68C3F30803002B42D1EFF31183002BC2
:108B30003ED14FF0E0202368816922689342FAD148
:108B400032689142F7D8D8F800004FF47A7202FBED
:108B500000F9A9EB0109B9FBF0F902FB03997B6865
:108B6000C3F308030BBBEFF31183F3B94FF0E02C11
:108B70002368DCF8181022689342F9D132689142D8
:108B8000F6D8D8F800C04FF47A7202FB0CF0401A05
:108B9000B0FBFCF002FB0300A0EB0903B3F57A7F06
:108BA000DDD3013DBCD2BDE8F883FFF72DFCF3E730
:108BB000FFF72AFC8146D2E700ED00E0841B01208C
:108BC000601C0120641C012001302DE9F84F594E32
:108BD00001F1FF38584CC7B2584DDFF864A132217B
:108BE00005204FF4FA79FFF791FE7368C3F3080389
:108BF000002B40F09680EFF31183002B40F0918022
:108C00004FF0E0202368816922689342FAD12A68F4
:108C10009142F7D8DAF800004FF47A7202FB00FBB9
:108C2000ABEB010BBBFBF0FB02FB03BB7368C3F3B5
:108C30000803002B72D1EFF31183002B6ED14FF09C
:108C4000E0202368816922689342FAD12A68914220
:108C5000F7D8DAF800C04FF47A7202FB0CF0401A31
:108C6000B0FBFCF002FB0300A0EB0B03B3F57A7F33
:108C7000DCD3B9F10109B8D1FA2138464FF47A7939
:108C8000FFF744FE7368C3F30803002B4DD1EFF3E5
:108C90001183002B49D14FF0E020236881692268BD
:108CA0009342FAD12A689142F7D8DAF800004FF4DB
:108CB0007A7202FB00FBABEB010BBBFBF0FB02FB90
:108CC00003BB7368C3F308032BBBEFF3118313BB20
:108CD0004FF0E0202368816922689342FAD12A6824
:108CE0009142F7D8DAF800C04FF47A7202FB0CF028
:108CF000401AB0FBFCF002FB0300A0EB0B03B3F542
:108D00007A7FDED3B9F10109BCD1B8F10108BFF413
:108D100066AFBDE8F88FFFF777FBEEE7FFF774FB70
:108D2000A2E7FFF771FB834680E7FFF76DFB834601
:108D3000C7E700BF00ED00E0841B0120601C01209C
:108D4000641C012038B5094C04F5407502E0083474
:108D5000AC4209D0A279002AF9D12046083420215A
:108D6000F1F76CFAAC42F5D138BD00BF9424012074
:108D70000023194901E0152B28D003EB43020133EE
:108D800011F802C00A448445F5D130B45478F8B1E2
:108D9000B4FA84F35B09DCB1104D10214FF0010CE3
:108DA0002A4603E001334E2B12D01179884202F19A
:108DB0001C02F7D10CF1010164455FFA81FCF1D18D
:108DC000C3EBC30305EB830030BC70470020704742
:108DD000002030BC704700BF482201209C4005089D
:108DE0002DE9F04F3B4C0025064688463A4FDFF808
:108DF000F8B0DFF8F090DFF8F4A02178607851B394
:108E0000B0FA80F35B0930B3334A4FF0100C4FF0E7
:108E1000010E04E001334E2B1DD092F804C06145D1
:108E200002F11C02F6D10EF1010C70455FFA8CFEC6
:108E3000F0D1C3EBC301DA0057F82110890AA1F57C
:108E40008011522934D819F801100D2930D81AF997
:108E500001108E422FD001350334152DCDD11F4B7B
:108E60001D68002D32DD1E4A00211E4FDFF87CC038
:108E700004E0013102F586728D4227D09068002807
:108E8000F7D0036800249B0AA3F58013522B04D863
:108E9000FB5C0D2B98BF1CF90340A642E9D1437936
:108EA0004345E6D192F80831002BE2D0BDE8F08FBF
:108EB00000218E42CFD1D01A07EB80004379434581
:108EC000C9D11BF81530002BC5D0EFE70020BDE855
:108ED000F08F00BF482201209C400508CC010020F3
:108EE000D0010020543A0508107901202CB705085C
:108EF000F0B5DFF8A8E00025234F06469EF80000F5
:108F00009EF80140E0B1B4FA84F35B09C4B11E4A93
:108F100010214FF0010C03E001334E2B10D01179DA
:108F2000884202F11C02F7D10CF1010164455FFA9D
:108F300081FCF1D1C3EBC30307EB83039E421DD039
:108F400001350EF1030E152DD8D1104B1C68002CE5
:108F500018DD0F480023024602E00133A34211D07E
:108F6000916802F586720029F7D08E42F5D14FF450
:108F7000867202FB030000F58470F0BD054800EB2B
:108F80004500F0BD0448F0BD9C400508CC01002020
:108F9000D001002010790120948605084822012084
:108FA000F8B5B8B316460F4600231D4A01E0152B4D
:108FB00030D003EB430C5D00013312F80C109444E5
:108FC0008142F4D19CF80140BCB1DFF85CE0102292
:108FD00001210023F44604E001334E2B1DD09CF800
:108FE000042090420CF11C0CF6D14A1C8C42D1B2E8
:108FF000F2D1C3EBC3030EEB83042046FFF778FFE7
:1090000003783BB9074B20461D4485F8507185F81D
:109010005161F8BD00242046F8BD0024EDE700BFF3
:1090200048220120C07701209C40050870B5054604
:1090300082B00E4600222B21FFF7B2FF04462846DD
:10904000FEF7AEFF00B10CB902B070BD0F4D2B2280
:109050000221C5F84001C280E279F1F7BBF90C4A60
:10906000A5F844612146002405F59670B2FBF6F39D
:10907000C3F34F0601949BB20096F2F723FBD5F899
:109080002C311C6085F83D41DEE700BFC077012030
:1090900040420F000C4B30B593F83B20002A0B4A9E
:1090A00014BF0121002111700CD0094C03F12005DF
:1090B0001A46083403CAAA4244F8080C44F8041CAF
:1090C0001346F5D130BD00BF546001208C4F012004
:1090D000904F01202DE9884801210220FEF7ECFF86
:1090E000604B1B7803F00503052B00F0B7800021CF
:1090F0000120FEF7E1FF00215B4C4FF0E0265B4DC5
:109100004FF47A77DFF86CB10846DFF86CA1FEF710
:10911000D3FF4FF4FA78DAF80430C3F30803002BD6
:1091200040F09880EFF31183002B40F09380236888
:10913000B16922689342FAD12A689142F7D8DBF8E4
:10914000000007FB00F2521AB2FBF0F207FB032902
:10915000DAF80430C3F30803002B74D1EFF3118362
:10916000002B70D12068B16923689842FAD12B682E
:109170009942F7D8DBF8002007FB02F35B1AB3FB38
:10918000F2F307FB0030A0EB0903B3F57A7FDFD3DE
:10919000B8F10108BFD1364B9B6833B11A689B8880
:1091A00051690B4218BF1B0493614FF03208DAF883
:1091B0000430C3F30803002B48D1EFF31183002BD5
:1091C00044D12368B16922689342FAD12A68914256
:1091D000F7D8DBF8000007FB00F2521AB2FBF0F2FE
:1091E00007FB0329DAF80430C3F3080343BBEFF3AA
:1091F00011832BBB2068B16923689842FAD12B6890
:109200009942F7D8DBF8002007FB02F35B1AB3FBA7
:10921000F2F307FB0030A0EB0903B3F57A7FE1D34B
:10922000B8F10108C3D1124B9B68002B3FF471AF1A
:109230001A689B8851690B4218BF1B04936168E749
:10924000FFF7E2F8E7E7FFF7DFF89CE7FFF7DCF866
:109250008146C7E7FFF7D8F8814679E715F082FA2B
:1092600045E700BFA8640120841B0120601C012089
:109270008C1B0120641C012000ED00E02DE98848D2
:1092800001210020FEF718FF01210846FEF714FF18
:1092900001210220FEF710FF434B1B7803F005036A
:1092A000052B7DD00021414C414D4FF0E027084671
:1092B000DFF804B1FEF700FFDFF800A10021012074
:1092C000FEF7FAFE00210220FEF7F6FE4FF032080C
:1092D000DAF80430C3F30803002B5DD1EFF31183F8
:1092E000002B59D12368B96922689342FAD12A68C0
:1092F0009142F7D8DBF800004FF47A7202FB00F6D7
:10930000761AB6FBF0F602FB03664FF47A79DAF8C8
:109310000430C3F30803002B3BD1EFF31183002B80
:1093200037D12068B96923689842FAD12B689942ED
:10933000F7D8DBF8002009FB02F35B1AB3FBF2F36A
:1093400009FB0030831BB3F57A7FE0D3B8F1010845
:10935000BED1184B1B6833B11A689B8851690B4208
:1093600018BF1B049361134B5B6833B11A689B8869
:1093700051690B4218BF1B0493610E4B9B68002B75
:10938000A4D01A689B8851690B4218BF1B049361D3
:109390009CE7FFF739F8D5E7FFF736F80646B4E75C
:1093A00015F0E0F97EE700BFA8640120841B0120CE
:1093B000601C01208C1B0120641C012000ED00E0DA
:1093C0002DE9F0470928664D2C6801D03F284ED181
:1093D0004FF00008634EDFF890A14746DFF8AC91EC
:1093E0002CB1224631685046F5F752FF10B9B0460D
:1093F00007B9374610364E45F2D3F7B1D7F800C05B
:10940000D8F800E058492B681CF803601EF80300E8
:10941000B04212D15A1C68B9FD2B0BD820262A6005
:10942000CE54885447450BD14F4E2B68A34219D8D0
:10943000BDE8F087CE542A60E5E72B68002BF1D118
:109440004A48F7F797FA474504D949480024F7F7FF
:1094500091FAE9E757F8100BF7F78CFA0920F7F7BC
:10946000BBFAF0E7305D0134F7F7B6FADDE73CB957
:10947000042805D13C493F48BDE8F047FCF744B813
:109480000C2804D13C48F7F775FA394809E07F28E1
:109490000BD1002CCCD0013C334B002237482C6040
:1094A0001A55BDE8F047F7F765BA002C47D00A28EF
:1094B00001D00D2840D12C4CF7F764FA2321204627
:1094C0003AF007F808B1001B28602B6800227BB92E
:1094D00002B12B604FF480720021234839F0F2FE74
:1094E000274B1B78002BA3D0CFE701220B46EEE7DA
:1094F000591E605C2028F8D002B12B6000223A2669
:10950000DFF86480E254174C276840463946FBF781
:10951000C5FD014640B9013E04F11004F4D11949DA
:109520001948F7F743FF05E0184B9C42F7D2E36870
:10953000384698470023CCE7FF2C3FF679AFA0F1DF
:1095400020035E2B3FF674AF14B920283FF470AFB0
:10955000631C2B60044B1855BDE8F047F7F73CBA85
:10956000146A0120F48205081269012045130608D7
:1095700059FC0508591306084B130608561306082C
:10958000186A01205A1306087613060894860508FF
:109590001A4B1B78222B1BD0194B1B782BB9194B5C
:1095A000187900F0010031F05FBE174B1B6823B340
:1095B00010B5164CF7F7C2F904E02068FEF768FE14
:1095C000FFF7FEFE2068FEF75BFE0028F5D110BD18
:1095D0000C4BD3F87C3133B119689A880B691A4265
:1095E00014BF012300230A4A0A4992F874220B800F
:1095F000531E18BF01234B80CEE77047E51B0120A7
:10960000186A0120C077012054580120D44F01204E
:1096100098280120E81B01202DE9F04F80468BB0EF
:1096200008460D4637F056FB024660B3A34928466C
:10963000F5F72EFE044630BBF7F7A4F9A04DA1487C
:10964000A14FF7F7B7F9A14E1420DFF8CC8230F024
:109650003FFAE11004F0070238460131F7F7DEF96E
:109660002B7F6A7F56F823104AB19948F7F716FA0C
:1096700001342435102CECD10BB0BDE8F08F4046FE
:10968000F7F70CFAF4E7284605AA924939F0DCFD11
:10969000054620B901464120FCF75CFAECE78E490B
:1096A000F5F7D2FD20B98D494046F7F79AFFE3E779
:1096B0008B4E0827002431682846F5F7C5FD0028A1
:1096C00008BF3446013F06F11006F4D154B985496C
:1096D0002846F5F7B9FD28B12A4683494046F7F7F1
:1096E00080FFC9E7002005AA7A498DF8130039F0F8
:1096F000ABFD0646002C3AD080B1F5F7BDFE451E05
:1097000009D4A37A9D4206DAE2684AB1012303FA3A
:1097100000F0104204D132467449DFE7744EFAE794
:10972000E0880027F4F7B0FF724903970978D0E981
:109730000232002908BF1A46217A637A05FB0133F9
:1097400002EB030B12F903A005AA6249002039F0CD
:109750007BFD8146A0BB0123674944B39BF90020F0
:109760002046CDE900312946FBF7A8FF84E768B120
:109770000DF11301FBF7E6FD28B19DF813502846C3
:10978000FEF70EFC20B932465C49A7E7584EFAE7CF
:109790002846A346F0F798FB82462846FCF7AAF82D
:1097A000039028462546FFF7E3FA0746CCE7CDE9C4
:1097B0000031524639469DF81300FCF787F95BE704
:1097C0004549F5F741FD064658BBACB1EDB24C4FEB
:1097D00072B229462079F0F74BFB00283FF44CAFDA
:1097E000028831460378384601360093C2F30323DA
:1097F000120BF7F753F9EBE7414C72B279793868FD
:10980000F0F77EFB00283FF437AF0288314603783B
:10981000204601360093C2F30323120BF7F73EF9FB
:10982000EBE738494846F5F70FFD10B34846F5F722
:1098300023FE064642B26CB1E9B22079F0F718FB7C
:10984000C8B9CDF800906B1C22682F494046F7F745
:10985000C8FE11E779793868F0F752FB58B99DF8DE
:1098600013302A491A09CDF8009003F00F03403253
:10987000ECE74FF0FF3606AF30463946FBF78AFD7E
:1098800008A95046FBF786FD564547D076B24CB145
:109890008BF8006008AB00976A1C21681C48F7F73A
:1098A000FDF8E9E69DF81320039B110919489E7005
:1098B00002F00F0208AB40310097F0E77C13060876
:1098C000800001208113060897130608B852050886
:1098D0000A150608CD0A0608BA000608A8130608E5
:1098E000D0030120BC130608C0130608CF130608D6
:1098F00059130608D84F01208D090108DF13060807
:10990000F1130608F00306081214060835140608B9
:109910005D140608801406083100060834B108AB4F
:109920006A1C21680648F7F7B9F8A5E69DF81320E8
:1099300008AB0448110902F00F024031F3E700BF01
:10994000A8140608C31406082DE9F04F07468DB089
:1099500008460D4637F0BEF9024630B901460120EF
:109960000DB0BDE8F04FFCF7E1B903902846AF49D0
:10997000F5F78EFC039A30B9AD4938460DB0BDE815
:10998000F04FF7F72EBEAB492846F5F781FC0446A9
:10999000002859D1F6F7F6FFA74FA848DFF8DCB248
:1099A000F7F708F8DFF8D882172030F091F817F9A8
:1099B000015B002D3AD029465846F7F72FF80022D0
:1099C000DFF894921346DFF884A2990028460592A6
:1099D00089B20493FFF704FA0390FFF789FA049B16
:1099E00001785E1C059AB9B11AB90490F6F7CAFF5E
:1099F0000498039B41789A79037802F00202C1B17E
:109A00000091002A14BF4A46524658F82330314686
:109A10008B48F7F743F80122042E3346D5D112B90B
